:1000000000000420B1C70400D9C70400DBC7040006
:10001000DDC70400DFC70400E1C7040000000000E2
:10002000000000000000000000000000E3C7040022
:10003000E5C7040000000000E7C70400E9C70400AA
:10004000D9C60400BDB00400456D0000EBC7040034
:10005000EBC70400EBC70400EBC70400EBC70400C8
:10006000EBC70400EBC70400EBC70400EBC70400B8
:10007000EBC7040099690000EBC70400EBC704005C
:10008000EBC70400EBC70400EBC70400EBC7040098
:10009000EBC70400EBC70400EBC70400EBC7040088
:1000A000EBC70400EBC70400EBC70400EBC7040078
:1000B000EBC70400EBC704000000000000000000D4
:1000C000EBC70400EBC70400EBC70400EBC7040058
:1000D000615D0000EBC70400EBC70400EBC7040040
:1000E000EBC70400EBC70400EBC7040000000000EE
:1000F00000000000EBC7040000000000EBC7040094
:1001000000000000000000000000000000000000EF
:1001100000000000000000000000000000000000DF
:1001200000000000000000000000000000000000CF
:1001300000000000000000000000000000000000BF
:1001400000000000000000000000000000000000AF
:10015000000000000000000000000000000000009F
:10016000000000000000000000000000000000008F
:10017000000000000000000000000000000000007F
:10018000000000000000000000000000000000006F
:10019000000000000000000000000000000000005F
:1001A000000000000000000000000000000000004F
:1001B000000000000000000000000000000000003F
:1001C000000000000000000000000000000000002F
:1001D000000000000000000000000000000000001F
:1001E000000000000000000000000000000000000F
:1001F00000000000000000000000000000000000FF
:1002000010B5054C237833B9044B13B10448AFF350
:1002100000800123237010BD0004002000000000B6
:10022000A8F9070008B5034B1BB103490348AFF316
:10023000008008BD0000000004040020A8F90700A9
:10024000A3F5803A704700BF174B002B08BF134B34
:100250009D46FFF7F5FF00218B460F461348144AD1
:10026000121A6CF0A1F80E4B002B00D098470D4BE2
:10027000002B00D098470020002104000D000D48FD
:10028000002802D00C48AFF300806CF013F8200077
:10029000290000F05FFB6AF04FFC00BF000008007F
:1002A0000000000000000000000004200004002006
:1002B000B44301200000000000000000C36823F0E8
:1002C0004A0343F00803C360704770B5856804466D
:1002D0004DB1284650F8046B60F0E5F828464CF024
:1002E0008CFB3546F4E762682068920029466CF082
:1002F0005BF82346C4E9025553F8180B984201D025
:100300004CF07BFB204670BD8268002322B1117F38
:1003100012680B44DBB2F9E7C068B3FBF0F070473A
:100320002DE9F041B4B0054668460C465FF064FE26
:10033000114F04F110080226444512D0394602A894
:100340005FF07CFA026852F80C2C034613444FF01D
:1003500030019E605FF0DDFA14F8011B5FF094FB42
:10036000EAE703A928465FF02DFC68465FF0E4FE4B
:10037000284634B0BDE8F081BD0200002DE9F0410F
:1003800086B01D460C9B0093C36804460E469046FB
:1003900000F11001426804A859F05CF89DF8103093
:1003A000002B46D0059F012F1FD12646002346F87B
:1003B000183FA4460020A3684CF8080F63B31A6ADC
:1003C000B2FBF7F107FB1121D3F800E056F821202A
:1003D000DAB9A2681A60A36046F821C01A680AB1A7
:1003E00046F8203008467346E8E7B7F1005F01D3CE
:1003F00058F0D5FFBA00104603924CF035FB039A33
:10040000002106466BF0D0FFD3E712681A6056F859
:10041000212001461360E5E7234653F8180B984264
:1004200001D04CF0EAFAC4E90067B8FBF7F607FB25
:1004300016862368C5F8208053F82620B7005AB1E5
:1004400012682A6053F826301D60E368284601339D
:10045000E36006B0BDE8F081A2682A60A5602A6862
:100460003AB1106A6168B0FBF1F201FB120243F885
:10047000225004F10802DA51E7E72DE9F0479A46E5
:10048000036853F8214080460F469146E4B1256841
:100490002B6A9A450BD1D9F80420AB689A4206D151
:1004A00092B16968D9F800006DF0F2FD60B12E6874
:1004B0007EB1316AD8F80430B1FBF3F203FB1212BB
:1004C00097422C4603D000242046BDE8F0873546ED
:1004D000DEE73446F8E700002DE9F7430646174A01
:1004E0000D46D1E900014CF08BFA7368B0FBF3F8CC
:1004F00003FB1808044603462A4641463046FFF7E8
:10050000BCFF08B10068A0B924204CF0ADFA4FF050
:1005100000090746294640F8049B60F057F801237C
:10052000009322463B464146304687F81C90FFF731
:1005300025FF1C3003B0BDE8F08300BF07690FC77B
:1005400010B58EB06C4684E80F0004AA0023114653
:10055000013314F8010B02F8010B102BF8D108A895
:10056000FFF7DEFE08A90748FFF7B6FF9DF8403009
:10057000037008A85FF097FF0248FFF7C5FE0EB0B2
:1005800010BD00BF1C04002010B50E4C20464CF0DE
:10059000B5FA0D4A0D4920464CF02AFA0C4800F1F4
:1005A000180301224FF07E5103600023C0E90123AC
:1005B0000161BDE81040C0E90533034A0549C36045
:1005C0004CF016BA380400200000002055CD04007D
:1005D0001C040020CB020000094B1A8872B9094A9A
:1005E0001188094A1288C2F500608142C8BF81B2F1
:1005F000198019B10548104406F022BC704700BFAD
:100600003C060020400E00203E0E00203E0600204A
:100610000749084A0B8810880344C3F30A030B8078
:1006200005490B881B1A0B8000231380FFF7D4BFEA
:100630003E0E00203C060020400E00202DE9F04731
:10064000194FDFF86C9006460D464FF0000AB84689
:100650003C88B9F800001549C4F50064A4B2AC4266
:1006600028BF2C4606EB040C66450CD0B8F80030C9
:1006700016F801EBC218C2F30A02013301F802E0D6
:10068000A8F80030F0E72D1BADB25444FFF7A4FFEB
:100690001FFA84FA2DB106F0C3FB10B9FFF7B8FFBB
:1006A000D6E75046BDE8F087400E00203E06002009
:1006B0003E0E00202DE9F743354D2E880F46134698
:1006C000A846CEB90A4633484FF400616DF0D2FC1B
:1006D000B0F5006F044607D32F48394606F0F6FD03
:1006E000204603B0BDE8F0832C4B28801E802C4BA5
:1006F0001E80FFF771FFF3E7284A2648158801930B
:100700002E44C6F30A06B5428CBFAD1BC6F5006584
:10071000ADB2914630440A4629466DF0ABFC041E4A
:1007200004DA1D48394606F0D1FDE2E7A54205DDB1
:10073000B8F800302344A8F80030DAE7B4F5006FC9
:1007400022DAB8F800306BB1FFF746FF06F068FB1D
:1007500010B9FFF75DFFF4E706F07BFC0146114896
:1007600006F0B4FD019B0B483A464FF400616DF072
:1007700081FC041E00DCFEE7094AA8F800400023C3
:10078000A9F800301380B4E707483946CBE700BF2B
:10079000400E00203E060020B03107003E0E002033
:1007A0003C060020D1310700EA310700F8B52A4F96
:1007B0002A4C05464618AE424CD92B780D2B26D034
:1007C00011D8082B11D00A2B1DD02388B3F5FF7F39
:1007D00030D801212846FFF731FF23885A1C228098
:1007E00029781F4A0DE07F2BEFD1238813B3032113
:1007F0001C48FFF723FF2388194A013B9BB2238043
:100800000021D15416E0184B1B780D2B12D0022179
:100810003846FFF713FF238811490022581ECA5497
:10082000944601445BB902B123800D4801F09CFC61
:10083000002323800C4B15F8012B1A70BBE70878B6
:100840000A2801D00D28EED1013B01F801C99BB265
:100850000122E7E7F8BD00BF073207003A06002093
:100860003A0400200432070039040020FFF7D0BE0C
:1008700007B50A49019000230B8009490B800949FB
:100880000B8009490B8006F0CBF9019A0749104605
:1008900003B05DF804EB01F065BC00BF3A06002030
:1008A0003E0E0020400E00203C060020B506000051
:1008B000F0B5E5B004A9054606F0BCFB24A904A8E0
:1008C00006F08BFB8022002104A86BF06DFD012354
:1008D000114A8DF88C308DF88B30104B1A926A4685
:1008E000164603F1100718685968344603C40833E4
:1008F000BB422646F7D10FCA0CAC84E80F00012397
:1009000024A904A88DF8863006F07BFB24A928468C
:1009100006F01FFB65B0F0BDCDAB1A003232070008
:1009200030B5084689B014460D4606F0DAFC03AA35
:1009300001461323284606F0D8FC9DF80C3000939E
:1009400020696169A269E369FFF7FAFD09B030BD6A
:10095000704700002DE9F04F99B04B4E019088464A
:100960004FF0000941460198DFF834A105F00AFF75
:1009700006F071FB0446FFF77BFF2046FFF798FF68
:100980000121204606F082FB3422002130466BF024
:100990000BFD102200210EA86BF006FD40F2BC43B7
:1009A0003A4AADF8483031462346204607F022F84F
:1009B00001230EAA3146204607F035F801212046D2
:1009C00006F09AFE0025AB4605F006FF07462046D6
:1009D00017B106F04AFBC5E706F004FD204605F016
:1009E00001FFBB4508BF55454AD1262202AD394615
:1009F0000EA86BF0D9FC2946254806F09BFB95E82C
:100A00000F000DF1480C8CE80F0040F2BC43394652
:100A10002046ADF85A3006F0DFFF0546E0B11D4F25
:100A20003B78052B1BD11C4B06AA03F1200B9646E5
:100A3000186859689446ACE8030008335B45624681
:100A4000F6D120227146284606F04DFC87F800902A
:100A500050B1284606F03FFC0025AB46B4E70F49ED
:100A6000172206F040FCF3E70EAB2A46314620463B
:100A700006F0E3FF3B7801333B700028E9D1EBE758
:100A800001354BF1000B9FE7440E002021090000C7
:100A90002A320700420E002009320700040000201D
:100AA0008038010008B5034A0349083004F02DFDE1
:100AB000002008BD423207001B35070010B50C6846
:100AC00024B9806806F0D3FA204610BD2320FCE745
:100AD000803002F08FBA00002DE9FF410D68044616
:100AE0000E4685B908306549039004F00EFD64494F
:100AF000039804F00AFD6349039804F006FD2846B4
:100B000004B0BDE8F0815E49304623F0A1F9002829
:100B100043D07368002B32D154F8080F5A4EDFF8D7
:100B20008C8106F0AFFB594902680546204604F067
:100B3000ECFC10273368EB5800937368424604219D
:100B4000204604F0FFFC013F06F10806F2D16A6C72
:100B50004F49504EDFF85481204604F0D6FC102750
:100B60003368EB580093736842460421204604F032
:100B7000E9FC013F06F10806F2D10025BFE746492E
:100B8000301D23F065F908B90725B8E7B568002DD1
:100B9000FAD1A06806F07AFBB1E73A49304623F073
:100BA00057F900283FD0736883BB54F8080F3B4DBA
:100BB000DFF8FC8006F0D6FD092706462B686A6838
:100BC000F35A4146204604F0A0FC013F05F1080518
:100BD000F4D1334FDFF8DC8005257A6841462046A2
:100BE00004F0D4FB57F8083B3344D3E900232046F4
:100BF00004F018FC013DF0D120462A4904F0C6FB60
:100C0000D6E90E23204604F00DFC78E72249301D7A
:100C100023F01EF90028B7D0B568002DB4D1A06824
:100C200006F0ABFD6BE71549304623F011F90028BB
:100C3000AAD07368A3B954F8080F1B4DDFF86C8075
:100C400006F085FD042607462B686A68FB58414676
:100C5000204604F05AFC013E05F10805F4D18CE76A
:100C60000D49301D23F0F4F800288DD0B568002D13
:100C70008AD1A06806F06FFD41E700BFAB370700DF
:100C80004B3207004F3207009044070053320700F1
:100C9000683207001044070083580700A843070084
:100CA000104507008C320700F04307006032070050
:100CB000753207007C32070008B5806806F0DFF95E
:100CC000002008BD2DE9F0430E468BB0454905468E
:100CD000304623F0BDF8074600B1043633685BBBED
:100CE000A868414EDFF81881DFF8189106F0DEF9A8
:100CF0000446002C58D005F108002146039004F06A
:100D00009BFB0398A7B1637CA17C0390032BC1F3E9
:100D1000400198BF59F82320237C0191A17C01F068
:100D20000101009188BF4246314604F02FFB039831
:100D300004F03AFB6469DCE72C49304623F088F87C
:100D400098B1706804A923F058F858B9089BA868AE
:100D50009B0C9B0443F4403343F4507304A9089361
:100D600006F0ADF90BB0BDE8F0832149304623F021
:100D70006FF8044650B1706804A923F03EF80028CB
:100D8000F0D1A86804A906F09FF9EBE719493046AD
:100D900023F05EF8074648B155F8080F06F01EFC30
:100DA0000146284604F05AFB2046DBE7124930464C
:100DB00023F04EF8044648B155F8080F06F006FC3B
:100DC0000146284604F04AFB3846CBE70B4930463B
:100DD00023F03EF820B155F8080F06F0FBFBDFE7E3
:100DE0002320BFE7A1320700A4320700CD3207005D
:100DF0006D370700D1320700DB320700E032070011
:100E0000725A0700C041070030B585B0044602A9F8
:100E1000806806F048FC0546F0B904F10800029A23
:100E20000F49019004F071FB9DF80C200D490198C9
:100E300004F06BFB9DF80D200B49019804F065FB55
:100E40009DF80E200949019804F05FFB9DF80F20E2
:100E50000749019804F059FB284605B030BD00BF92
:100E6000E6320700F83207000D33070006330700AB
:100E70001E33070070B50C6886B005460E4664B98F
:100E800055F8080F02A906F064FD2846102202A9B1
:100E900004F0ACFA204606B070BD4B685BB9102276
:100EA00002A9204622F0B3FF0028F4D1A86802A9C5
:100EB00006F054FDEFE70B49304622F0C9FF70B150
:100EC000A868746806F096FB0190A86806F023FBFA
:100ED0000199024602AB204606F05EF8E4E70720DF
:100EE000D9E700BF33330700383002F0F9BF00F50F
:100EF000EA50103003F06CB870B5044680680E46B6
:100F000010F0FCFC054606F0BDF885420CD00849FF
:100F1000304622F09DFF48B104F1080005492A46F9
:100F200004F0F3FA002070BD0C20FCE70720FAE77C
:100F3000733707001B35070010B5044654F8080F37
:100F400006F0CCFB03490246204604F0DEFA0020FE
:100F500010BD00BFCE350700024B034A083004F035
:100F6000BBBB00BFD3770000C97700007FB50C463C
:100F700000232349ADF80E300546204622F068FFD5
:100F8000064610B1606800BB0434206838B30DF128
:100F90000D0122F0DBFE00BB9DF80D001F281BD8C1
:100FA0000124844005F10800DEB1164B164A0221E7
:100FB00004F002FB154BBDF80E20A86800952146F1
:100FC00006F070F948B9242007E00DF10E0122F077
:100FD000CEFE10B90834D8E7072004B070BD04462F
:100FE000E0E70B4B0B4A052104F0E6FA0A4BBDF88B
:100FF0000E20A8680095214606F04FF9E2E700BFF1
:10100000363307006142070054420700591F0000B1
:101010005C420700404207006122000010B500F169
:101020000804806806F07AFB044A0549002818BFC6
:101030001146204604F069FA002010BD3D33070038
:1010400042330700303002F075BC883003F0B0BB8B
:10105000403004F0C9B8096800686BF0BABA000003
:1010600038B50C68054608464CB906F00BF8094936
:10107000024605F1080004F048FA002038BD064990
:1010800022F0E6FE18B105494FF4C972F1E72320BA
:10109000F4E700BF1B35070048330700424507004F
:1010A00038B50C4605460949204622F0D1FE58B114
:1010B00064684CB906F008F90549024605F10800D4
:1010C00004F023FA204638BD0720FCE74C33070024
:1010D000B064070013B50C687CB90830084901906A
:1010E00004F054F90749019804F050F901980649B1
:1010F00004F00BFA204602B010BD2320FBE700BF2E
:101100005233070054330700D6F007002DE9F041B1
:101110000B68044694B008467BBB54F8080F1C4E7D
:10112000DFF8808002AF394606F0E7F8BDF8082006
:101130001849204604F0E9F9BDF80A20164920466E
:1011400004F0E3F9BDF80C201449204604F0DDF961
:1011500008253368FA182046516801915288009298
:10116000FB5A7268414604F0D0F9013D06F10806C9
:10117000EFD1002014B0BDE8F081094922F068FEEB
:1011800018B1A06806F0BBF8F3E70720F2E700BF4C
:101190000042070059330700633307006C33070030
:1011A000835807007933070037B5054608680DF105
:1011B000070170B9A86804F0CBFF044630B99DF967
:1011C00007200A4905F1080004F09FF9204603B002
:1011D00030BD22F003FE04460028F7D19DF9071028
:1011E000A86804F0C9FF0446F0E700BF9633070083
:1011F00037B50C68054674B955F8080F05F020FF9F
:101200000E494FF47A72B0FBF2F2284604F07DF9F1
:10121000204603B030BD4B686BB901A9204622F0CF
:1012200044FE0028F5D1019BA8684FF47A71594318
:1012300005F00AFFEDE70720EBE700BFF4320700F7
:1012400010B5044608460A4922F002FE30B10022D9
:10125000A0681146BDE8104006F094BA0549A068A0
:10126000224606F08FFA002808BF242010BD00BFD8
:1012700087330700311F00000B6837B505460C4661
:1012800083B980680DF1070104F08EFF044630B980
:101290009DF90720144905F1080004F036F92046AD
:1012A00003B030BD1149204622F0D2FDC8B16068BC
:1012B0000DF1070148B9A86804F076FF044600283C
:1012C000EDD19DF907200A49E5E722F087FD0446A4
:1012D0000028E4D19DF90710A86804F06FFF0446C8
:1012E000DDE70724DBE700BF8D3307009D330700F0
:1012F000B064070070B50E6804460D468EB954F808
:10130000080F05F0CFFE054628B120460F4904F02E
:10131000FCF8304670BD20460D4904F0F6F828462A
:10132000F8E70A49284622F093FD064628B1012134
:10133000A068BDE8704005F0A9BE0549284622F026
:1013400087FD08B13146F3E70720E3E7A53307003F
:1013500074F2070038B50D685DB9044654F8080FFB
:1013600005F07BFE04490246204604F0CEF82846EC
:1013700038BD0720FCE700BFF4320700F0B50B686A
:1013800085B005460E4663B955F8080F05F0A1FE75
:101390000446002C50D02146284604F05FF824690A
:1013A000F7E72749304622F053FD50B1706869468F
:1013B00022F023FD18B9A868694605F08EFE05B035
:1013C000F0BD2049304622F043FD50B170686946B7
:1013D00022F013FD0028F2D1A868694605F082FECC
:1013E000EDE71949304622F033FD074638B1174B77
:1013F000174A311D05F1080004F05CF9DFE71549D3
:10140000304622F025FD044648B155F8080F06F095
:10141000E9F80146284604F021F83846CFE70E499E
:10142000304622F015FD48B155F8080F06F0DEF8F9
:101430000146284604F012F82046C0E72320BEE704
:10144000CD3207006D370700A8330700F7700000A2
:10145000EF700000B4330700BA33070038B50D68E9
:101460005DB9044654F8080F06F030F90449024605
:10147000204604F04AF8284638BD2320FCE700BF88
:10148000F43207000B6837B50546084683B9A868EB
:1014900005F1080405F0D4FE10B1A86804F0F2FDCF
:1014A0000146204604F042F80024204603B030BD37
:1014B0000DF1070104F0C0F804460028F5D19DF8AD
:1014C00007201AB9A868114605F0B3FE9DF8071069
:1014D000A86805F0BBFE04460028E6D19DF8073059
:1014E000002BE2D00249A8682A4605F0A2FEDCE7FC
:1014F0007D1E00000B6837B505460C469BB9806819
:101500000DF1060105F0D8FE044648B9BDF80620E5
:101510009DF806300D49120A05F1080003F0F5FFA9
:10152000204603B030BD084622F08BFC02280AD1C9
:101530002368A8681A78597801EB022189B205F06E
:10154000B6FE0446ECE70724EAE700BFC033070015
:1015500070B50E6804460D4666B954F8080F06F0DB
:101560009CF806F09EF818490246204603F0CDFF8D
:10157000304670BD1549284622F06AFC20B1A068AB
:10158000BDE8704006F07AB81149284622F060FCA8
:1015900020B1A068BDE8704006F075B80D49284636
:1015A00022F056FC20B1A068BDE8704006F058B9A2
:1015B0000949284622F04CFC20B1A068BDE87040E3
:1015C00006F05FB90720D4E71B350700C5330700D5
:1015D000CE330700D4330700DB330700F8B50E46DF
:1015E00005461249304622F033FC074628B1012156
:1015F000A868BDE8F84006F07FB80D49304622F0F3
:1016000027FC044608B13946F2E70A49304622F081
:101610001FFC48B106F080F80749024605F10800B2
:1016200003F073FF2046F8BD2320FCE75D6207004E
:10163000E2330700733707004245070037B5054618
:1016400008680DF1070170B9A86804F077FD044639
:1016500030B99DF907200A4905F1080003F055FF4C
:10166000204603B030BD22F0B9FB04460028F7D174
:101670009DF90710A86805F03FF80446F0E700BFA1
:101680009633070030B50D68044687B008466DB93B
:1016900054F8080F1822694605F0EEFC0B496A461B
:1016A000204603F032FF002007B030BD084922F089
:1016B000CFFB48B154F8080F05F0DBFC02460B469F
:1016C000204603F0AFFEEEE70720EDE71B350700ED
:1016D000A949070010B50446006888470349024637
:1016E000204603F012FF002010BD00BF4245070056
:1016F0002DE9F0430D6895B004460E468DBB806819
:10170000DFF8908006F052F8A9460646AFB2BE4216
:1017100036D9A068ADF80E9008AA394606F0CBF885
:10172000E8B99DF84930C3F3C0021B0717D4ADF8E0
:101730000E20A06804AB0DF10E02394606F0C0F889
:1017400068B904F1080341461846BDF838200193F2
:1017500003F01CFE019804A903F080FEE9E70135BF
:10176000D4E70A49304622F073FB58B173685BB97D
:10177000074904F10800FFF7ADFF15B0BDE8F0839D
:101780000020FAE72320F8E70720F6E7B337070041
:10179000BF770000E73307002DE9F7430D680446E3
:1017A000002D38D100F10806284B294A294FDFF8CF
:1017B000AC80DFF8B0900321304603F0FDFEA06856
:1017C000E9B206F0F4F8F0B1A90201ABA0680DF19E
:1017D000060201F47C4106F0F0F839462A4630460C
:1017E00003F0D4FDBDF806204FF6FE739A421BBFEE
:1017F0009DF804301849194A920A04BF43464946E5
:10180000304603F082FE01353F2DD8D10025284611
:1018100003B0BDE8F083284601A922F0A8FA0546E6
:101820000028F4D154F8080FBDF804100DF103039B
:101830000DF1060206F0C1F89DF80330BDF8062050
:101840000749204603F061FEE1E700BF7042070050
:1018500064420700EE330700F73307001BA30700BD
:101860000F3407000334070073B50C6805460E46B5
:101870003CB10DF10701204622F0B0FA60B102B090
:1018800070BD55F8080F06F082F808490246284650
:1018900003F03BFE2046F2E773682BB99DF9071071
:1018A000A86806F078F8EAE70720E8E7B0640700E0
:1018B00037B50D686DB90446694654F8080F05F050
:1018C0007BFC20460822694603F090FD284603B0C1
:1018D00030BD0720FBE737B50C6805465CB955F805
:1018E000080F05F018FE08220146284603F07EFD89
:1018F000204603B030BD08226946204622F087FA10
:101900000028F6D1A868694605F009FEF1E7000055
:10191000F0B5044600F10805134B144A144F154E58
:101920008DB00221284603F047FEA06806F096F825
:101930000446B4B120463022694605F002FC6A46EE
:101940003946284603F022FD04F112003022694690
:1019500005F0F7FB6A463146284603F0D6FD246BB6
:10196000E7E720460DB0F0BD7C4207007442070057
:101970001E3407002734070037B50C6805465CB9EC
:1019800055F8080F05F000FC08220146284603F030
:101990002DFD204603B030BD08226946204622F0C6
:1019A00036FA0028F6D1A868694605F0F1FBF1E7A0
:1019B00030B50C6885B0054664B955F8080F69461E
:1019C00005F0E6FD28461022694603F00FFD20468B
:1019D00005B030BD10226946204622F018FA0028D2
:1019E000F6D1A868694605F0D8FDF1E730B50B6877
:1019F000044687B0084683BBA06801A905F072FEC3
:101A0000054638BB08341A49204603F0BFFC0822BB
:101A100001A9204603F0EAFCBDF80C201549204638
:101A200003F073FD9DF811201349204603F06DFD6E
:101A30009DF812201149204603F067FD9DF8132000
:101A40000F49204603F061FD9DF815200D49204601
:101A500003F05BFD284607B030BD0B4922F0F8F9D2
:101A600020B1A06805F043FE0546F3E70725F1E73E
:101A7000313407003C34070045340700593407006F
:101A80006E340700123307007734070073B50C6813
:101A900005460E4634B101A9204622F006FA60B18F
:101AA00002B070BD55F8080F05F0A9FB07490246C2
:101AB000284603F02AFD2046F2E7736823B901990E
:101AC000A86805F0A1FBEBE70720E9E7F43207007F
:101AD00030B50C4687B005462149204622F0B8F9BA
:101AE000A0B1201D0DF1170103F0A6FD044638B981
:101AF0009DF817303BB11B492A46A86805F050FFF6
:101B0000204607B030BD02460146F6E7206820B304
:101B10000DF1170122F01AF904460028F0D19DF8C2
:101B200017001F2817D8012181400F4B0193002374
:101B3000A868029500934FF6FF7205F0F4FD044685
:101B40000028DDD1094B0A4A072105F1080003F0FE
:101B500033FD2424D4E70724D2E70146E5E700BF9C
:101B60007E340700BD2100006122000034430700DD
:101B700018430700024B186800B9FEE7704700BF22
:101B8000780E0020037813F0010F0B461CBF722261
:101B900003F8012B0278920744BF642203F8012B5B
:101BA0000278520744BF6E2203F8012B8B4204BF18
:101BB0002D2203F8012B00221A70084670470000FE
:101BC0007FB50C68002305460E468DF804308CB9AD
:101BD00055F8080F05F0BCFC03A98DF8080002A811
:101BE000FFF7D0FF1E490246284603F08EFC204630
:101BF00004B070BD1B49304622F02AF938BB336867
:101C00000146013B044613F8012F5AB16E2A05D054
:101C1000722A05D0642A20D10124F4E70121F2E7D9
:101C20000120F0E728B19DF8043043F001038DF85E
:101C300004302CB19DF8043043F002038DF80430D9
:101C400029B19DF8043043F004038DF804309DF869
:101C50000410A86805F08BFCCAE70720C8E700BF9E
:101C60001B3507001BA30700F0B50446A1B00D46C5
:101C70000026227DF3B29A421BD92269284652F8E7
:101C80003310DF0022F0E4F801360028F1D0694675
:101C9000284622F0E6F82369A4693B4428465E689A
:101CA00022F0EAF80138C1B201AA2046B04721B0BB
:101CB000F0BD2320FBE770B5064600680C4608B966
:101CC000072070BD2F216AF077FB054688B104F12B
:101CD0000801013022F03AF80028F2D1227A013AC4
:101CE0003F2AEDD8287030682146BDE8704021F0C9
:101CF000D1BF1720E5E70000013002289ABF024B50
:101D000053F8200001487047283E0700F59C070063
:101D10002DE9F341804608680F4616461D46C0B1BE
:101D2000114622F06AF800232B70044668B1386827
:101D300001A922F067F840B9324601A9404605F0F2
:101D4000E6FA044608B901232B70204602B0BDE82C
:101D5000F0810724F9E7000038B50C4600F10805CA
:101D6000284603F069FB228A1D49284603F00EFB32
:101D7000A37C1C49032B96BF1B4A1C4A52F8232004
:101D8000284603F003FBE27C194902F001022846D1
:101D900003F0FCFAA37CE3B9E37C5B0714D5154997
:101DA0006269284603F0F2FA04F11801284603F0AC
:101DB00043FBA37C032B07D1E37C628D0E49C3F365
:101DC0004003284603F0E2FA2846BDE8384003F015
:101DD000EBBA228D0949284603F0D8FAE9E700BF9B
:101DE000CD3507001A350700B0410700725A0700C9
:101DF00093340700A0340700C0340700B434070050
:101E000010B500238EB0CDE901330446A06801AAC5
:101E100003A905F099FD20B903A92046FFF79CFF0F
:101E2000F4E700200EB010BD30B597B00B680093FA
:101E30008B88ADF804300E490E4B0F4D00F10804AD
:101E4000002A14BF1A460A46204600230292ADF823
:101E5000563003F0A9FA684605F03BFA28B903AA00
:101E60002946204603F051FBF5E717B030BD00BF0F
:101E7000DE340700DB3407001B35070013460A4633
:101E800001461846FFF7D0BF024A0349083003F065
:101E90007DBA00BF343E07001B350700437F37B5CE
:101EA000044673B181B30846019105F0D2F8019A56
:101EB0001649034604F1080003B0BDE8304003F0C2
:101EC00024BB037F03B9FEE724291DD000F10805D8
:101ED00079B90F49284603F018FB002304F12000CC
:101EE000237706F033FF204603B0BDE83040FFF70C
:101EF000CBBF0846019105F0ACF8019A03490346AF
:101F0000284603F002FBE8E703B030BDE1340700E8
:101F1000EE34070010B505490446083003F0F5FA21
:101F200020460021BDE81040FFF7B8BFF33407009A
:101F3000FFF7F0BF10B419B95DF8044BFFF7AEBF5F
:101F400091F901300A785DF8044B0249083003F03A
:101F5000DCBA00BF063507000B4601461846FFF7FE
:101F6000E9BF000070B504460D4611461A4603F05D
:101F7000B9F923460026164AA683C4E9025443F859
:101F8000202F2946C4E90A342246C4E90C5404F13E
:101F9000380001F081FD2246294604F1400003F09B
:101FA0004FF822462946C4E9205404F1880002F083
:101FB000E1FB04F5EA5022462946103001F0D6FF35
:101FC000204626616661A661FFF75EFF204670BD70
:101FD000FB1F000010B5054C13460A46014620467B
:101FE000FFF7C0FF024B1C6010BD00BF800E002039
:101FF000780E00200021FFF751BFC068FFF7FABF3D
:102000002DE9FF410B680393234B00930C230546F6
:102010000E464A2221490DEB030005F0ECFD044673
:1020200078B182686368511005EB6200D20748BF3F
:102030006A5806F1040148BFD358984704B0BDE878
:10204000F0811749304621F003FFE8B1DFF84C80FA
:10205000144F05F1080654F80820394630460C3470
:1020600003F053FAB4F55E7FF5D10E4F00242A7DBC
:10207000E3B29A420DD92A69394652F833203046E4
:1020800003F043FA0134F2E731462846FFF7ECFD4E
:10209000D4E70020D2E700BF57100000383E070009
:1020A000143507001B35070030B50446A3B00D46B4
:1020B00001B9FEE7437F5BB1202201A9284621F048
:1020C00097FDA0B101462046FFF7E8FE23B030BDE2
:1020D000037F002BFAD1012303774FF4C071284608
:1020E00006F0A8FCB0F5C07FE6D30620EAE7019B26
:1020F00023B923772046FFF7C7FEE7E701A920466B
:10210000FFF77EFF0028DDD1019B002BDAD1237F72
:10211000002BEFD0DAE70000F0B501230F4E104F8F
:10212000437789B00446142556F8041B1D226846DF
:102130006AF0A4FE00236A46394604F108008DF8CF
:102140001D3003F0E2F969462046FFF7ADFF013D7F
:10215000EAD12846657709B0F0BD00BFC842070044
:1021600019350700FFF736BF07B50190FFF702FDED
:10217000019903B05DF804EBFFF796BF082203F066
:1021800023B9000013B50C4608300A49019003F04A
:10219000FDF801982146FFF7F1FF227A06490198E0
:1021A000C2F3001302F00F0202B0BDE8104003F0CA
:1021B000ACB900BF1E350700383507000B46014695
:1021C0001846FFF7DFBF000038B504460D4619B9C1
:1021D000BDE83840FFF762BE91F839309B0604F144
:1021E000080412D501F108022046164903F0CEF882
:1021F0001549204603F0CAF805F119012046FFF7FA
:10220000BDFF1249204603F0C1F86A8E10492046EE
:1022100003F0BCF829462046FFF7B0FF95F83620BA
:102220000C49204603F0B2F895F937200A492046B8
:1022300003F0ACF895F8382008492046BDE838404E
:1022400003F063B94F350700F433070070A00700AF
:1022500058350700623507006A35070071350700F9
:102260000B4601461846FFF7AFBF00002DE9F04FBF
:102270000C468FB085490546204621F0E9FD06460B
:1022800000287ED18249204621F0E2FD00287FD13E
:1022900020680DF1020121F06AFD064600286CD18C
:1022A000BDF80210A86802AA05F000FB0646002847
:1022B00063D10835BDF822207649284603F025F978
:1022C000BDF820207449284603F01FF928467349B9
:1022D00003F05CF808220DEB0201284603F086F8B3
:1022E0009DF831209DF80030C2F3000161F3000336
:1022F000C2F3400262F3410362F3820301A968461C
:102300008DF80030FFF73EFC65490246284603F091
:10231000FCF89DF8312063492846C2F3001203F00F
:10232000F4F89DF824206049284603F0EEF8049A5A
:102330005E49284603F0E9F8059A5D49284603F00E
:10234000E4F89DF825205B49284603F0DEF89DF966
:1023500026205949284603F0D8F8BDF82E205749C1
:10236000284603F0D2F808E04946204603F00EF86C
:102370008AE0204603F018F8002630460FB0BDE88A
:10238000F08F4F4B4F4A0E2105F1080003F014F96E
:10239000A868DFF85491DFF854A1DFF854B105F0D4
:1023A00005FA00278046B9B2414505F10804E0D29C
:1023B000A86802AA05F07FFA002865D19DF831309F
:1023C0001B0761D4BDF82220002ECDD051462046F7
:1023D00002F0DCFFBDF820205946204602F0D6FF6F
:1023E000049A3949204602F0D1FF059A3649204621
:1023F00002F0CCFF9DF825203449204602F0C6FFAC
:102400009DF824203249204602F0C0FF9DF831207B
:10241000304902F00102204602F0B8FF9DF8312059
:102420002C49C2F34002204602F0B0FF9DF8312053
:102430002849C2F38002204602F0A8FF9DF8302010
:102440002549204602F0A2FF9DF831202349C2F31E
:102450000012204602F09AFFBDF82C201B492046AE
:1024600002F094FFBDF82E201849204602F08EFF9E
:102470001B49204602F08AFF02A92046FFF77EFE94
:102480001849204603F041F801378CE74E3A07001F
:1024900079350700BB350700C83507003134070020
:1024A000D3350700DC350700F2350700FF3507009C
:1024B0006E340700453407000C3607001536070058
:1024C000B8420700804207008F35070098350700A3
:1024D0009F350700A6350700AB350700B03507006C
:1024E000F433070011350700B73507007E350700C4
:1024F000853507002DE9F0430C4693B0002392493F
:10250000ADF806300546204621F0A2FC064600281C
:1025100040F00D818D49204621F09AFC002840F0C2
:102520000D818B49204621F093FC0646002840F09F
:10253000A9808849204621F08BFC0746002800F03E
:10254000F4808249201D21F083FC38B9824B834AF4
:10255000042105F1080003F02FF83E46DFF8488219
:102560007F4FDFF84892A86808AA0DF1060105F030
:102570008FF8002840F08280BDF8302005F1080473
:10258000002E00F0C3804946204602F0FFFE08A955
:102590002046FFF7F3FD0A9802A9152205F0F7F887
:1025A00002AA20466F4902F0F1FE0B9802A91522FB
:1025B00005F0EDF86C4902AA204602F0A6FFD2E72A
:1025C000BDF830204946204602F0E0FE2C4608AA1D
:1025D00054F8080F0DF1060105F05AF800284AD109
:1025E000002EEDD09DF8463013F0080F14BF4322A3
:1025F00052224146204602F0C9FEBDF8302039463D
:10260000204602F0C3FE0A9A5849204602F0BEFE58
:102610009DF93D205649204602F0B8FE9DF93E2026
:102620005449204602F0B2FE9DF846205249204609
:1026300002F0010202F0AAFE9DF846204E49204613
:10264000C2F3400202F0A2FE9DF846204A49C2F3BE
:102650008002204602F09AFE2046484902F096FE8B
:1026600008A92046FFF78AFDBDF8442044492046CA
:1026700002F04BFFAAE7204602F096FE002013B0BE
:10268000BDE8F08305F108043E4B3F4ADFF81C81AA
:102690003E4F3F4E0721204602F08EFFA86808AA51
:1026A0000DF1060104F0F4FF0028E7D1BDF8302059
:1026B0004146204602F06AFE08A92046FFF75EFD6B
:1026C00002A9BDF8400002F03DFE39460246204610
:1026D00002F05CFE02A9BDF8420002F033FE314672
:1026E0000246204602F052FE9DF93D20294920462F
:1026F00002F04CFE9DF93E201D49204602F046FEA8
:102700000A9A2549204602F000FFC7E741462046C5
:1027100002F03CFE08A92046FFF730FDDDE90A2360
:102720003946204602F0F1FE1DE70720A7E71B4BC4
:102730001B4A0A2105F1080002F03EFFDFF868900D
:10274000DFF86C80174F41E74E3A070079350700F4
:102750002E36070092360700904307003C430700DF
:10276000AD3607009B360700A33607004236070048
:102770004A36070051360700A6350700F433070034
:10278000583607009E430700744307006D36070064
:102790007836070082360700893607009443070021
:1027A0004C43070085350700873507006136070071
:1027B0003A3607002DE9F04F0C4689B06E490546C0
:1027C000204621F045FB074600286ED16B49204684
:1027D00021F03EFB00286FD120680DF10A0121F0A5
:1027E000C6FA0646002840F0C280BDF80A10A86864
:1027F00003AA05F0A4F80646002840F0B8809DF82A
:102800001C205F49083502F00102284602F07DFED7
:102810009DF81C30DA0740F1AA809DF8162059492E
:10282000284602F072FEBDF814205749284602F0EF
:102830006CFE9DF8172055499202284602F065FE6D
:102840009DF81C205249C2F34002284602F05DFE6A
:102850009DF81C309B0740F18A8028464D4902F0C4
:1028600095FD03A92846082202F0C0FD9DF8182016
:102870004949284602F049FE9DF819204749284653
:1028800002F043FE9DF81A204549284602F03DFE1D
:102890009DF81B204349284602F037FE67E01A46A0
:1028A0004946204602F072FD59E03F4B3F4A09215C
:1028B00005F1080002F080FEA868DFF81091DFF84B
:1028C00010A1DFF810B105F038F8002680462C463C
:1028D000F3B254F8080F019303AA194605F02FF834
:1028E00000283CD1019B002FD9D09DF816205146DD
:1028F000204602F04BFDBDF814205946204602F058
:1029000045FD9DF817202A49204602F03FFD9DF81D
:1029100018202849204602F039FD9DF81920264943
:10292000204602F033FD9DF81A202449204602F08B
:102930002DFD9DF81B202249204602F027FD21494C
:10294000204602F023FD03A92046FFF717FC9DF85F
:102950001C201D49C2F34002204602F0D6FD01367C
:10296000F3B24345B3D9204602F01EFD002630469F
:1029700009B0BDE8F08F00BF4E3A07007935070077
:10298000D936070025330700C8350700E3360700AE
:10299000F236070031340700FB36070045340700E4
:1029A0005934070004370700F4410700D0410700FD
:1029B000C4360700CB36070098350700D23607002B
:1029C0007E350700F43307000B350700B7350700E5
:1029D0006335070085350700F7B50C6805460E46D8
:1029E0001F464CB120460DF1060121F0C0F9044606
:1029F00050B1204603B0F0BD006890470749024639
:102A0000284602F082FDF4E7736823B9BDF806108A
:102A10002868B847EDE70724EBE700BF4245070009
:102A2000F8B50E4605461A49304621F011FA38B17C
:102A3000184B194A311D05F10800FFF7CDFFF8BD0D
:102A40001649304621F004FA044610B1144B154AD9
:102A5000F0E71549304621F0FBF908B90720EEE709
:102A6000776857B955F8080F04F065FA0F49024620
:102A7000284602F04AFD3846E1E70D49301D21F0B5
:102A8000E7F90028EAD0A86804F059FA2046D6E70A
:102A90000C3707002F6F0000276F00001937070061
:102AA0001F6F0000176F0000223707004245070024
:102AB00083580700F7B50C6805460E461F4644B11B
:102AC000204601A921F0F1F9044650B1204603B097
:102AD000F0BD0068904707490246284602F015FD00
:102AE000F4E773681BB901992868B847EEE7072433
:102AF000ECE700BFF432070008B5034A034B083087
:102B0000FFF7D8FF08BD00BF057500000D75000078
:102B100008B5034A034B0830FFF7CCFF08BD00BFE0
:102B20000D7800001578000038B50C4605460E49B2
:102B3000204621F08DF938B10C4B0D4A211D05F1CD
:102B40000800FFF7B7FF38BD0A49204621F080F999
:102B500038B1094B094A211D05F10800FFF73CFF78
:102B6000F1E70720EFE700BF263707006176000096
:102B7000597600002E370700757600006D7600004C
:102B8000F7B50D461E462B68074611464BB128681F
:102B90000DF1070121F0DAF8044640B1204603B0F8
:102BA000F0BDFEF797FD04460028F7D0EFE76B680D
:102BB00023B99DF807103868B047EFE70724EDE721
:102BC00008B5034A034B0830FFF7DAFF08BD00BF22
:102BD000E7770000EF77000008B5034A034B0830A1
:102BE000FFF7CEFF08BD00BF1D780000257800006C
:102BF00008B5034A034B0830FFF7C2FF08BD00BF0A
:102C00008D7800009578000008B5034A034B083022
:102C1000FFF7B6FF08BD00BF9D780000A578000053
:102C200008B5034A034B0830FFF7AAFF08BD00BFF1
:102C30002D7800003578000070B50C460546104927
:102C4000204621F005F9B0B1261D0E49304621F08D
:102C5000FFF840B10C4B0D4A04F1080105F10800E2
:102C6000FFF78EFF70BD0A49304621F0F1F820B120
:102C7000084B094AF0E72320F4E70720F2E700BFFA
:102C800038370700423707001B720000137200003C
:102C9000403707002B7200002372000073B50C460A
:102CA00006460DF106012068154621F060F828B9A6
:102CB00063682BB9BDF806103068A84702B070BD34
:102CC0000720FBE738B50C6800F108054CB98068AF
:102CD00004F078FA05490246284602F016FC204620
:102CE00038BD034A2846FFF7D9FFF9E749370700FF
:102CF000CD710000F7B50E4605462149304621F05A
:102D0000A7F838B11F4A311D05F10800FFF7C6FFCB
:102D100003B0F0BD1C49304621F09AF8074668B16F
:102D200004361A49304621F093F820B1A86804F01F
:102D3000F4F90020ECE7164A3146E5E7154930463C
:102D400021F086F8D0B155F8080F0DF1070104F015
:102D5000E9F9064670B13C460F4F9DF80720E3B2F3
:102D60009A4207D936F813203946284602F00EFB5E
:102D70000134F2E7284602F017FBDAE72320C7E721
:102D8000CD320700FF7000005037070038F1070010
:102D90000D71000057370700B735070070B50C6894
:102DA000164605461A4614B1FFF778FF70BD006855
:102DB000B04703490246284602F0A7FB2046F5E744
:102DC0004245070008B5034A034B0830FFF7E6FF0A
:102DD00008BD00BFAD770000B577000008B5034A15
:102DE000034B0830FFF7DAFF08BD00BFF77700009C
:102DF000FF77000073B50C4606460DF10701206809
:102E0000154620F0A3FF28B963682BB99DF8071079
:102E10003068A84702B070BD0720FBE737B50C4605
:102E200011461A46236805462BB121462846FFF76E
:102E3000E1FF03B030BD0192FEF74CFC019A00287F
:102E4000F7D0F2E7F8B50D4606461049284620F0BF
:102E5000FFFF06F1080748B1B0680EF047FD0246D3
:102E60000B49384602F051FB0020F8BD09492846BD
:102E700020F0EEFF18B1B0680EF03CFDEFE7064B16
:102E8000064A29463846FFF7C9FFEEE79DF30700DB
:102E90005B37070061370700537100004B7100007A
:102EA00008B5034A034B0830FFF7B8FF08BD00BF61
:102EB0003D7800004578000008B5024A0830FFF769
:102EC00099FF08BDDD77000008B5024A0830FFF71A
:102ED00091FF08BD4F78000038B50C68054644B92D
:102EE0000068904704490246284602F00EFB20463F
:102EF00038BD0720FCE700BF1B35070038B50C467E
:102F000005461149204620F0A3FF30B10F4A211D8C
:102F100005F10800FFF7E0FF38BD0D49204620F01D
:102F200097FF08B10B4AF2E70B49204620F090FFCB
:102F300008B10A4AEBE70A49204620F089FF08B1A8
:102F4000084AE4E70720E7E729A20700AD7300007D
:102F50006B370700B573000071370700BD730000C1
:102F60007B370700C573000038B5094A04460830AE
:102F70000D46FFF7B1FF48B1296831B16B6823B93D
:102F8000A068BDE8384004F05CBB072038BD00BF36
:102F90003B76000038B5094A044608300D46FFF775
:102FA0009BFF48B1296831B16B6823B9A068BDE8BF
:102FB000384004F023BB072038BD00BFF575000082
:102FC00038B50C4605460A7A074902F09EFA62882F
:102FD0000649284602F099FA626805492846BDE884
:102FE000384002F092BA00BF384507004545070057
:102FF000574507001FB50B680446E3B90F4902F0B7
:10300000C5F9206801A903F081FF78B9204602F0D4
:10301000CBF90B49BDF80420204602F076FA01A94D
:103020002046FFF7CDFF002004B010BD0549204623
:1030300002F06BFAF7E72320F6E700BF6A450700C6
:1030400077450700884507000968006869F0C1BA3C
:103050000968006869F0BDBAD1E9002302F0E2B95D
:10306000D1E9042302F0DEB9B1F85A20014902F097
:103070004CBA00BF4245070001F13002014902F09D
:1030800044BA00BF1B350700B1F85820014902F0CF
:103090003CBA00BF493707000A6F014902F035BA50
:1030A0008E4507004A6D014902F02FBAF43207003D
:1030B0000822413102F09AB91022203102F096B96B
:1030C000493102F0FDB90B6810B514461A1D0A60AB
:1030D0001868214620F0DEFD08B92081A07210BDDD
:1030E0000B6810B514461A1D0A60186804F1100127
:1030F00020F0D0FD08B92083A07610BD0B68181D04
:103100000860186802F15A0120F031BE0B68181DE2
:103110000860186802F1580120F029BE0B68181DDC
:103120000860186802F1700120F0BFBE0B68181D1E
:103130000860186802F1540120F0B7BE0B68104611
:103140001A1D0A6000F141010822186820F05FBED4
:1031500030B50B6885B015461A1D0A6018686946B7
:1031600020F04BFE044628B96B4603CBC5F8490056
:10317000C5F84D10204605B030BD0B68186830B159
:1031800004330B60014602F1300003F007BF072053
:10319000704700002DE9F0410D4607461B4928689D
:1031A000144620F055FE2B681A1D2A6020B3D3F870
:1031B0000480B8F1000F27D094F8773093B104F170
:1031C000300694F8783093B104F1410204F15C03C5
:1031D0003146404603F0E0FE10B92B6804332B6003
:1031E000BDE8F081386804F005FA0646E9E738687A
:1031F00004F091F90246E9E704F15C011868BDE8C2
:10320000F041102220F003BE0720E9E73333070026
:1032100008B5FF220021024869F0C6F8002008BD69
:10322000E02B002070B50C46E2B005461749204659
:1032300020F00EFE18BB1649204620F009FE18B3F8
:103240000126FE236068ADF8063022AA0DF10601C2
:1032500020F0EBFD78B9BDF806308DF8863102A973
:1032600022A803F0A2FE044628B9286822A946B97C
:1032700003F06FFE00B10446204662B070BD002628
:10328000DFE703F070FEF5E70724F5E79645070052
:103290004864070010B50C6834B9044991F8FE2061
:1032A00002F0A4F8204610BD0720FCE7E02B002028
:1032B00030B50C46A1B005461D49204620F0C8FD9A
:1032C00028B11C49286803F03FFE21B030BD1A49DF
:1032D000204620F0BDFD20B11649286803F03EFECF
:1032E000F3E71649204620F0B3FD50B1286869463F
:1032F00003F0A0FE0028E8D10E49684603F06DFEF9
:10330000E3E70F49204620F0A3FD78B1094D60683E
:10331000FE232A466946ADF8003020F086FD0028DD
:10332000D3D1BDF8003085F8FE30CEE70720CCE7DA
:1033300096450700E02B0020486407009D450700E4
:10334000A145070038B50D4604460C49284620F033
:103350007FFD28B120680A49BDE8384003F0F9BD77
:103360000849284620F074FD28B120680449BDE8CA
:10337000384003F0F8BD072038BD00BF9645070070
:10338000E02B00204864070010225C3102F02EB8C8
:103390000B6810461A1D0A6000F1200110221868FF
:1033A00020F035BD70B51368A2B006460D460192F7
:1033B000D3B91E4802A903F0F8FD044688B96B682A
:1033C00022AA134413F80C3C5BB1EA68AB685110B5
:1033D000D50706EB620048BF725802A948BFD35810
:1033E0009847204622B070BD8022002102A868F0D4
:1033F000DBFF6A692B69511006EB6200D20748BFF8
:10340000725801A948BFD35802AA98470446002819
:10341000E7D16B68054922AA1344012203F80C2C5A
:1034200002A803F0EEFD0446DBE700BFE02B00201E
:1034300038B50C460A882249054601F0A7FFA37853
:10344000D80703D51F49284601F0A0FFA3789907A4
:1034500003D51D49284601F099FFA3785A0703D5E3
:103460001A49284601F092FFA3781B0703D5184993
:10347000284601F08BFFA378D80603D515492846C6
:1034800001F084FFA378990603D51349284601F07B
:103490007DFFA3785A0603D51049284601F076FF30
:1034A000E378DB0703D50E49284601F06FFFE27889
:1034B0000C492846C2F34202BDE8384002F025B864
:1034C000B73507008F370700E6E907006C5F070094
:1034D000F6480700B93A07000B49070068E2070001
:1034E00072AA0700414507006C31FFF7A1BF000039
:1034F00073B50023019313680E46186801A9154699
:1035000020F035FC044600287FD129684A680B1D4D
:103510002B60002A77D0013A12F8013F002B5BD0D4
:10352000722B05D8622B05D8432B3FD0522B4CD0A1
:1035300007246AE0633B0F2BFAD801A050F823F070
:10354000A335000031350000B735000031350000EB
:1035500031350000313500003135000031350000D3
:103560003135000031350000313500008F35000065
:1035700081350000C135000031350000993500006B
:103580009DF8063043F001038DF80630C4E79DF83E
:10359000063043F00203F7E79DF8063043F00403DA
:1035A000F2E79DF8063043F00803EDE79DF806309A
:1035B00043F01003E8E79DF8063043F02003E3E70B
:1035C0009DF8063043F04003DEE79DF8073043F0F6
:1035D00001038DF807309FE7886801F108032B602D
:1035E00088B10DF1030120F0B1FB88B92B689DF87B
:1035F00003200433072A2B609AD89DF8073062F322
:1036000043038DF8073001983060204602B070BD4A
:103610000446FAE713460A4603F16C01FFF768BF58
:1036200007B5044B00930E22182304F0E4FA03B00C
:103630005DF804FB493000002DE9F047A2B00446D4
:10364000084602A903F0B1FC064658BBDFF85CA0AF
:10365000DFF85C80DFF85C900C27DAF80430019327
:10366000414601A8FFF7DCFF436822AA1344054640
:1036700013F80C3C93B1DAF800204946204601F0DB
:1036800085FEEB685A1013F0010F18BFA25804EB27
:103690006300AB6802A918BFD3589847013F0AF1ED
:1036A000080ADAD1304622B0BDE8F0879846070014
:1036B00064470700845D070070B5C0B005460E463C
:1036C0000068694603F040FC044630B933683BB9F2
:1036D00069462846FFF7B0FF0446204640B070BD5B
:1036E0000649304620F0B4FB30B19DF8FE20694613
:1036F000284601F07BFEF0E70724EEE7453A070095
:1037000070B5C0B005460E460068694603F026FC59
:10371000044630B933683BB969462846FFF78CFF49
:103720000446204640B070BD0649304620F090FB6C
:1037300030B19DF8FE206946284601F057FEF0E7BB
:103740000724EEE7453A07002DE9F047C4B00E46DE
:1037500004468022002104A868F026FE334FDFF8DB
:10376000D880331D02934FF00009029BD3F800A0CC
:10377000BAF1000F38D0394603A8CDF80CA0FFF7F6
:103780004FFF0546C0B14269029B511004EB620035
:103790000433D20748BF625802932B6902A948BF7D
:1037A000D35804AA984700283AD16B6844AA134416
:1037B000012203F88C2CD8E70298414620F048FB00
:1037C000002830D0029B1A1D02928022ADF80C20F6
:1037D000586824AA03A920F028FB08BB029B9DF887
:1037E0000C9004330293C0E71149304620F030FBBF
:1037F000054668B90F49304620F02AFB98B1CDE95B
:10380000005520684B4624AA04A903F0C0FB07E03A
:10381000CDE900AA20684B4624AA04A903F0ADFB19
:1038200044B0BDE8F0870720FAE700BF644707000F
:103830009645070048640700453A07002DE9F04F18
:10384000002493B0CDE90344DFF8E090DFF8E0A076
:10385000059406460D4601F104082746D8F800B045
:10386000BBF1000F38D02E49CDF808B002A8FFF701
:10387000D7FE48B1426812AB1A44012102F83C1C41
:10388000C3460BF10408E9E74946404620F0E0FA58
:1038900070B12022ADF80820D8F804000AAA02A9C5
:1038A00008F1040B20F0C1FA48B99DF80870E8E768
:1038B0005146404620F0CCFA044618B9072013B010
:1038C000BDE8F08FD8F8040006A908F1040B20F039
:1038D00094FA0028D5D0F2E71249284620F0B8FA29
:1038E00058B130680CB10DF1180BCDF800B03B4663
:1038F0000AAA03A903F03CFBE1E70B49284620F0A4
:10390000A7FA0028DAD030680CB10DF1180BCDF809
:1039100000B03B460AAA03A903F034FBCFE700BF7F
:10392000644707009645070048640700453A0700CA
:103930000FF20700F0B50B6885B005460C4623B9B9
:103940002049FFF779FE05B0F0BD1F49204620F061
:103950007FFA60B11D4F1E4E0024E25931462846C1
:103960000C3401F0D2FD6C2CF7D10020EBE723687A
:103970001849039303A8FFF753FE014620B1221D07
:103980002846FFF70FFDDEE723680393124B0093F1
:103990000C230DEB03000D49092204F02CF903461A
:1039A00068B182685B68511005EB6200D20748BFBE
:1039B0006A5804F1040148BFD3589847C3E723204D
:1039C000C1E700BFE02B002014350700F8460700D0
:1039D0001B35070064470700513000000968006884
:1039E00068F0F7BD38B50C6805464CB9006803F0BF
:1039F000A9FC04490246284601F087FD204638BD4F
:103A00000720FCE74245070038B50C680546084624
:103A10004CB9286803F09AFC08490246284601F090
:103A200074FD002038BD064920F012FA18B128684C
:103A300003F090FCF5E70720F4E700BF42450700DC
:103A40008358070030B50C4687B00546114920461B
:103A500020F0FEF9D8B102A9201DFEF72CF9172895
:103A600007D1002360688DF810300822694620F0E5
:103A7000CEF930B99DF81030286823B102A903F0BF
:103A80008FFC07B030BD694603F085FCF9E70720DD
:103A9000F7E700BFB4480700C0E900127047437C55
:103AA0005A0744BF702301F8013B437C1B0744BF06
:103AB000612301F8013B437CDA0644BF642301F82B
:103AC000013B437C9B0644BF632301F8013B437CDD
:103AD0005A0644BF722301F8013B437CDB091CBF3B
:103AE0006F2301F8013B837CDB0744BF732301F89C
:103AF000013B837C9A0744BF6E2301F8013B837C22
:103B00005B0744BF442301F8013B00230B7070475F
:103B100030B50C4687B0054601F0AAFC01A9204645
:103B2000FFF7BDFF9DF8043023B1094901AA2846DB
:103B300001F02CFC607C40F3010040B2FEF7DCF8A1
:103B4000A38A04490246284601F0DFFC07B030BDD5
:103B50001A350700BA480700037D1B0744BF7323CB
:103B600001F8013B037D5A0744BF6E2301F8013B76
:103B7000037D9B0644BF612301F8013B00230B70CA
:103B80007047000030B50C4687B0054601F070FC68
:103B900001A92046FFF7E0FF9DF8043023B1094951
:103BA00001AA284601F0F2FB207D40F3010040B25B
:103BB000FEF7A2F8638A04490246284601F0A5FCF4
:103BC00007B030BD1A350700BA48070038B50C46B3
:103BD00005464A68114901F0D9FB227A04F109012E
:103BE000284601F0F1FB0E49284601F0CFFB94F87E
:103BF000072104F58471284601F0E6FB94F80631AC
:103C0000DB0703D50749284601F0C0FBB4F80022C2
:103C100005492846BDE8384001F077BCC348070095
:103C200070A00700C8480700CD35070013B9006829
:103C300003F098BB1720704713B9006803F097BBD7
:103C40001720704713B9006803F096BB1720704720
:103C5000F0B5ADF51B7D00230E4662490093044686
:103C6000154601F052FC4FF6FF77334606AA694627
:103C70002046FFF7DBFF50B9BD4203D0BDF82C3022
:103C8000AB42F2D106A92046FFF742FFEDE75649C5
:103C9000204601F03AFC002300934FF6FF773346AD
:103CA0000CAA69462046FFF7C7FF50B9BD4203D0B2
:103CB000BDF84230AB42F2D10CA92046FFF762FFBB
:103CC000EDE74A49204601F020FC002300934FF61F
:103CD000FF77334619AA69462046FFF7B3FF50B96C
:103CE000BD4203D0BDF86432AB42F2D119A92046DF
:103CF000FFF76CFFEDE7002E5DD14FF6FF739D429D
:103D000059D13B493B4D204601F0FFFB009620680E
:103D100001AA694603F035FB88B90DF1060120467A
:103D200001F0A6FB9DF805309DF80420002B14BF80
:103D300063232D232946204601F0E7FBE7E72068AF
:103D400012A903F023FB2C49204601F0DEFB9DF86D
:103D500060309D0732D5BDF84A202849204601F041
:103D600015FB9DF86030D8072DD5BDF848202449B3
:103D7000204601F00BFB9DF86030190728D5BDF8EF
:103D80005E201E49204601F001FB9DF860305A0775
:103D900023D59DF84C200DF14D01204601F014FB78
:103DA0009DF86030DB0603D51649204601F0EEFA97
:103DB000204601F0F9FA0DF51B7DF0BD12492046B1
:103DC00001F0E4FACDE71049204601F0DFFAD2E72E
:103DD0000D49204601F0DAFAD7E70C49204601F0F8
:103DE000D5FADDE7CB480700D5480700DD480700D6
:103DF000E7480700F1480700F8480700B735070013
:103E0000893507000A490700074907001BA3070077
:103E100030B5C3B0FF2305468DF8073081B900687F
:103E20000DF1070302AA03F088FA044628B99DF8A9
:103E3000072002A9284601F0D9FA204643B030BD38
:103E40000C24FAE72DE9F04F85B000244FF6FF73FC
:103E5000DFF88480DFF88490ADF80E3006460D461A
:103E60002746A2465FFA84FB05EB8B0355F82B200F
:103E7000D2B11846414601931FF0EAFF019B70B989
:103E8000494618461FF0E4FF60B955F82B000DF1C4
:103E90000E011FF06CFF18B105B0BDE8F08F82462F
:103EA0000134DFE70746FBE7BDF80E20BAF1000F4B
:103EB00000D14FB14FF6FF739A420BD127B1514653
:103EC0003046FFF7A5FFE7E730465146FFF7C0FE53
:103ED0000020E1E70720DFE7D5320700453A070079
:103EE0002DE9FF410B6805460C4693B9DFF8788051
:103EF0001A4F002656F80820394628460C3601F09D
:103F000004FB302EF6D123682BBB232004B0BDE880
:103F1000F081134920461FF09BFF0028E6D123685B
:103F20000393104B00930C230DEB03000E49042266
:103F300003F061FE03460028E7D082685B685110F9
:103F400005EB6200D20748BF6A5804F1040148BF7C
:103F5000D3589847DAE70020D8E700BF1B350700A1
:103F600014350700DD39000024490700C0E90012BC
:103F7000027A6FF30002027270470968002330B5BD
:103F8000136001394FF47A730A2411F8010FE8B174
:103F9000A0F13005092D11D8B3F57A7F02BF106862
:103FA0006043106008781568303803FB0050B3F5A3
:103FB0007A7F1060E9D0B3FBF4F3E6E72E2804D152
:103FC000B3F57A7F01D16423DFE7072030BD00001D
:103FD00070B50E4692B004464E4930461FF038FF89
:103FE00028B1206803F0F7F9002012B070BD4A49EB
:103FF00030461FF02DFF054600B1043600213C225B
:1040000003A868F0D1F9454930461FF021FF68B197
:10401000706803A91FF0F1FE0028E6D1206803A90B
:1040200003F048F808B90720DFE708363C49304676
:104030001FF00EFF18B101238DF8443004362068BC
:104040000DF1070307AA3146FDF762FE0028CCD127
:104050009DF807303BB13349204601F097F907A995
:10406000204601F0FBF9706800282ED1B0680028C6
:1040700031D1F368002B35D1306900283BD1736909
:104080006BB102AA06F114012046FFF776FF002863
:10409000ABD1029BB3F5803FC5D2ADF84030B369D8
:1040A000002BC0D1204B0B93204B206803A9CDE9F6
:1040B0000C3403F08BF9002897D1237A002D65F397
:1040C0000003237208BF24208FE70EA91FF04FFEC4
:1040D0000028CBD089E70DF13A011FF048FE0028F7
:1040E000C7D082E70FAA06F10C012046FFF745FF73
:1040F0000028C1D079E70DF142011FF027FE00280A
:104100007FF473AF9DF84230B3FA83F35B098DF807
:104110004330B4E7E2330700873307005449070010
:10412000574907005A49070069410000154200003D
:1041300037B54A8A08320C46054692B2084901F062
:1041400025F92146284601F077F9238A0093A28AAF
:10415000A37D0449284601F0D8F903B030BD00BF63
:104160007D4907008C4907000B4601461846FFF7BA
:10417000DFBF0000024B186800B9FEE7FDF78EBEF6
:10418000780E002037B50C460A884B881E49054634
:1041900001F0FCF822889AB1237B8BB963889A429C
:1041A0000ED3D11A4FF47A734B430A2193FBF2F3E7
:1041B0002846B3FBF1F201FB1233144901F0E6F893
:1041C000628892B16368608901904FF47A714B43C1
:1041D000B3FBF2F2B2FBF1F301FB132200920C49A4
:1041E00022899BB2284601F0D1F8284601F0DCF87C
:1041F000297A11F0010105D1284603B0BDE830400D
:10420000FFF7B8BF03B030BDAC490700D94907007C
:10421000F24907000B4601461846FFF7B3BF0000FE
:104220002DE9F04790F8A4528AB004460E46002DBE
:1042300040F0E2800B68002B42D10123A0F8A832A5
:1042400040F6262540F6262204F5397104F52B7038
:1042500003F0F8F82022002102A868F0A5F8674BC7
:10426000039394F8A832002B00F0BF80644B0593B1
:10427000644B069304F10806634B0793206802948D
:1042800004F60A5302AA3146CDE9083503F0B5F821
:10429000054688B95D4B039320685D4B049302AAE1
:1042A00004F51E71029403F0C0F80546002800F0E2
:1042B0009F80304603F0B7F828460AB0BDE8F08783
:1042C000544930461FF0C4FDA8B1A4F8A852706844
:1042D0000028B5D002A91FF0E8FD05460028EBD163
:1042E000029DEB1D05EBD3056A1E40F625239A427D
:1042F000A8D90725E0E7484930461FF0A9FD074641
:1043000018B10123A4F8A832E1E7444930461FF070
:104310009FFD0028EDD040F2011304F5C658A4F823
:10432000A83208F1180804F5D15A04F01BFF0AF16D
:104330000C0A404604F5BA592DF05EF909F1180946
:10434000504604F5C25508353CF00CF9484628F0B3
:1043500089F8284628F0C8FB3A463149284628F013
:104360008CF83946284628F081F82E49284628F04E
:104370008DF803221146284628F005F9032211463C
:10438000284628F0FBF8E922274900973B4650468B
:104390003CF0F0FD024618B12449204601F0B5F882
:1043A00040F22D32224940462DF0B0FD024618B1B0
:1043B0002049204601F0A9F840F299221E494046C2
:1043C0002DF0A4FD024618B11C49204601F09DF8CD
:1043D0002946484628F094FA024600283FF477AF71
:1043E0001749204601F091F871E7164B04933FE717
:1043F000012384F8A4325FE718255DE7394E0000F9
:10440000994E00000B4F0000914800003D4900000C
:104410007D4900001C4A0700234A07002C4A070078
:10442000F5940000F4580700304A0700194B0700C4
:104430003A4B0700674E07008E4E070027510700D2
:104440004E5107005D4C000090F8A43223B10B6878
:1044500023B9083002F0E3BF0D20704707207047F2
:104460000968006868F0B5B80B68F7B50446CBBBBF
:1044700090F8A432C3B390F8A932ABB104F08CFE2B
:1044800004F5C250083028F099FB04F5BA501830F2
:1044900028F0D2FA04F5D1500C303CF067F804F55E
:1044A000C65018302DF0ADF804F1080002F0BBFF43
:1044B0000027064684F8A77204F52B70019002F0DD
:1044C000CFFF019802F0CEFF054604F51E7002F002
:1044D000B7FF84F8A4724EB9BD4208BF054628460E
:1044E00003B0F0BD0725FAE70D25F8E73546F6E7F6
:1044F0000B6810B504465BB990F8A43253B108308C
:1045000002F08FFF18B984F8A50284F8A60210BD46
:104510000720FCE70D20FAE70B6833B990F8A432C6
:104520002BB100F51E7002F089BF072070470D20E7
:1045300070472DE9FF4190F8A43205460E46002B46
:104540005DD041F23C73C358002B5ED10F68002F41
:1045500057D04C68002C54D190F8A83243B390F84F
:10456000A9820846B8F1000F13D01FF06AFC02467A
:1045700005F5BA503946183029F070FE002842DAA5
:1045800020F0800010F5D24018BF012004B0BDE833
:10459000F0811FF056FC03AA03460092CDF8048078
:1045A0003A4605F52B7105F1080002F04DFFEDE7E5
:1045B00090F8A7324BBB00F53974C0F8D832C0F878
:1045C000DC4208461FF03DFC40F62622904203D80C
:1045D00030461FF036FC02463168C5F8E02220461E
:1045E00068F0C6FA002205F5367105F1080002F000
:1045F00010FF0028CAD1012385F8A732C6E70D2095
:10460000C4E70720C2E72046C0E70520BEE730B573
:1046100090F8A43287B005460C46A3B1206801A9E2
:104620001FF0EBFB58B9606805A91FF0A0FB30B97B
:10463000A36833B901A905F1080002F0E6FE07B04E
:1046400030BD0720FBE70D20F9E730B590F8A43224
:1046500087B004460D46CBB1286801A91FF0CDFBF9
:1046600080B9686805A91FF082FB58B9AB685BB9CF
:1046700004F51E74204602F0E1FE18B901A9204697
:1046800002F0DAFE07B030BD0720FBE70D20F9E7A6
:104690002DE9F0471F4690F8AA32ADF5007D04469B
:1046A0000E46154663B990F8A932002B3CD01FB1D5
:1046B0002B49204600F029FF0DF5007DBDE8F0876D
:1046C000002AF4D090F8A93283B300F5BA56DFF887
:1046D0009880DFF8989018360DF10C0A4FF4FA72B2
:1046E000514630462AF0A6F9021E07DA12F5D24FDB
:1046F0000CD04946204600F008FFEDE7CDF800A0B9
:1047000013464146204600F000FFE5E715492A46DA
:10471000204600F0FAFECAE7454500D0FEE72946EC
:10472000304602F07AFEC2E7002AC0D003A9304624
:1047300002F071FEDFF838904FF00008039A002A6B
:10474000EAD0D2E901234946009220461A4600F0F9
:10475000DCFE039B9A681B6803939044EEE700BF5E
:10476000D7510700A1510700845107006C51070081
:10477000BA510700C0E900120121A0F8A81241F2C5
:104780003C710022C0F8A42280F8AA22425000F511
:10479000BA510A6041F24871425041F2507200F140
:1047A0000801815041F2547200F52B71815070471D
:1047B0002DE9FF410B6805460C4693B9DFF8788078
:1047C0001A4F002656F80820394628460C3600F0C5
:1047D0009CFE782EF6D123682BBB232004B0BDE8C5
:1047E000F081134920461FF033FB0028E6D12368EF
:1047F0000393104B00930C230DEB03000E490A2288
:1048000003F0F9F903460028E7D082685B6851108D
:1048100005EB6200D20748BF6A5804F1040148BFA3
:10482000D3589847DAE70020D8E700BF1B350700C8
:10483000143507006144000014590700042A96BF8C
:10484000104B114A53F82220104910B5044600F0CD
:104850005CFE94F8A93223B104F5BA50183028F060
:10486000E8F841F23C72002384F8A532A4F8A6329D
:10487000A35004F5BA5204F52B701360BDE8104044
:1048800002F0EEBD00590700725A0700F25107000E
:1048900013B50446019102F0B5FD019A214602B01C
:1048A000BDE81040FFF7CABF38B5154690F8A522FD
:1048B000044662B11D4900F069FD2946204600F01A
:1048C00009FE20461A4900F020FE012038BD00F103
:1048D0000801196090F8A9320BB90020F6E700F53D
:1048E000C255083513460121284628F001F9024631
:1048F00018B11049204600F008FE41F62823002296
:10490000E158284627F0E6FD04F5D15204F5C651DA
:104910000C321831284627F0BFFD02460028DCD0B3
:104920000549204600F0F1FDD7E700BFFA51070026
:104930002A520700435207006B52070037B50D4655
:104940000446019202F076FD019B2A46214603B0FF
:10495000BDE83040FFF7A8BF38B51D460123044627
:1049600080F8A532044900F011FD29462046BDE833
:10497000384000F0C1BD00BF9152070037B50D4669
:104980000446019202F056FD019B2A46214603B0DF
:10499000BDE83040FFF7E0BFF0B52B4F87B00446CD
:1049A00000F5BA5633681BB90025284607B0F0BD9C
:1049B00004F52B710846039102F050FD0028F3D056
:1049C00035680399B5F5826F2B4628BF4FF4826393
:1049D00098424FF0000215D99D4294BF0025012551
:1049E000059294F8A922FAB104F5BA501A4639464C
:1049F000183029F033FC002806DD33680590984212
:104A00001DD9FEE71546EBE720F0800010F5D24FE8
:104A100015D001250D49204600F077FD41F23C728A
:104A20000023A3503360C0E705AA0195009204F16A
:104A300008003A4602F008FD05460028EAD133682E
:104A4000059A9B1A3360ADE7AB520700BC560700CE
:104A500041F24C7370B5C25841F248734FF4FA54A6
:104A6000C358590804FB02140849B4FBF3F4054683
:104A700000F04BFD4FF47A732846B4FBF3F204497F
:104A800003FB1243BDE8704000F03FBDD156070064
:104A900013570700F8B50D4604463F4928461FF056
:104AA000D7F9D8B13D49204600F070FC41F23C7383
:104AB000E6582EB13A49204600F027FD0020F8BD07
:104AC00041F24873E5583DB12046364900F01DFDDE
:104AD0002046FFF7BDFFF1E73349ECE733492846AD
:104AE0001FF0B6F950B394F8A732002B52D141F21F
:104AF0003C76A119A359002B4CD16868B8B94FF482
:104B00009033A351AB68CBB901F053F841F2447331
:104B100041F23C76E05004F5BA5394F8A852A759F4
:104B20001F606DB12046BDE8F840FFF735BF1FF0AC
:104B3000BCF90028C3D1A359002BE3D10720BEE75D
:104B400004F5397340F626226121184667F02CFCE3
:104B500007F6252140F625229142AFD941F2307166
:104B600041F234726550A05040F62622B7FBF2F3B2
:104B700002FB1373002B08BF134641F23872214425
:104B8000A35004F108002A4602F043FC002895D007
:104B9000A55194E7052092E72E57070035570700E7
:104BA0004C570700545707005E5707006757070028
:104BB00038B5044600F0FDFF41F2447341F23C7504
:104BC000E358C01A41F24873E05041F24C73625905
:104BD000E2502046FFF73CFF0023635138BD000040
:104BE000F8B590F8A8520446114605B1FEE741F227
:104BF0003C7600F53673825942B9994205D190F856
:104C0000A73203B9FEE780F8A722F8BD994200D188
:104C1000FEE700F5BA528F681368BB4200D2FEE788
:104C2000DB1B136040F6252293420ED940F6262363
:104C30008B602A46083002F0ECFB0028E5D00649DC
:104C4000204600F062FCA551DFE7002BDDD1BDE876
:104C5000F840FFF7ADBF00BFBC56070013B50446D0
:104C6000019102F0CFFB019A214602B0BDE810404D
:104C7000FFF7B6BF73B500F5BA55183511490446AC
:104C8000284627F043FC024618B10F49204600F0A1
:104C90003CFC0E220D49284627F020FC024618B1A4
:104CA0000B49204600F031FC002604F5BA51094BAF
:104CB000094A00961031284627F0E2FB84F8AA62E0
:104CC00002B070BD6B570700755707009A57070071
:104CD000A95707009D7400006974000038B590F86A
:104CE000AA320546CBB900F5BA50183027F0D6FCE9
:104CF0000124024638B90A49284600F006FC85F826
:104D0000AA42204638BD20F0800313F5D24FF8D0D8
:104D10000449284600F0F9FBF3E70024F1E700BF5F
:104D2000D9570700F0570700F0B590F8A43287B0C4
:104D300004460F46002B5FD000680DF1030301AA63
:104D4000FCF7E6FF054608BB9DF803303BB12B4955
:104D5000204600F01BFB01A9204600F07FFB78688D
:104D600005A91FF004F8054680B9BB68002B41D0A7
:104D700007F10805224928461FF06AF8064640B99F
:104D8000204928461FF064F820B90725284607B0B7
:104D9000F0BD0126FB68002BF7D194F8A9326BB166
:104DA000002304F5C2501A461946083027F0A0FE29
:104DB000024618B11449204600F0A7FB324601A96B
:104DC00004F1080002F023FB05460028DED1012390
:104DD00084F8A532734084F8A63294F8A932002BE7
:104DE000D4D0002ED2D12046FFF744FF2046FFF753
:104DF00075FFCBE70126D0E70D25C7E70958070067
:104E000032580700375807004352070010B50446D0
:104E1000084900F07AFB94F8A93253B194F8A6320D
:104E20003BB92046FFF726FF2046BDE81040FFF7BC
:104E300055BF10BD3C58070007B5019002F0E2FADB
:104E4000019903B05DF804EBFFF7E0BF38B590F8C7
:104E5000A8320446154603B9FEE7114600F52B704B
:104E600002F0FAFA94F8A93213B12046FFF736FFA0
:104E700041F23C73E35873B104F5BA531B6823B194
:104E80002046BDE83840FFF787BD25B92046BDE87C
:104E90003840FFF78DBE38BD37B50D460446019248
:104EA00002F0B0FA019B2A46214603B0BDE830402B
:104EB000FFF7CCBF2DE9F0411F4600F108039942EE
:104EC00004460D46164600D0FEE790F8A5328BB991
:104ED00090F8A922012380F8A53280F8A6323AB9C9
:104EE0003B46324629462046BDE8F041FFF7D0BB9D
:104EF000FFF7C0FE94F8A932002BF1D02046FFF74F
:104F0000EDFE0028ECD0BDE8F081F7B50D46164661
:104F10001F46044602F076FA009733462A46214699
:104F2000FFF7C8FF03B0F0BD70B50C4686B005466C
:104F3000134920461EF08CFFB0B1043400262068CF
:104F400001A91EF05AFF68B9606805A91EF00FFF9D
:104F500040B9A36893B92868334601AA05F10C014A
:104F600002F061FD06B070BD064920461EF070FFDC
:104F700010B104340226E2E70126E0E70720F1E75A
:104F80008C5907008F59070030B587B004460DF1E2
:104F90000303006801AA0D46FCF7BAFEB8B99DF8F4
:104FA00003303BB10C49204600F0F0F901A920463E
:104FB00000F054FA686805A91EF0D9FE38B9AB684C
:104FC0003BB9206801AA04F10C0102F031FD07B0E1
:104FD00030BD0720FBE700BF0958070000F10C01B6
:104FE000006802F01BBD000013B500F10C0104467F
:104FF0000068019102F003FD40B9064A019920685A
:10500000234602B0BDE8104002F0F4BC182002B004
:1050100010BD00BFE15200000968006867F0D9BA0E
:1050200010B50C680B4634B100F10801BDE8104022
:10503000184600F001BB017A00F078FA204610BD56
:1050400010B50123C0E90012044603723422002186
:105050000C3067F0A9F9204610BD73B53023054622
:105060000C468DF807306126DCB101220DF10701F5
:10507000284602F038F9A8B99DF807305A2B07D016
:105080007A2B0AD0392B0AD141238DF8073001E061
:105090008DF80760013CA4B2E6E73023F5E7013361
:1050A000F3E7204602B070BD70B590B0054601919F
:1050B000322603AA0DF10A0101A8ADF80A601EF01C
:1050C000BDFE044608B124280AD1BDF80A2003A970
:1050D000284602F008F908B1044601E0002CE8D1A6
:1050E000204610B070BD0000F0B58DB00F46012312
:1050F0008DF805300546037A8DF80430262200210C
:1051000002A867F051F9BB68EBB128680DF10603FE
:1051100006AA3946FCF7FCFD0446002857D19DF845
:1051200006303BB12C49284600F030F906A9284644
:1051300000F094F978680DF12A011EF018FE04467B
:10514000002844D10837286801A902F045FC06462A
:1051500000283BD0214938461EF07AFED0B178684D
:105160000DF106011EF003FE044678B9BDF80610E5
:105170003046FFF772FF044640B9286802AB32465A
:1051800005F10C0102F059FC044600B3304602F070
:10519000A2F81CE0124938461EF05AFE28B1796880
:1051A000C1B13046FFF780FFE5E70E4938461EF0F3
:1051B0004FFE00B104373C6864B138461EF041FE32
:1051C00021460246304602F08EF8D4E703242046FA
:1051D0000DB0F0BD0724D9E792590700B859070070
:1051E000453A0700BB5907002DE9FF410B6805460A
:1051F0000C4693B9DFF878801A4F002656F808203D
:10520000394628460C3600F080F9482EF6D123683E
:105210002BBB232004B0BDE8F081134920461EF0CB
:1052200017FE0028E6D123680393104B00930C234C
:105230000DEB03000E49062202F0DDFC03460028B8
:10524000E7D082685B68511005EB6200D20748BF67
:105250006A5804F1040148BFD3589847DAE70020A0
:10526000D8E700BF1B3507001435070019500000B0
:10527000E8590700F0B50446ADF2E45D08460D4676
:10528000164602F02AF80746284602F02AF8114985
:105290003A1A204600F07AF806F11001204600F094
:1052A000CBF8728C0C49204600F070F8284602F0CA
:1052B00018F801AA014640F2DB53284602F015F81F
:1052C00001AA002313540549204600F01EF90DF2EF
:1052D000E45DF0BDBE590700ED3507001B35070042
:1052E000FFF7C8BFC0E9001270472DE970430023E3
:1052F00004460D46137554EA050306D1302302F126
:105300001306D3743046BDE8708302F114062046BC
:1053100029460A22002363F001FF303206F8012DEE
:10532000204629460A22002363F0F8FEA946A0463B
:10533000B9F1000F08BFB8F10A0F04460D46E6D2D6
:10534000E0E7000037B50546072268460C4603F043
:10535000DCFB42F2107303FB05F04FF6FF73B0FB6A
:10536000F3F064230549B0FBF3F203FB1203684634
:1053700003F0F3FB204603B030BD00BF305A0700F6
:10538000D0E9003018474068FFF7FABF0EB403B504
:1053900003AA52F8041B0192FFF7F5FF02B05DF873
:1053A00004EB03B0704700000149FFF7EFBF00BFF7
:1053B000644E07000A46024B0249FFF7E7BF00BFF1
:1053C000F59C0700585A0700F8B5074E07460C46EB
:1053D0008D18AC4206D014F8012B31463846FFF741
:1053E000D5FFF6E7F8BD00BF385A070010B50446F0
:1053F000FFF7EAFF2046BDE81040FFF7D5BF0000E9
:1054000010B586B01946044610466A46FFF76DFF90
:10541000034902462046FFF7B9FF06B010BD00BFA2
:105420001B35070010B50446FFF7EAFF2046BDE82C
:105430001040FFF7B9BF000010B58AB0044628221B
:105440000846694601F07BFE03496A462046FFF79D
:105450009DFF0AB010BD00BF1B35070010B5044604
:10546000FFF7EAFF2046BDE81040FFF79DBF0000B0
:1054700010B58CB004462D220846694601F063FE43
:1054800003496A462046FFF781FF0CB010BD00BFFC
:105490001B35070013B5CC884B880A8864BAA4B2C0
:1054A0000194898849BA89B25BBA52BA00919BB219
:1054B000024992B2FFF76AFF02B010BD3D5A0700E1
:1054C00010B50446FFF7E6FF2046BDE81040FFF7A1
:1054D0006BBF000010B58CB0044630220846694608
:1054E00001F02FFE03496A462046FFF74FFF0CB03C
:1054F00010BD00BF1B35070010B50446FFF7EAFFDB
:105500002046BDE81040FFF74FBF0EB417B505AAFF
:10551000044652F8041B0192FFF735FF2046FFF7BF
:1055200043FF03B0BDE8104003B07047034A044B8B
:10553000002914BF11461946FFF7E7BF4E5A07006E
:10554000B43B07000CB473B506AD044655F8046BC4
:10555000FFF730FF2A46314620460195FFF713FF3B
:105560002046FFF721FF02B0BDE8704002B070474F
:105570002DE9F341DFF83C800D4F14468E18B442FC
:105580000FD041460190FFF701FF14F8015B01982D
:10559000002DF4D03946013D0190EDB2FFF7F6FE43
:1055A000F5E7044902B0BDE8F041FFF7AEBF00BF28
:1055B0001BA3070033A207002DE9F04FDFF870901E
:1055C000DFF870B085B004460E461F46154603F15D
:1055D000FF3802EB810A55451CD055F8043B18F8FA
:1055E000012F03921846029367F0DCFA039A029B9C
:1055F0000230904206D8C2F1010259462046FFF718
:10560000C5FEE8E700934946134620465242FFF79D
:10561000BDFEE0E720460549FFF777FF3A463146F1
:10562000204605B0BDE8F04FFFF7A2BF12350700D6
:105630005C5A0700565A070070B50D4609490646E0
:105640001EF006FC044618B101232B70002070BD2B
:10565000054930461EF0FCFB08B12C70F6E723200C
:10566000F5E700BF635A07006A5A070073B506469C
:1056700008460DF107011546FFF7DEFF044630B975
:105680009DF807103068A847204602B070BD23245B
:10569000FAE737B5054608460DF107011446FFF74E
:1056A000CBFF28B99DF807102868A04703B030BD8C
:1056B0002320FBE770B50E68154604461A461EB156
:1056C000BDE87040FFF7D2BF0068A84701462046FA
:1056D000FFF72CFF304670BD70B50E6815460446C6
:1056E0001A461EB1BDE87040FFF7D3BF0068A84757
:1056F00001462046FFF71AFF304670BD00F14020FA
:1057000000F50030002382B0036003680193019B21
:1057100002B0704708B5094B020103EB0010084BBB
:105720004168C3F84813C168C3F808130089FFF73C
:10573000E5FF044B0021995408BD00BF7C5A0700C7
:1057400000400240E02C002037B521490122D1E879
:105750004F3FDBB28DF807309DF8073063B1BFF3E0
:105760002F8F1C4BD3F804211B4B12B91A68D20798
:105770002BD51868023025E0C1E8432F002BE6D175
:10578000144B0222C3F80823BFF35F8FD3F8043110
:10579000114A4BB1136801331360BFF35F8F4FF4AD
:1057A0008270FFF7ABFF01230A4C10680225C4F892
:1057B0000453BFF35F8F00240C7013B113680133DF
:1057C00013600130400803B030BD1868FAE700BF2D
:1057D000302D002000400240342D00202DE9F04102
:1057E00006460C46FFF7B0FF0546BFF35F8FDFF8B4
:1057F0002080D8F80475BFF35F8FFFF7A5FF3060F6
:10580000854218BFD8F804752760BDE8F08100BF55
:105810000040024013B5044601A96846FFF7DEFFC9
:10582000019A43F6095340F2FF100021E2FB030105
:10583000400A009A064B40EAC150490AE2FB0301C4
:1058400024B94FF47A72002363F068FC02B010BDF3
:105850000080841EF8B5194D05EB001304460601BF
:105860001889FFF74BFF0F462046FFF7D3FF37B9E4
:10587000134B3344D3E90223904299411CD335445E
:10588000104B6A68C3F84823022CEA68C3F808235F
:105890000AD0032C0CD00A4A012393550A4A1370EC
:1058A000BDE8F84000F0ABBFBDE8F84043F0BCBD38
:1058B000BDE8F84043F0DCB8F8BD00BF7C5A0700F3
:1058C000E02C002000400240202D00202DE9F04176
:1058D0003D4D3E4E05EB021C1401DCF80C70C6F881
:1058E0000873DCF80470C6F84473D3E90063B0426F
:1058F0005ED9861B002E00DA013B0026401846EBDD
:10590000060703EB070C311832B94FF47A7303FB27
:105910000CF0A1FB031C84442D4B480B40EACC4007
:105920004FEA5C36A0FB030E03FB06EE000F40EAD5
:105930000E104FEA1E7E43F609534FEA4E2646EA02
:10594000D0564702A0FB0308091A03FB0E8E6CEB2E
:105950000E0C40F23140DFF880E048430EFB0C00B3
:10596000A1FB0E1E0139704447F6FF7140EB0100A8
:10597000C00BC01946F1000720F07F46A0FB0301D1
:1059800003FB071140F2FF13C01841F10001AAB157
:10599000400A40EAC150490A0E4B0C4A2344C3E96D
:1059A00002012B5903F5A87342F82360BDE8F0818A
:1059B000A3D2361A002EB8BF01339EE74FF4FA2265
:1059C000002363F0ABFBE7E77C5A0700004002408E
:1059D000D07B6308E02C00207B2DE8BDF0B585B0BE
:1059E00006460F46684601A91446FFF7F7FE019DDB
:1059F0002A4A43F6095340F2FF100021E5FB030158
:105A0000400A009B40EAC150490AE3FB020124B965
:105A10004FF47A72002363F081FBCDE9020102ABFF
:105A2000224639463046FFF751FF1D4BD3F8043567
:105A30009D4203D001A96846FFF7D0FE019B43F6C3
:105A40000952023340F2FF100021E3FB0201400A39
:105A5000009A124B40EAC150490AE2FB030124B903
:105A60004FF47A72002363F059FB0E4B03EB0413DF
:105A7000D3E90253A84299414FEA041206D3012107
:105A80002046FFF7E7FE40BF05B0F0BD064B1344CC
:105A9000DA68034BC3F80423F6E700BF0080841ED6
:105AA00000400240E02C00207C5A070038B52A480C
:105AB0004022002166F078FC284B00201860284B1B
:105AC0001870284B00240025C3E9004546F000FC6F
:105AD00046F03CFC0028FBD0234BC02283F8242353
:105AE0001022C3F884215A60204A0023C2F80835E6
:105AF0004FF48270FFF702FE0223C2F844334FF4E2
:105B0000A070C2F80433FFF7F9FD4FF48033C2F8F8
:105B100048334FF4A270C2F80833FFF7EFFD4FF49B
:105B20000033C2F848334FF4A470C2F80833FFF7CB
:105B3000E5FD4FF48023C2F848334FF4A670C2F855
:105B40000833FFF7DBFD4FF40023C2F84833C2F8F7
:105B500008330123136038BDE02C0020342D0020D1
:105B6000302D0020282D002000E100E00040024000
:105B70002DE9F04100260B4F0446B0460A4D87F848
:105B800000802B7C1BB120462E7403F093F92B78F8
:105B90001BB120462E7003F055F93B78002BEDD158
:105BA000BDE8F081202D0020E02C00200120FFF72F
:105BB00031BE08B5FFF7FAFF4FF47A72002363F0A5
:105BC000ADFA08BD084611460022FFF707BF0020C6
:105BD000FFF7A0BD08B5FFF7E9FF08BD084611466D
:105BE0000122FFF7FBBE0120FFF794BD704770470D
:105BF000044B4FF48022C3F80823BFF34F8FBFF349
:105C00006F8F704700400240024B4FF48022C3F870
:105C10000423704700400240FFF7DCBF1F2070479D
:105C20000222FFF7DBBE0220FFF774BD7FB5134EE3
:105C3000134D694601A8FFF7D1FD009C43F60952B8
:105C400040F2FF100023E4FB0203400A019A40EAFD
:105C5000C3505B0AE2FB0603CDE90203032202AB59
:105C60003E21FFF733FE4FF40023C5F80433D5F887
:105C700004359C42DDD104B070BD00BF0080841E9D
:105C80000040024037B5044603200D46FFF7C2FD31
:105C90006B46CDE90001032229462046FFF716FE98
:105CA000034B4FF40022C3F8042303B030BD00BF00
:105CB000004002400320FFF72DBD0000214A08B537
:105CC000012353604FF4A070FFF718FD4FF48033A9
:105CD000C2F848334FF4A270C2F80833FFF70EFD44
:105CE0004FF40033C2F848334FF4A470C2F80833BD
:105CF000FFF704FD4FF48023C2F848334FF4A67039
:105D0000C2F80833FFF7FAFC4FF40023C2F8483317
:105D1000C2F808330223C2F808334FF48270C2F885
:105D20004833FFF7EBFCFFF7C5FF074B1022C3F822
:105D30008420C3F88421002283F82423BDE808408E
:105D400046F0F0BA0040024000E100E00048704731
:105D50004C410240014B986B704700BFE02C002083
:105D6000114BD3F8042170B522B10222C3F80823E5
:105D7000FFF7EAFC0D4D0C4E0024D6F80423EB6827
:105D80001A420AD02B8903F1402303F500331B6824
:105D90001BB10021E0B2FFF75DFD0134042C05F1D9
:105DA0001005EAD170BD00BF004002407C5A0700D8
:105DB000FFF7FCBE01238340074982B0DB4351E873
:105DC000002F0192019A1A400192019A41E80020A5
:105DD0000028F4D102B070477C2D0020074A82B021
:105DE00052E8003F0193019B23F001030193019BC3
:105DF00042E800310029F3D102B070477C2D002029
:105E00000123094A82B003FA00F052E8003F0193EF
:105E1000019B03430193019B42E800310029F4D127
:105E200002B000F0ECBC00BF7C2D0020F42382B057
:105E30000B70CE234B7036238B704FF080531A6E4D
:105E40005B6EC1F80330CA7102B0704707B501A894
:105E5000ADF8041042F094FE03B05DF804FB0000BE
:105E6000054B01F1080010F8012D03F8012B8842C1
:105E7000F9D142F087BE00BFD02D002007B501A8A0
:105E8000ADF8041042F080FE03B05DF804FB0000A2
:105E900008B5114B01221A70104B7F221A70104B5B
:105EA000104A1A60104ADA60104A00231370104A30
:105EB000194642F823100833802BFAD110227F2193
:105EC0000C4866F071FA0C482022002166F06CFA4A
:105ED000BDE8084042F065BE793000208B2D0020DF
:105EE000582E0020D92D0020C02D00207830002011
:105EF000782E00208C2D0020A02D002008B542F027
:105F000095FE42F073FE024B00221A6008BD00BFEE
:105F10007C2D002008B50C4B1B7883B942F07AFE2B
:105F200004280ED004D8022814BF0220012008BD86
:105F30000638C0B2022834BF03200220F7E7002051
:105F4000F5E70320F3E700BF79300020034B1A7810
:105F500012B10020187070470D2070477930002072
:105F600010B5084C23784BB9FFF7D4FF012803D0B4
:105F7000054B1B68DB0703D501232370002010BDF0
:105F80000D20FCE7793000207C2D002008B542F080
:105F900050FE28B900F091FDFFF720FF002008BD5A
:105FA0000020FFF71BFFFFF72BFFF7E70B68F7B5A4
:105FB0008A8803F8012C07460C4642F02BFE022883
:105FC00001D100F079FD204600F080FC90B1204620
:105FD00000F081FC70B1E37E9B070BD41C4B204684
:105FE000197800F096FC1B4B196820464A1C1A6071
:105FF00000F091FC6369A07953B125680090226993
:106000000121681E42F02FFEF8B1002501260FE0A5
:1060100042F09CFDE57E206815F0040503D00138B0
:1060200042F060FEF1E72946013842F010FE0646D4
:10603000FFF7D4FE384621460BF03AFC16B9022091
:10604000FFF7DEFE284603B0F0BD0D25DEE700BFFA
:10605000742D0020782D002000487047582E002015
:1060600008B5064B4FF4206043F00103984742F017
:1060700008FEBDE8084042F006BE00BFC05A070057
:10608000FB20704742F010BE084642F00FBE0846A3
:1060900042F00EBE07B5ADF8041001A8002142F091
:1060A00009FE00280CBF0320002003B05DF804FBAC
:1060B00008B50846012142F0FDFD00280CBF032071
:1060C000002008BD07B5ADF8041001A8002142F07A
:1060D000FAFD00280CBF0A20002003B05DF804FB85
:1060E00008B50846012142F0EEFD00280CBF0A2049
:1060F000002008BD002042F0E9BD012042F0E6BDCD
:106100004FF47A7310B55A430A4C0B4B2260084681
:106110001970FFF763FE42F019FD206842F0ABFDF5
:1061200020B10520FFF746FE002010BD0520FFF737
:1061300067FEF9E7842D0020812D002010B50C4664
:1061400021B142F016FD2070002010BD0720FCE7B1
:1061500013B50C4661B101A842F0C2FD054A9DF895
:10616000053012785E3B9B1A2370002002B010BDF0
:106170000720FBE78A2D002013B50A4B1878084446
:1061800040B210F15E0F0BDB0024019442F002FDDF
:106190008DF8050001A842F09CFD204602B010BD1C
:1061A0000720FBE78A2D002021B1034B1B780B70E1
:1061B00000207047072070478A2D0020F7B50B4C50
:1061C000054601A80E4694F9007042F089FD9DF83D
:1061D0000530227826705E3B9B1A59B22846FFF79D
:1061E000CBFF00B1277003B0F0BD00BF8A2D0020A7
:1061F000F8B50026404D044637462B684BB1204683
:10620000002229460BF04CFB28682F60013842F031
:1062100036FD0136102E05F12005EED1374D2B68E5
:106220009B0714D5364E0120FFF7C4FD326835496F
:10623000002A20464FF0000318BF32460BF040FB07
:10624000306820B1013842F01AFD002333602B681A
:106250005F0708D50220FFF7ADFD2A490F23002272
:1062600020460BF02DFB2B681E0708D50320FFF7F7
:10627000A1FD24490E23002220460BF021FB2B68B0
:10628000D80608D50420FFF795FD1F4B00211A788A
:1062900020460BF005FB2B68590608D50620FFF7B2
:1062A00089FD1A4B204693F900100BF016FB2B6862
:1062B000DA0708D542F0BDFC0446A8B900F0FDFBA2
:1062C0002046FFF777FD00242B689B0611D5104B65
:1062D000187842F03BFC0F4B186842F0CCFC28B910
:1062E000BDE8F84000F08BBA0124EDE70520FFF788
:1062F00061FD002CF4D1F8BD782E00207C2D00200B
:10630000A02D0020582E002078300020802D002065
:10631000812D0020842D00202DE9F047DFF8D48066
:106320001F4604468946924600235D0108EB43164A
:1063300058F8051000294DD12022304666F034F877
:10634000631C48F805302378B38086F8159086F8EA
:1063500016A042F00AFCB0716278DFF89C9012F04F
:1063600020023ED1454405F11008EB7D62F30003A5
:1063700088F80730FFF72EFC21788246384642F035
:106380000CFC0746FFF712FCAAEB0703C01A61F1E9
:106390000001C5E90201002389F800306378124C3E
:1063A00013F0200F10D0304600F086FA60B198F854
:1063B0000730227862F3410388F807300B4B1B68E3
:1063C0002B610B4B1B782B7500232370BDE8F04726
:1063D00000F015BA0133102BA7D1002301341C6043
:1063E000FFDE99F80020BDE7402D00203C2D002065
:1063F000382D0020782E00209C2D0020431E092BD4
:1064000009D8DFE803F00516191C1C1C1C051C1C10
:106410000D4B12221A700D4A002313700C4A0828E3
:10642000137001D005280DD1074A00201370FFF723
:10643000E7BC054B1122EDE7034B1622EAE7024BBE
:106440000122E7E70420F2E7783000209C2D0020AD
:10645000402D002070B54378234A244EC3F3001129
:1064600088B01B0711704FF000010446317034D51D
:106470001A220DF1060065F097FF631C0093684631
:106480002378ADF8043000F037FA0446684600F08F
:1064900022FA10B30CB3164B1B789C421FD05A1E25
:1064A00094421ED001339C4217D1124B124D134A15
:1064B00029681160124A029314702146012268462D
:1064C000327000F026FA296868464B1C2B6000F0F9
:1064D00022FA0C49684600F0EDF908B070BD0A4B8D
:1064E000E4E70A4BE2E700BF9C2D0020402D00208E
:1064F000742D0020442D0020782D00203C2D0020FC
:10650000382D0020D02D0020542D0020642D002097
:106510002DE9F047DDF820A0144C90461F460D46AB
:1065200029B92160BDE8F0470120FFF769BCFFF7FA
:1065300051FBA946064619F8011B504642F02DFBB7
:106540008246FFF733FBA6EB0A06801B61F10001D0
:10655000C4E90201C4F800902B78A38084F8158068
:10656000A77542F002FBA071DCE700BFA02D002060
:1065700007290ED8012303FA01F111F0D20F03D13C
:1065800011F02C0F03D170470220FFF739BC032014
:10659000FBE7704708B542F0F9FA034B1870BDE805
:1065A00008400620FFF72CBC802D00206FF0630010
:1065B0007047000010B50A4C204600F087F970B112
:1065C000204600F088F950B1E37EDB0607D4054B86
:1065D000A36020460449BDE8104000F06BB910BD2F
:1065E000582E0020542D0020D02D002070477047D9
:1065F00000F0F6BEFFF7DCBBF8B50020DDE906656C
:1066000017461C4645F028FE0A4B1F7094E80F0001
:10661000094F0A4C87E80F0096E80F0084E80F0046
:1066200095E80F00064C84E80F00BDE8F840002014
:1066300045F014BE742D0020642D0020542D002040
:10664000442D002010B500200C4645F005FE034BFC
:1066500000201C60BDE8104045F000BE782D0020F1
:1066600010B500200C4645F0F7FD054B1A68A24214
:1066700038BF1C600020BDE8104045F0EFBD00BFF2
:10668000782D0020A0F10B030F2B9DBF024B1B1890
:1066900013F90B0C7F2070478C2D002008B5FFF7F5
:1066A000F1FF074B93F900307F2B04D09842A8BF2D
:1066B000184640B208BD7F2808BF0020FAE700BF97
:1066C0008B2D002010B508460C4642F03FFA42F0F0
:1066D000A1FA022801D100F0EFF92046FFF7DEFF12
:1066E00042F045FA42F0ADFAFFF778FB00280CBF04
:1066F0000D20002010BD000010B50C4642F035FA08
:106700007F2C07D0044B1C70FFF7C8FF42F02FFA14
:10671000002010BD0720FCE78B2D002021B1034B8A
:106720001B880B800020704707207047882D0020B1
:106730007047000008B5034B08461980FFF7F8FFC3
:10674000002008BD882D0020FEE7000010B50C4C8D
:1067500000F0B1F900F05EF8FFF7D0FB00F0CEF9E1
:1067600023780BB900F0BBF9207800F04EFA00F066
:106770008DF9FFF7A3FABDE8104000F0A1B900BF02
:106780001031002010B5124C23780BB1FFF7DEFF5B
:10679000104B0122C3F8402545F082FD00F08EF930
:1067A000FFF784F900F02CF923780BB900F0B5F865
:1067B000207800F025FA00F093F9FFF769FB00F06C
:1067C0001FF800F077F900F0A8F80023237010BD3F
:1067D0001031002000E00140014B1878704700BFE5
:1067E0001031002010B50446FFF702FD00F011FA49
:1067F00000F016F82046BDE81040FFF7B9B9704721
:10680000034B0022C3F8042501221A60704700BF21
:1068100000C00040014B01225A60704700C0004098
:106820001A4BF7B51A4CD3F8002125688AB100221B
:10683000C3F80021D3F800210192019AD3F808256A
:10684000D3F80835920544BF6FEA83536FEA935338
:106850002360FFF7ABF90F4B0F4FD3E90026821AE5
:1068600061EB060697424FF00002B2413FBF074A74
:1068700001261660C3E900012368AB4204D003B0CF
:10688000BDE8F04042F07AB903B0F0BD00C000406E
:106890007C3000208030002080C3C90170477047E1
:1068A000034B18680028B8BF033040F387007047D7
:1068B0007C30002005F02DB808B504F027FC00F46A
:1068C0004050A0F500535842584108BD036818785D
:1068D000C0F3C000704707B50DF1070104F078FE62
:1068E00040B99DF80700A0F108035842584103B091
:1068F0005DF804FB0020FAE707B500230DF107015E
:106900008DF8073004F0B4FE9DF8070003B05DF881
:1069100004FB04F0C3BE04F07BBE704708B545F02D
:10692000E3FE002008BD08B5086845F033FF0020ED
:1069300008BD08B5104645F0F1FE80F00100C0B278
:1069400008BD002070470000074A084B196813680B
:1069500099421FBF1368591C116003F07F031ABFCF
:10696000034AD05C002070478C3000208830002023
:1069700090300020074B002282B0C3F80021D3F8EA
:1069800000210192019A0122C3F804231A6002B087
:10699000704700BF00D00040154BD3F8002113B55D
:1069A00022B3D3F80823D20720D50022C3F8002150
:1069B000D3F800210192019A0E49D3F808450E4BF5
:1069C0001A680868121A7F2A06D81A68501C1860BC
:1069D00002F07F02094884541B680A689B1A7F2BC7
:1069E00081BF034B0122C3F808235A6002B010BDD7
:1069F00000D000408C3000208830002090300020F3
:106A000038B5802200211C4865F0CEFC1B491C488B
:106A100000230B6003601B4BC02283F80D234FF44F
:106A20000052C3F880211A60174BD3F8042542F0B6
:106A30000102C3F80425D3F8002222F00102C3F8B2
:106A40000022FFF797FF03680A689B1A032BFAD905
:106A500003680A689B1A032B0CD904250020040242
:106A6000FFF772FF013D40EA0400F8D1BDE838406D
:106A700066F07ABF0020F9E7903000208C300020CB
:106A80008830002000E100E000D00040074B0122E8
:106A9000C3F808235A60064B4FF40052C3F8802015
:106AA000C3F88021002283F80D23704700D00040F6
:106AB00000E100E0704770477047704700F040B851
:106AC00000F04CB80CB407B504AB53F8042B019399
:106AD00000F04AF803B05DF804EB02B0704770476D
:106AE0004FF08043044AD3F8001411604FF0FF3296
:106AF000C3F80024704700BF143100207047000025
:106B000008B500F088F80A4B187018B1094B042238
:106B10001A6008BDBFF34F8F0749084BCA6802F4DB
:106B2000E0621343CB60BFF34F8F00BFFDE700BFB0
:106B3000103100201431002000ED00E00400FA05BF
:106B400008B50121002045F059FB0028A2BF024BE7
:106B500001221A7008BD00BF18310020014B00222D
:106B60001A7070471831002070B51E461E4B1B78F6
:106B7000A4B004461546002B33D0FFF71AF81B4B80
:106B80001B4A0090802103A866F08CF9601E032840
:106B900096BF184B184B53F82030184A6D210DF151
:106BA0001F0066F07FF9133084B22A4603AD3346E6
:106BB000C4F1800115FA80F067F05CFA002810DB60
:106BC0000444A4B2802C28BF802404F190036B44B9
:106BD0000A2203F8842C621C92B22946002045F058
:106BE000E1FA24B070BD00BF18310020CB5A070075
:106BF000D35A0700FC5A0700C65A0700DE5A07009E
:106C000008B900F00AB800F009B808B900F092B865
:106C1000704700F03DB90020704770477047000092
:106C200030B52E4D287885B0002855D14FF0A043BF
:106C30002B4C4022C3F8082506210322C3F818274D
:106C4000C3F82007C4F80C150821C4F81415202136
:106C5000C3F81C07C3F80815C3F814270523C4F8A4
:106C600008350723C4F810350123C4F86C354FF0FC
:106C7000EB73C4F82435C4F82001D4F82031039311
:106C8000039BC4F82401D4F824310293029BC4F876
:106C90000801D4F808310193019B4FF48073C4F8C4
:106CA00004334FF40173C4F804330E4BC02283F84D
:106CB00002230422C3F880211A6045F04FFB45F0FF
:106CC0008BFB0028FBD00823C4F800350123236088
:106CD00000202B7005B030BD1820FBE724330020C6
:106CE0000020004000E100E038B50F4D2B78C3B123
:106CF0000E4B00240422C3F88020C3F8802183F8BF
:106D000002430B4B4FF48072C3F808234FF4017217
:106D1000C3F80823C3F8004545F04AFB2C70204611
:106D200038BD1820FCE700BF2433002000E100E05C
:106D300000200040024B1B780BB1FFF7D5BF704716
:106D4000243300201FB5284BD3F8042391051ED50A
:106D5000D3F82421DAB10022C3F82421D3F8243156
:106D60000193019B204BD3F82021002A3AD0002226
:106D7000C3F82021D3F8202103921C49039A012251
:106D80000A70DA6004B0BDE81040FFF738BDD3F8F0
:106D900004235207E6D5D3F80821002AE2D00022C6
:106DA000C3F80821D3F8082111490292029AD3F8B6
:106DB00018450A880F4892B284540A880132C2F3F7
:106DC00008020A800A880C4909880132C2F30802C5
:106DD00089B2914204BF4FF40172C3F80823FFF750
:106DE0000EFDBFE704B010BD002000401E330020A0
:106DF0001C3100201E3100201A310020064908B540
:106E00000B683BB1054B1A7822B100220A601A7058
:106E1000F9F72CFD08BD00BF203300201E330020F1
:106E200008B5054B1B681BB1044A1378002BFCD036
:106E3000FFF7E4FF002008BD203300201E330020B0
:106E400073B5104D2B6804460E4683B90E4B2C606B
:106E50000020C3F82001D3F820210192019AC3F841
:106E600044450122C3F848659A6002B070BD074BE3
:106E70001B780BB10520F8E7FFF7D2FF2B68002B3A
:106E8000E4D0F7E720330020002000401E3300202C
:106E900038B51A4B1A4C1D881A88238892B29BB2B7
:106EA0009A42ADB226D023889BB29D420BD2208855
:106EB0002188144BC1F5007113FA80F089B2F9F7FB
:106EC00075FC0023238023889BB29D4209D920882A
:106ED00021880C4B691A89B213FA80F0F9F766FC25
:106EE0002580094BD3F8042352075CBF4FF401728D
:106EF000C3F80423BDE83840FFF780BF1C310020F1
:106F00001A3100201E3100200020004000F5FF4013
:106F1000243000F0B3BD48F20203C05A704700F5B8
:106F200000400BF0F9BF00F500400088704700F505
:106F300000400CF027B848F20403C05A704748F2EA
:106F400004030022C252704700F5A640383005F015
:106F5000E0BD00F5A640343005F0C8BF00F5A640FE
:106F60006C3005F0D6BD00F5A640683006F08BBA4F
:106F700000F5A640343006F009B900F5A6403430DB
:106F800006F0B2B800F5A640683006F0FFB800F58C
:106F9000A640683006F0A8B806F0D4BD08B507F0E2
:106FA00039F9182808BF002008BD30B5C3B0054620
:106FB00068460C4605F034FA6846294605F01BFB86
:106FC000684605F039FA30B16846214605F05AFAAC
:106FD000002043B030BD0720FBE730B5C3B0044606
:106FE00068460D4605F01CFA2146684605F0E2FBAE
:106FF000044618B92946684605F0EFFA204643B022
:1070000030BD30B5C3B004460D46684605F008FAF9
:107010002946684605F0EFFA2146684605F0CAFBA6
:10702000044618B92946684605F0D7FA204643B009
:1070300030BD00000846014905F08AB90837002034
:1070400047F65C73C058704700F5FE404C3006F0C0
:107050005BBE00F0F3BD02F05BBB48F23413C058D6
:10706000704748F23013C05C704702F061BB02F019
:107070003DBB143001F044BF143001F0B9BF02F041
:107080007ABB0000004870470C5B070000F5A24087
:1070900008B57C3019B11CF0F1F9002008BD1CF0D6
:1070A00017FAFAE745F22023C05C704745F27C13DB
:1070B000C058704700F5A2407C3009F024B900F5B3
:1070C000A2407C3009F0D7B800F5A2407C3009F02E
:1070D00032BA00F5A3400068704700F5A2407C304A
:1070E00009F008B800F5A2407C3009F0C5B945F2B6
:1070F0008413C05C704745F28413C154704700F597
:10710000A7400A465230002108F0F8BB00F5A7401E
:107110000A465230012108F0F1BB45F2D633002275
:10712000C254704745F2D633C35C0B7000F5A740DC
:10713000523070470B460146184608F00FBB08F066
:1071400087BB09F041BA08F067BB45F26A43C05CEF
:10715000704738B545F2A9630446C35C93B900F59E
:10716000A840603002F07AFF054648B904F5A64011
:10717000343005F0DFFD04F5A640683006F022F952
:10718000284638BD0D25FBE700F5A94014307047AF
:1071900038B545F2A9630446C55C5DB900F5A94060
:1071A0000C3004F063FD04F5AD40283011F064F9B3
:1071B000284638BD0D25FBE70148FEF737BE00BF66
:1071C0000837002045F26843C05A704738B545F289
:1071D000A9630446C55C85B900F5A840603002F09B
:1071E00037FE04F5A640343005F0A4FD04F5A640B2
:1071F000683006F0E7F8284638BD0D25FBE700F5B6
:10720000AD40083002F0A1BB00F5AD40083002F0FF
:10721000B2BC45F27843C05C704745F27843C15434
:10722000704745F27943C05C704745F27943C154D9
:10723000704710B545F2AC43C418C150626010BD30
:1072400045F26043C05CC0F3C000704745F22023A4
:1072500010B5C45C34B900F5A840603003F0BEFA44
:10726000204610BD0D20FCE745F2202310B5C45C7C
:1072700034B900F5A840603002F074FD204610BD1E
:107280000D20FCE700F5AA401030704700F5AA4039
:1072900088220021103065F087B800F5A8406030E2
:1072A00002F029BF00F5A840603002F049BF00F5A8
:1072B000A840603003F0AEBA21B100F5A8406030BC
:1072C00003F0C4BA07207047012070470FB404B020
:1072D000704700F001BD00F03EBEC08B704700F06B
:1072E0003EBE008C704700F046BF00F0D2BE10B525
:1072F0001C4600F01DFF204610BD02F046BA02F009
:107300008EBA0B4600220146184607F04AB870B5FF
:1073100000F5FB4086B00E4604306946154618F06D
:1073200066FB044638B932466946284608F071F9CA
:10733000204606B070BD0D24FAE700F5FB4004308E
:1073400018F000BB47F68853C05C704747F68A6365
:10735000C05C704747F6885200F5FB43825C83F8B7
:107360000A21704700F5FB40043018F09DB800F585
:10737000FB40043018F0A8B800F5FB40043018F0CA
:10738000B3B800F5FB40043018F0B3B800F5FB408B
:10739000043018F086BD00F5FB40043018F0FEBD47
:1073A00000F5FB40043018F009BE000000487047AB
:1073B000565F070000487047575F07000048704756
:1073C000595F070000487047585F070000F500400C
:1073D00084301CF033BE00F5004084301CF0ACBD9E
:1073E00001F0E0BA10B50446FFF73BFE20B1201DC6
:1073F000BDE8104001F04ABC10BD0B4601461846DE
:1074000009F0FABCD0F81C02704709F0A6BB09F0DD
:10741000FBB809F05CBA09F034B909F03FB909F0DA
:1074200057B909F05CB909F05FB90B460146184637
:1074300009F0ECBA006A704709F0B3BB09F006BB6B
:1074400009F00FBB09F027BF10B4044608462146D7
:107450005DF8044B09F05ABF09F025BF09F03CBFA5
:1074600009F03EBF09F042BF1FB50023019303ABF3
:107470000093144613460A46D0E9001009F046FF6F
:1074800020B9039804B118B104B010BD0148FBE75E
:107490000148F9E70094FFFF8097FFFF2DE9F743CC
:1074A000D0F800908846484601A91546FFF7B3FF7B
:1074B00008BB0446AC4202D0019E4EB9BDB90022C1
:1074C00021464846FFF7A9FF204603B0BDE8F083F8
:1074D000B26871682F1B974228BF174608EB04005B
:1074E0003A4665F045FB336801933C44E2E7002CE3
:1074F000E5D10248E9E70248E7E700BF0097FFFF50
:107500000094FFFF45F2C463C058704700F5AD40DA
:10751000283013F0D7BB00F5A7402830704738B5A6
:1075200045F2A9630446C55C85B900F5A74028303B
:1075300005F0E8FF04F5A640343005F0FBFB04F548
:10754000A640683005F03EFF284638BD0D25FBE714
:1075500007B545F2AA636946C35C8DF8043001A8FB
:1075600017F059F89DF8000003B05DF804FB13B55F
:1075700004468DF80410684601A917F05FF804F579
:10758000AD409DF80010283013F0B4FB02B010BDE0
:1075900000F5A74058300DF076BC38B545F2A96328
:1075A0000446C55C85B900F5A74058300DF05AFD7A
:1075B00004F5A640343005F0BDFB04F5A640683064
:1075C00005F000FF284638BD0D25FBE700F5B0406B
:1075D0006030704700F5B0404830704700F5B0406B
:1075E0003030704700F5B0407830704700F5B1405A
:1075F0000C30704700F5A7403030704745F2A96263
:1076000038B5825C0546A2B9A9B10B789BB100F5EB
:10761000A740303006F026FE044605F5A64034307B
:1076200005F088FB05F5A640683005F0CBFE204646
:1076300038BD0D24FBE70724F9E700F5A7404130EA
:10764000704745F2A963C35C23B900F5A740303009
:1076500006F01CBE0D20704745F2E833C058704755
:1076600000F5A740012258300DF072BC45F21E43D0
:10767000C05A704745F21E43C152704700F5AD40F5
:10768000283012F001BB00F5AD40283012F0E2BA0C
:1076900000F5AE40143017F06DBD45F2A963C05C33
:1076A000704717F013B838B500F5AD4428342046BC
:1076B0000D4610F011FE38B1204610F0B5FF03C89A
:1076C00085E80300002038BD1020FCE708B500F570
:1076D000AD40283010F0A8FF006808BD45F2B8633F
:1076E000C05A704700F5AD40283011F0A9B900F537
:1076F000AD40283012F0BCBA00F5AD4010B52830CE
:107700000C4621B1BDE81040002113F0CFB9012192
:1077100010F030FE204610BD0420704700F5AD404B
:10772000283014F09CBA7FB505910A990391099904
:1077300002910021019100F5F1409DF82010009187
:10774000703005A90CF030F807B05DF804FB00F5C7
:10775000AB407C30704700F5AB40102200217C30FC
:1077600064F022BE10B500F5AD442834617820469F
:1077700010F0EAFC04F5807010BD00F5AD40283033
:1077800010F0D2BC00F5AD40283013F0ADBB13B5FE
:107790000446684601F0B9F94FF47A7000236A464E
:1077A000A4FB000101F0D4FB02B010BD45F6C803F4
:1077B000C05A704700F5B14048300BF01ABD00F5D3
:1077C000AD40283014F0C1BB00F5AD40283013F0B7
:1077D0001DBF00F5AD40283013F042BF00F5AD40AD
:1077E000283015F027BC47F6B703C05C704747F652
:1077F000B703C154704700F5FE4005F0C3BE08B59D
:1078000000F5FE4005F015FF002008BD47F6C863EF
:10781000C058704747F6C863C150704747F6B40375
:10782000C05C704747F6B403C154704747F6B503D0
:10783000C05C704747F6B503C154704747F6C803AC
:10784000C05C704700F5AD40283015F039BD3E29C9
:1078500004D800F5E34050301BF0D0B80720704743
:1078600045F2A963C35C022B05D0033B012B94BFF7
:1078700000200D20704700F5AD400321283015F0A1
:10788000A1BC00F5AD40283015F0EAB947F6B603C3
:10789000C05C704747F6B603C154704747F6C7034C
:1078A000C05C704747F6C703C154704700F5B1404C
:1078B00048300BF0AFBC00F5B14048300BF0C4BC11
:1078C00030B500F5B14087B0483015461C460BF086
:1078D00009FC80B3837F03F00F03012B02D0063B2A
:1078E000012B28D82B88009000226846ADF806307E
:1078F0008DF804200BF00EF9BDF80630052B02D9E7
:10790000172007B030BD68460BF0ABF800F110034C
:1079100050F8042B44F8042B9842F9D1BDF80630F6
:1079200068460133ADF806300BF0F4F8BDF80630C8
:107930002B800020E5E70720E3E73E20704700F5B5
:10794000E34050301BF0ABB800F5F240603009F076
:10795000F1BF00F5A74058300DF0A4BA38B545F294
:10796000A9630446C55C85B900F5A74058300DF001
:10797000A5F904F5A640343005F0DCF904F5A6407D
:10798000683005F01FFD284638BD0D25FBE747F69A
:10799000C903C056704700F5AD40283016F060BAF4
:1079A00010B547F6E403C418C150626010BD00F57D
:1079B000F0406030405CC009704707B500F5E34017
:1079C00050300AB90DF106020BB90DF105031BF099
:1079D00015F903B05DF804FB10B50446084600F045
:1079E00093FA024604F5A1400021BDE810402C3076
:1079F00009F0DCBD00F5A1402C3009F0FCBE45F2D9
:107A0000B403C3581BB1994206D01B6BFAE7172089
:107A1000B0FA80F0400970470020F9E700F5A14076
:107A20002C3009F011BF00F5A1402C3009F062BDE7
:107A300000F5A1402C3009F0A1BD10B492F83240FD
:107A400014F00C0F06D000F5A1405DF8044B2C306B
:107A500009F0E2BD07205DF8044B704745F2B4031E
:107A6000C05870474FF6FE720280002202777047BE
:107A70004FF6FE7303800023037770470B4601889F
:107A80004FF6FE7291421DBF07C883E80700002031
:107A90001720704707B502884FF6FE739A4209D047
:107AA00001230091044805491A4619F04FFC03B020
:107AB0005DF804FB1720FAE700B60020555F0700C9
:107AC0007FB5054601AE2348314619F099FCBDF853
:107AD00004202C88A2424FF6FE7320D09A4235D063
:107AE0009C420CBF01240324029B1B4AB3F5967FE2
:107AF00038BF4FF49673934294BF0293029296E874
:107B0000070085E807002A462146144816F082FF40
:107B100013482A4621460CF0F3F804B070BD9A428F
:107B200016D09DF80C202B7A9A420BD1BDF8062076
:107B30006B889A4208D16C68029B9C4214BF042453
:107B40000524D1E70324CFE70424CDE70224D6E7B8
:107B50000024D4E700B600209BC42000CCB600204F
:107B6000D4B6002070B588B00023174C01930546A9
:107B700002AA01A9204617F097FCB0B99DF81A3067
:107B80005B07F5D505F10C04214602A807F01FFBA1
:107B900048B92E7F02AD0FCD0FC4002E2B68237085
:107BA00018BF02260AE0032608E02B7F53B11122FA
:107BB000002105F10C0064F0F7FB01260348314673
:107BC0000CF054FB08B070BD8CB40020D4B600207B
:107BD00010B50446FFF774FF2046BDE81040FFF7DC
:107BE000C1BF034608461A7F1AB103F10C0107F022
:107BF00059BC104670472DE9F84F0A9D80468946CA
:107C000016469A464FF0000BB34512D20BEB060412
:107C1000671007FB0A9739464046A8470028C4F377
:107C20004F0407D003DD01341FFA84FB3446264697
:107C3000EAE700273846BDE8F88F000025289ABFFC
:107C4000024B53F820000248704700BFE85C070071
:107C5000475B0700F0B5ABB004460D46164604A9D5
:107C6000962202A81F4600F050FF0E21204600F089
:107C7000E1FE0E4B0E491844009023460E220D4C97
:107C800002A800F06AFF3A46314602A800F044FF1D
:107C90002146094A02A800F060FF04AB22461021E9
:107CA0002846FEF70FFF2BB0F0BD00BFA15D070017
:107CB000805D07001B350700F59C07000EB403B577
:107CC00003AB012153F8042B0193FFF7C3FF02B06C
:107CD0005DF804EB03B070472DE9F74F044600F15F
:107CE0000C014922684600F010FFB4F856504FF6D8
:107CF000FE739D425DD04FF6FF739D4200F097806A
:107D00009DB34FF6FD739D425BD0B4F856504A497F
:107D1000DFF83491DFF834A1DFF828B1684600F0CD
:107D20001CFF4FF6EF736F1E9D428CBF0123112382
:107D300005F110081F441FFA88F8BFB22E46BE4254
:107D400048D0A388B34240D9236851469A5D68461B
:107D500000F003FF06F00703072B03D159466846DE
:107D600000F0FBFE0136B6B2E9E73E21A06800F064
:107D700061FE00F10A06B6B2C6F1480606EBD672FD
:107D800057103D21C2F34F02684600F0F5FEA3886C
:107D9000A2682A49684600F0E0FEF21B92B23D213B
:107DA000684600F0E9FE4FF6FD73A4F85630002057
:107DB0003EE048222D21684600F0DEFE4FF6FF73BC
:107DC000F3E70023A4F856309FE74946684600F0E1
:107DD000C4FEBFE71A49DFF87890684600F0BDFEA0
:107DE000AE4218D0A388AB4211D923685F5D7E2FC5
:107DF0000FD8384664F050FA002808BF2E273A46BC
:107E000049466846013500F0A8FEADB2E8E72027F4
:107E1000F5E72E27F3E70B49684600F09EFEA3889E
:107E2000A4F856804345C2D84FF6FE73BDE717202D
:107E300003B0BDE8F08F00BF12350700895D070071
:107E400070A00700113507009D5D0700975D0700D2
:107E5000F548070010B5002300F5A1424360083241
:107E600000F1080319468033934204D0446843F874
:107E7000804C4160F6E745F208030022C25010BD75
:107E8000F8B50F4E04460F46656895B145F20802F5
:107E90002B686360A35A01339BB2A35245F20A01D7
:107EA000625A934238BF1346635200232B60284620
:107EB000F8BD394630460FF075FC0028E4D0F6E7EF
:107EC000B88C002010B500F5A043083341B14268DA
:107ED0000C680A601A884160013A1A802146F5E769
:107EE00010BD4A681AB98B680BB9FFF7EBBFFEE704
:107EF00045F20803C05AC0F1A00080B27047A0202C
:107F00007047017042707047024B002808BF184646
:107F1000704700BFB05D0700F8B504460F46054640
:107F20004C26BE422968E0680FD219B17C362D6814
:107F3000B6B2F6E794F83110C1F34101FFF7A0FFA4
:107F400028600028F2D1032004E000242C60FFF711
:107F5000B9FF2046F8BD0146C068FFF7C2BF38B57B
:107F6000838B0D46194489B29942044608D3FFF722
:107F7000D3FF20B9238CE583AB4200D9258438BDDB
:107F80000720FCE7036801201BB101301B68C0B269
:107F9000FAE77047038CC28B1944914200DDFEE77B
:107FA00089B29142018400D9FEE77047C38B8B42AE
:107FB00000D2FEE70184704790F83030C3F3C3036A
:107FC0000A2B09D8012202FA03F340F24E7213423F
:107FD00014BF01200020704700207047C38B8B42E4
:107FE00000D2FEE75B1AC383038C828B8B420A4468
:107FF00086BF591A89B2002182830184704730B547
:10800000C48BA1420BD300219980118898888842A3
:1080100088BF998011889B88CB1A138030BD158842
:108020000D44A542A4BF641A1480848B9860214437
:1080300089B24B29044605D8343008441860C1F190
:108040004C01E1E74C39246889B20CB99C60FEE729
:108050007B2906D89C6004340C441C60C1F17C016F
:10806000D2E77C39EFE70B880BB9938070479368B0
:108070001B68936003B9FEE7043313607C2393808D
:108080000B887B2B98BF93800B8892889B1A0B8060
:108090007047F0B587B01546ADF806300DF1060211
:1080A00003AB0646FFF7ABFF2C46BDF8107067B177
:1080B00003993A46204664F05BFD03AA0DF10601E0
:1080C00030463C44FFF7CFFFEFE7601B80B207B0BC
:1080D000F0BD10B51C46FFF7DCFFA04214BF062020
:1080E000002010BD70B586B01546ADF806301C46B0
:1080F0000DF1060203AB0646FFF781FFBDF8102025
:108100008AB10A9B039829461DF098FB58B1BDF827
:10811000103003AAE41A0DF1060130461D44A4B242
:10812000FFF7A1FFEAE7B4FA84F0400906B070BD9A
:1081300030B587B01446C28BADF806300B4493427D
:10814000054600DDFEE703AB0DF10602FFF757FF22
:10815000BDF810206AB12146039864F00BF9BDF810
:10816000103003AA0DF1060128461C44FFF77BFFDF
:10817000EEE707B030BD2DE9F041B0F81E800F46A4
:1081800008EB020189B205461646FFF7E8FE0446F1
:1081900028B933463A4641462846FFF7C9FF2046EC
:1081A000BDE8F0812DE9F0410D46C98B86B0174638
:1081B0001A4491420646ADF8063022DBB0F81E8024
:1081C000434499B2FFF7CBFE0446D8B903AB0DF197
:1081D000060239462846FFF712FFBDF810308BB172
:1081E000039A41463046FFF7A3FFBDF8103003AABB
:1081F00098440DF1060128461FFA88F8FFF733FF6F
:10820000EBE70624204606B0BDE8F081F8B5044649
:108210000D46164600F13407A38B9E4218D994F8F8
:108220003110E068C1F34101FFF72AFE30B3236843
:108230000360A38B20604B2B06D83430C3F14C0273
:10824000F918184464F094FCA38B7C33A383E3E710
:108250009B1BE28BA383238C3244334492B29BB2A8
:108260009A42E28300D2FEE723844DB12046334692
:108270002A460021FFF75CFF0020F8BD0320FCE741
:108280002846FAE7F0B582420D4689B00646144604
:10829000194601D1AB4216D36B460EAA2046FFF712
:1082A000AEFEBDF804307BB3009A29463046FFF796
:1082B0003FFFBDF804106A460D4420460EA9ADB23A
:1082C000FFF7D1FEEDE7BDF838201544D318ADB265
:1082D0009CB2BDF83830BBB1202B1F4628BF2027E9
:1082E000E41BDB1BA4B2ED1BADF838306A463B46FD
:1082F0002146ADB23046FFF7CCFE3B466A462946E2
:108300003046FFF715FFE4E709B0F0BD37B5154675
:1083100000910246294600230446FFF7B3FF294691
:10832000204603B0BDE83040FFF758BE1F2900D9F2
:10833000FEE700EBD100802390F82C2001F007012C
:1083400043FA01F10A4214BF0120002070471F299F
:1083500000D9FEE700EBD100802301F007010B41BB
:1083600090F82C1021EA030180F82C1070471F2987
:1083700000D9FEE700EBD100802301F0070143FAAA
:1083800001F190F82C30194380F82C10704700F15F
:108390002C033030834205D013F8012B002AF9D08A
:1083A000012070470020704738B50B8883848B7894
:1083B00080F826300D46044691F9031028300CF061
:1083C000CDFE297904F12A000CF0FBFE6B7994F8BC
:1083D0003120C3F3000363F3000284F831206B798A
:1083E00094F83220C3F3400363F3410284F832204F
:1083F00038BD0B6910B503B1FEE74B6873B98C68E3
:1084000064B991F83130086164F3C30381F8313005
:10841000036823B9C1E90111016009E0FEE75B6867
:108420004B6004688C6099600368012A5960F3D03E
:1084300010BD91F831301B0754BF0B6900239842DF
:1084400000D0FEE74B68C3B18B68B3B102689142BC
:1084500003D1994208BF00230360D1E90132536080
:108460008A689A6091F83120002363F3C302C1E95E
:1084700001330B6181F831207047FEE710B5FFF73B
:10848000D8FFBDE810400846FFF765BD10B50446AB
:1084900023682BB1596819B12046FFF7EFFFF7E7C2
:1084A00010BD006800B14068704702460B4652F8A4
:1084B000230030B9032B1ABF0133DBB203469942C4
:1084C000F5D1704708B50021FFF7EFFF00B1406814
:1084D00008BD08B550F821304BB103291ABF01314E
:1084E000C9B20021FFF7E1FF00B9FEE74368184673
:1084F00008BD0021FFF7D9BF10B50446006994F804
:1085000031301B0707D528B1FFF7F3FFA04214BF96
:108510006068002010BD0028FCD00068F6E710B5A8
:108520000C46FFF7BEFF024678B123880133238053
:10853000FFF728FD6388D18B1844636860800B4483
:1085400063601046FFF7D8FFEDE710BD10B5044695
:10855000086818B920606060204610BD406820603F
:108560000028F8D0FFF7C8FFF5E710B504464068CB
:10857000206008B1FFF7C0FF606010BD38B50B691F
:1085800005460C4603B1FEE7086191F8311041F051
:10859000080184F83110C1F34101FFF786FF38B1BB
:1085A0004368C4E901309C60446045F8214038BD0F
:1085B000C4E90144F9E791F8313010B51C07C3F361
:1085C000C00248BF0A69904200D0FEE7C3F34103EE
:1085D00050F8232091420BD18A68914218D092F82A
:1085E0003140C4F341049C4218BF002240F82320CC
:1085F000D1E9012393604A685A600023C1E901333D
:108600000B6191F8313043F0080381F8313010BD2F
:108610000022EBE7032938B504460D461DD8006952
:1086200038B994F8313065F3420384F831300020D2
:1086300014E094F83130C3F341028A42F7D01B07AB
:10864000EFD52146FFF7B7FF94F8313065F34203C9
:1086500084F83130FFF792FFE9E7072038BD2DE9B4
:10866000F0410D465978074690461E46FFF708FC34
:10867000044648B38022002163F096FE3178238EB1
:10868000E76005F0070545EA012525F0F805ED0549
:1086900023F4837323F00103ED0D1D4394F832306E
:1086A000A4F81C8023F00D0343F00503258684F80D
:1086B000323071782046FFF7ADFF014638B12146D0
:1086C0003846FFF70EFC00242046BDE8F081204626
:1086D000FFF745FC0028F7D0F1E70000014B00222E
:1086E000FFF7BDBFB05D0700014BFFF7B8BF00BF8C
:1086F000B05D0700F7B590F83130C78B0E4690F8A3
:108700003010C3F30002C3F341038DF804208DF849
:108710000530828B054601ABC06801F00701FFF709
:108720009EFF044600283DD0BE4228BF3E46334649
:1087300000222946FFF736FD002836D12A8C134641
:10874000B242E28B28BF33469A4200D2FEE723842E
:1087500095F8303094F83020C3F3C30363F3C602B6
:1087600084F8302095F8322094F8323062F3000318
:1087700084F8323095F8323094F83220C3F3810314
:1087800063F3830284F83220AB69A3616B8C63844A
:10879000AB8CA38495F8263084F826302B8D238566
:1087A0006B8D6385204603B0F0BD2046FFF7D3FBF9
:1087B0000024F7E710B5FFF7FEFEBDE810400846BD
:1087C000FFF7C9BB10B504462046FFF77BFE014604
:1087D00018B12046FFF7EEFFF6E710BD10B50446CE
:1087E0000846FFF76FFE0346206010B1FFF784FED6
:1087F00003466360204610BD08B5FFF763FE08BD61
:1088000010B50C46FFF7F8FF024678B12388013314
:108810002380FFF7B7FB6388D18B184463686080BF
:108820000B4463601046FFF767FEEDE710BD0000E4
:1088300006490022C0E90022C0E90212C0E9042270
:10884000C0E90622C0E90822704700BF0189000084
:1088500003680B430360436819434160083000F02C
:108860000BBA4368194201D1FFF7F2BF704700000D
:1088700070B50568044685B3002303602946174890
:1088800012F058FB164829460BF038FE15482946C9
:1088900004F0CAFE144829460AF034FB134829465E
:1088A00018F032FD124829460AF050F811482946BE
:1088B00016F0A2F8104829460BF00CFA0F4829468A
:1088C0001BF08AFE04F11806A64206D0236913B1F4
:1088D0006169284698470834F6E770BDB08D0020DE
:1088E0005CB7002008B6002004B70020E0B50020E7
:1088F000F4B70020CCB60020D4B60020A889002010
:108900000148FFF7B5BF00BF3037002007B5074A61
:10891000138803B9FEE7013B9BB213801BB901909A
:1089200000F03AFC019803B05DF804FB2633002008
:1089300031B16FF00043994208BF012101607047D7
:108940000121FBE737B50E4C23884FF6FF729342A7
:10895000054600D1FEE763B900F004FC04210DEBED
:10896000010000F027FC00B1FEE701990548FFF780
:10897000DFFF238828460133238003B030BD00BFCA
:108980002633002028330020026848F24E33A2FB31
:10899000032313EB520244BF22F000420132026073
:1089A00010467047034B1B8803B9FEE70248FFF7E8
:1089B000EBBF00BF2633002028330020814210B5D2
:1089C000044600D8FEE7FFF7EDFF091BC0B290FB9D
:1089D000F1F301FB13002044C0B210BD814210B579
:1089E000044600D8FEE7FFF7DDFF091B80B290FBCD
:1089F000F1F301FB1300204480B210BD814210B599
:108A0000044600D8FEE7FFF7CDFF091BB0FBF1F3EA
:108A100003FB1100204410BD814238B50C4688BFCD
:108A200084B26100054601310020FFF7E7FF2844CA
:108A3000001B38BD10B540B10023441E98B28142DE
:108A400003D90133E25C002AF8D110BD024610F8C8
:108A5000013B1BB18B42F9D1104670471A46FBE728
:108A6000F0B5066800240625374601363B78303BD2
:108A7000DBB2092B0AD804EB840403EB44039CB259
:108A8000A2424FF00005EFD2062501E007600C700E
:108A90002846F0BDFF22FFF7E3BFA0F14103192BE9
:108AA0009CBF2030C0B2704738B503463AB1012AA6
:108AB00011D01B78002B0CBF0222012209E00139E2
:108AC00011F8014F034610F8015B002CF1D0AC42C5
:108AD000F6D0104638BD0139044611F8015F23462F
:108AE00014F8010B002DE4D0FFF7D7FF024628460B
:108AF000FFF7D3FF8242F0D00022EAE708B5FFF784
:108B0000D3FF831E5842584108BD10B500240160B0
:108B10008480C2800C7010BD38B504461346E588C9
:108B200082880068AA4234BFAD1A002510440A4664
:108B3000294665F09FFA002800DAFEE7A388E2885C
:108B4000184480B2904228BF2368A08022BF9B189F
:108B5000002203F8012C204638BD0EB417B505AA33
:108B6000044652F8041B0192FFF7D6FF204603B0DB
:108B7000BDE8104003B070472DE9F041094F0546AC
:108B80000E4614464FF6FF78013CA4B2444505D08A
:108B9000324639462846FFF7E0FFF5E72846BDE8AC
:108BA000F08100BFF548070070B505460E46002469
:108BB000B44226D2285D030604F1010405D462F014
:108BC000F9FD0028F4D000201CE010F04003FAD09A
:108BD000810612D5C20612D50307F4D40323013B44
:108BE000DBB2FF2BE4D0B442EDD02A5D02F0C0022C
:108BF000802A04F10104F2D0E5E70123EFE7022324
:108C0000EDE7012070BD10B5044663F0CBFF0146CF
:108C10002046BDE81040FFF7C7BF2DE9F0410546EB
:108C20001F4614461AB902700020BDE8F0811046B4
:108C3000FFF700FF814206460BD9012F03D12046E2
:108C4000FFF7E1FF38B1721C2146284663F090FF20
:108C5000EAE70720E9E70620E7E70000036823B911
:108C6000016004484960F7F773BE5A684A6059606A
:108C700001607047083700204368014613B9024875
:108C8000FFF7ECBF704700BF0C37002038B5002558
:108C90000468056054B1606884421CBF4368636027
:108CA0000368456008BF00249847F3E738BD436870
:108CB000496810B59C1A8A1AD20FB2EBD47F08BF4C
:108CC0005B1A4FEAD47008BFD80F10BD70B50568A5
:108CD0000C4625B9BDE870404B68084818478B68BA
:108CE00098476A68831A002B01462368B8BF121A96
:108CF000BDE870400148A8BF00221847083700208F
:108D000038B50C461146A2689442034606D0056861
:108D1000AC4204D10260FFF7D9FFA46038BD2A46F7
:108D20000021002AF9D0944208D011469268F8E751
:108D30008B68002BF1D09B688B60EEE70029F7D1A0
:108D4000002DEAD0AA681A60E7E700000146024A4F
:108D50000248FFF7D5BF00BFC05D070010370020F5
:108D60002DE9F047936805460C461646984732466B
:108D7000814621462846FFF7C3FFD5F800A04FF0F3
:108D80000008574647B14A4639462046FFF78FFF4D
:108D900010B9B846BF68F5E7B8F1000F08D1C4F8BC
:108DA00008A031462C602846BDE8F047FFF78EBF8B
:108DB000D8F80830A360C8F80840BDE8F087000084
:108DC0004160024A01460248FFF7CABFC05D070082
:108DD00010370020002A00DAFEE71144FFF7F0BF49
:108DE00013B504460191FCF7E4FE019A01462046C2
:108DF00002B0BDE81040FFF7EDBF8368984203D092
:108E00004368CB1A002B01DAFFF7DABF704770B561
:108E1000066804460D467EB18B6898477368C01A91
:108E2000002809DB20462A463146FFF769FF3368F0
:108E30003046BDE87040184729462046BDE87040DE
:108E4000FFF744BF10B50446FEF70BF930B104F14B
:108E500008000349BDE81040FFF7D9BF10BD00BFAF
:108E6000C05D07004160024A01460248FFF778BF33
:108E7000B45D070014370020002A00DAFEE7114431
:108E8000FFF7F0BF13B504460191FCF7A3FE019A6A
:108E90000146204602B0BDE81040FFF7EDBF0000DC
:108EA0000146024A0248FFF72BBF00BFB45D07002E
:108EB0001437002010B50446FEF7D3F830B104F1A2
:108EC0000C000349BDE81040FFF7A1BF10BD00BF73
:108ED000B45D070010B50446FCF76BFE002320606C
:108EE00063600146054BA36004F10800206101F1B5
:108EF0008041FFF765FF204610BD00BF418F000095
:108F000010B50446FCF755FED4E90031E2689A42F8
:108F1000A0EB030002D10028A8BF013100221018E5
:108F200041F1000110BD0368C168994202BF436866
:108F30000133436001F180410830FFF741BF000079
:108F40000148FFF7F0BF00BF1C3700200000000001
:108F50002DE9F34116461F4623A3D3E900238B4294
:108F600008BF824204460D4611D219A3D3E900235B
:108F700060F0D4F8184902463046FFF7EEFD20466F
:108F800013A3D3E90023294660F0C8F81446134917
:108F9000B4FBF1F201FB12414EF660244FF47A78F3
:108FA000B1FBF4F3304604FB13140D49B4FBF8F5A0
:108FB0000095FFF7D2FD47B10A4908FB154230463C
:108FC00002B0BDE8F041FFF7C8BD02B0BDE8F081D6
:108FD000005C260500000000CC5D070080EE360036
:108FE000D25D0700E15D0700FF5B26050000000081
:108FF00013B504466846FFF788FD2046FFF780FF5B
:1090000001236A46FFF7A4FF02B010BD704710B5F8
:1090100090B183880B2B11D90468204637F038F8BB
:10902000062037F029F801220146204637F060F883
:10903000003818BF012010BD0720FCE70120FAE727
:1090400008B538B183880B2B06D9006837F024F8AF
:10905000002008BD0720FCE70120FAE713B504460D
:10906000684600F04EFA6CB1A3880B2B0CD9BDF802
:1090700004200099206837F001F9003818BF01205A
:1090800002B010BD0720FBE70120F9E708B548B1A1
:1090900083880B2B08D9006837F04AF9003818BFCD
:1090A000012008BD0720FCE70120FAE708B548B118
:1090B00083880B2B08D9006837F04AF9003818BFAD
:1090C000012008BD0720FCE70120FAE708B520B120
:1090D00000682EF055FF002008BD0720FCE710B502
:1090E000044648B18388EF2B08D900682EF05CFF56
:1090F00000202060A08010BD0720FCE70120FAE7D7
:1091000008B550B18388EF2B09D9006800212EF0F3
:1091100067FF003818BF012008BD0720FCE70120C9
:10912000FAE708B548B18388EF2B08D900682EF01C
:1091300073FF003818BF012008BD0720FCE701209D
:10914000FAE708B548B18388EF2B08D900682EF0FC
:109150006BFF003818BF012008BD0720FCE7012085
:10916000FAE7000007B5094836F010FD084836F068
:1091700051FB0023054A07490548009336F077FB69
:1091800000B1FEE703B05DF804FB00BF74340020BB
:109190002C330020D5FB030008B5044836F0A8FCAA
:1091A000BDE80840024836F049BB00BF74340020D7
:1091B0002C33002008B50A460146034836F0F8FB78
:1091C000BDE8084000F0D0B82C3300202DE9F04F66
:1091D0009DB0222B0F46DDF89890BDF89C400646C6
:1091E0001146984600D9FEE71A4613A863F0C0FC62
:1091F00019F0010500D0FEE74FEA590305931CABB7
:1092000003EB08090DF12C0B002C76D001352B0E49
:1092100009F8243C2B0C09F8233C0DF13C0A2B0ADD
:1092200009F8223C09F8215C08F10403CDF800A0FC
:1092300013AA3946304634F001FA20B100F094F810
:109240001DB0BDE8F08F07AB00935246102339469E
:10925000304634F0F3F90028F0D107A852464FF019
:10926000040C136850F8041BBCF1010C81EA0301E3
:1092700042F8041BF5D101230393039B059A934203
:109280002AD2CDF800B0102307AA3946304634F070
:10929000D5F90028D2D107AB00935A46102339469E
:1092A000304634F0CBF90028C8D1042358460DF1DC
:1092B0001C0E514604930A685EF8043B50F804CB38
:1092C000534083EA0C0341F8043B049B013B0493A5
:1092D000F1D1039B0133CFE7102CA24628BF4FF0FA
:1092E000100A289852460FA963F042FC289BA4EB71
:1092F0000A0453442893A4B286E72046A0E700F16D
:10930000080310B50360102383800446FFF77FFE37
:1093100000B1FEE7204610BD10B50446FFF790FEF1
:1093200000B1FEE7204610BD08B5FFF797FE00B17B
:10933000FEE708BD08B5FFF7A9FE00B1FEE708BDCE
:1093400008B52022FFF7B2FE00B1FEE708BD00001D
:1093500010B503490446034837F0FCFE204610BD13
:10936000055A0200ED59020010F5405F00F0BB8085
:109370006DDC10F5D04F00F0B88038DC10F5D24F1E
:1093800000F0B3802EDC10F5FE4F2ED006DB10F57A
:10939000F04F5AD010F5E24F00F0A980C00F70478F
:1093A00000F140030C2BF9D801A252F823F000BFC2
:1093B0004B9400009D930000EB9300004B94000041
:1093C0004B9400009D9300009D9300009D9300002E
:1093D000EF9400009D930000EF9400009D93000027
:1093E0004B94000010F5D14FD8D10320704710F5F1
:1093F000705F7CD015DC10F57C5F78D002DC10F556
:109400007E5FF1E710F5765F71D005DC10F57A5FCD
:109410006DD010F5785FBFE720F0800313F5745F1F
:10942000BAE710F5665F10D00CDC10F56A5F5ED00D
:1094300005DC10F56E5F5AD010F56C5FACE710F5E7
:10944000685FA9E710F5645FA8D10820704710F5A0
:10945000025FFAD037DC10F51C5FF6D00EDC10F599
:10946000225FC2D005DC10F5265FBED010F5245F68
:1094700092E720F0800313F5205F8DE710F50E5F73
:1094800035D011DC10F5145F31D007DC20F08003FB
:1094900013F5185F2BD010F51A5F7DE710F5125FFA
:1094A00025D010F5105F77E710F5085F1FD004DCBA
:1094B00020F0800313F50C5F6EE710F5065F16D001
:1094C00010F5045F68E710F1330F06DA10F1400F72
:1094D000BFF666AF10F58C5F86E710F11E0FB4D0B3
:1094E00010F11C0FB0E701207047052070470720DE
:1094F000704700BF08B5084691B2FFF75BFE002039
:1095000008BD0A6802608A888280704738B50025E5
:109510000446C0E90155C5601030FFF719FF04F19A
:109520001100FFF70FFA214604F11400FFF7D2FCF7
:10953000214604F12800FFF77BF9214604F1500091
:109540001CF044FB214604F17400FEF783FC214625
:1095500004F5A14004F04AFF04F5A24021467C3006
:1095600019F082FF04F5A440214624301AF042F895
:1095700004F5A540214620301AF02AFE04F5A64045
:109580002146343003F0CEFE04F5A6402146683073
:1095900003F006FF04F5A7402146283003F0CEFF74
:1095A00004F5A7402146303004F078FE04F5A743C7
:1095B00004F5A74083F85650214658300BF080FD43
:1095C00004F5A84021465C300BF071FE04F5A8407C
:1095D0002146603000F058FC04F5AB4021463030A5
:1095E0000CF0F6FE04F5AD402146283011F08CFF5A
:1095F00004F5F140214670300AF0BAF804F5F24063
:109600002146603008F05AFC04F5FB402146043046
:1096100016F004FD04F5FD402146583017F08AFD90
:1096200004F5FD4021467C3018F01EF9214604F572
:10963000FE4003F08FFF04F5FE4021464C3004F05D
:10964000DDFA04F5FF4021462430FEF70BFA04F55D
:10965000FF402146443015F055F804F5FF402146FF
:109660004C300AF0EBFD04F5FF4021467C3009F058
:10967000B3FB214604F5004009F08CFC04F50040E2
:109680002146143009F002F804F50040214630303C
:1096900018F028FF04F50040214654300AF02AFE55
:1096A00004F50040214684301AF024FC04F5004003
:1096B0002146EC3009F0C4F848F23013E554FFF7C6
:1096C00071F948F23413E050204638BD38B5054CE6
:1096D000236823B9044D28461AF0C6F8256020688F
:1096E00038BD00BF40B8002048B80020FDF708BAD8
:1096F00010B548F2301301220446C25460301CF009
:109700009BF904F5AD402830BDE8104010F06EBD67
:1097100010B548F23013054CE35C2BB92046FFF737
:10972000F5FE2046FFF7E4FF004810BD0837002093
:1097300038B548F230130446C25CDAB10025C5548E
:109740002946FDF7D9FF29462046FDF79FFC29460B
:109750002046FDF789FD04F160001CF073F904F563
:10976000A9400C3002F0BAFA04F11100BDE838400B
:10977000FFF7CCB838BD10B5044660301CF064F972
:109780002046BDE81040FDF7BBB973B50C46054651
:109790004822002105F17406204662F005FE30469D
:1097A000FEF7ADFB20803046FEF7A2FB45F27E03BC
:1097B000608005F5AB46EB5AA380303604F1080112
:1097C0003046FFF71DF804F1100106F11000FEF716
:1097D000A6FE05F5A14004F118010C30FFF710F8C2
:1097E00005F5A24004F120014830FEF798FE05F58A
:1097F000AE4004F128011830FEF791FE05F5A440B3
:1098000004F1300124300191FEF789FE05F5A440F2
:109810000199483002B0BDE87040FEF780BE45F2C5
:109820007C03C25A45F27E03C2527047807F00F02B
:109830000F00012804D0063801288CBF0020012029
:10984000704700000022C0E90022826002460449FD
:1098500042F80C1F4261028B02F0800202837047C3
:10986000119B0000054A064845F24273D35C054A45
:1098700003F00F03072B18BF10467047083700206E
:109880002C8E0020E88D002010B504460C30FFF728
:109890005DFAE37A6FF38703E372238B03F08003AF
:1098A000238310BD38B50C46FFF7DCFF0546FFF7F4
:1098B000BDFFB0B145F292430B4AD25A4FF6FE7348
:1098C0009A4202D0094B9D4207D12B6823606B68F6
:1098D000636002232372002038BDAB8B23800123F9
:1098E000F8E70B20F8E700BF083700202C8E002097
:1098F000084A45F2C463D058074B834228BF034649
:109900004FF47A705843B0F57A6F88BFA0F57A604B
:10991000704700BF083700209BC4200038B543695A
:1099200000F10C059D4204460ED0FFF7E1FF63688D
:10993000834209D1FCF73DF9626820600146284660
:10994000BDE83840FFF746BA38BD08B50146FFF715
:10995000CFFF8B6833F07C4204D0C3F319039842E5
:1099600028BF184608BD08B50146FFF7C1FF0B7EAA
:109970009A0702D5642828BF64205B0704D5B0F598
:109980007A7F28BF4FF47A704B7E13F0F00F02D02D
:10999000BC2828BFBC208B6833F07C4204D0C3F3C2
:1099A0001903984228BF1846002808BF0A2008BD9E
:1099B000012938B54568044602D1FFF7D4FF60603D
:1099C000FCF7F7F86369014604F10C0098420DD0EA
:1099D0006268AA420DD0246813195B1A0A2B4CBF87
:1099E0000A222146BDE83840FFF7F4B962682160D9
:1099F000F8E738BD027E10B4D4070ED4084C45F207
:109A0000AA61615C090700D5FEE742F001025DF83A
:109A1000044B02760121FFF7CBBF5DF8044B704782
:109A20000837002038B5037EDA0705461CD5114AF1
:109A300045F26043D35C5B0716D4FFF713FFFFF7D3
:109A4000F5FE88B105F10C00FFF780F90A4800F037
:109A5000C8FB044618B10D2806D0012100E00146DC
:109A60002846FFF7A5FF03E02846FFF70DFF0D246A
:109A7000204638BD08370020688B0020017ECA07C9
:109A80000FD5C1F3C302013202F00F0262F3C60127
:109A9000042A017601D8FFF7C5BF027E6FF3C60224
:109AA00002767047037E13F0010F08D06FF3C603F0
:109AB00003760B681B78DB0601D5FFF7B3BF704751
:109AC000F0B4047EE6071ED5104E45F2FE67F75D42
:109AD0003F0718D006F5AE463688022E13D909681E
:109AE000097809070FD573B96AB1214663F3C60136
:109AF000136801761B78DB0602D5F0BCFFF792BF36
:109B0000F0BCFFF70BBFF0BC704700BF0837002068
:109B10000148FFF787BF00BF908D0020037EDB0761
:109B200002D50121FFF744BF7047037E10B4C3F391
:109B300040048C4209D061F341030376DB0704D56E
:109B40005DF8044B0121FFF733BF5DF8044B70470C
:109B5000C37A13F0FC010DD0FC290BD0FC33C37287
:109B600013F0FC0306D1417E63F307114176012116
:109B7000FFF71EBF704708B531B1092915D96FF03D
:109B80007C43994228BF19468368C3F319028A426D
:109B900001D1002008BD61F319038360037EDB0758
:109BA000F7D50121FFF704FFF3E70720F2E70000F4
:109BB000F0B5067E87B0002316F0010604460F4676
:109BC00015468DF8143019D08B885BB103A938463F
:109BD00001F015FB01230093244803AB2A463946C4
:109BE0000CF0ACFD2046FFF73DFE837F180707D140
:109BF0002046FFF749FE1E4810F046F807B0F0BDBA
:109C000005F0FB030B2B1DD0637E05BB13F0F00F9B
:109C10000ED10026237E590725D5238B23F47063AC
:109C200023F00403238301212046FFF7C1FEE5E76B
:109C3000F03313F0F00F6376EBD1E37A65F387032B
:109C4000E372E7E7237E43F004032376EBE75A1C35
:109C500002F00F0262F30303032A6376DDD8237E4A
:109C60005A07CBD4EFE7002EC8D0DCE7B88C002031
:109C7000B08D0020C37A427E10B403F0FC04FC2CAB
:109C80001CBF0433C372002908BF08210F2928BF55
:109C90000F211309C9B2994238BF1946134661F31F
:109CA00007134376037EDB0707D512F0F00F04D1CC
:109CB0005DF8044B0121FFF77BBE5DF8044B704754
:109CC000F0B58DB005AE00240F460DF126010594C8
:109CD0008DF824408DF82E40B48007ADFFF7E2FDEB
:109CE00050BB9DF82E20164B3C68022A0BBF15492D
:109CF00045F29242D1E900019A5A16BFADF81C20F4
:109D0000C5E9000101228DF8242045F26842304661
:109D1000995A01F021FF08230022CDE902320523E0
:109D2000CDE90063084821462B4603220DF024FAB2
:109D30000421204601F069FD20460DB0F0BD00BFB2
:109D4000083700209C8B0020B88C0020037A012B60
:109D500006D100884FF6FF73C31A58425841704726
:109D600000207047037861F3000300F82C3B09B131
:109D700001F09EBF01F0B2BFF0B5154687B00C46AA
:109D80003C22002128468DF8141062F00DFB6CB3C4
:109D900023681B785B0703D00626304607B0F0BD6A
:109DA00003AF3946204601F0B9FA06460028F4D13F
:109DB0009DF81430022BEFD197E8030085E80300EB
:109DC00005F132012046019101F077FA019910B1B5
:109DD000204601F0FAF9A37985F8363094F9153068
:109DE00085F83730A37D85F83830D6E70726D4E7E5
:109DF0000378DB0704D500F1100114301CF022BCFD
:109E00000B20704710B5026A90B004460B461AB199
:109E100021B9416A1846904710B010BD01AAFFF75A
:109E2000ABFF0028F8D1D4E9083101A89847F3E73F
:109E3000036A07B54BB17F2907D0027C8DF8051066
:109E40008DF80420416A01A8984703B05DF804FB2F
:109E500003898B4210B5044606D1BDE8104009487D
:109E60004FF40041FEF7FDBC018106484FF400416C
:109E7000FEF7EEFC218904F12C00BDE8104001F052
:109E8000E9BE00BF30370020F0B5036885B003F0AD
:109E9000C003036004460191FEF784FD2071FEF7C4
:109EA00081FD00252B4B6071A360A5712A4807F046
:109EB0001DFD0B2323740F2323834FF0FF33C4E9CD
:109EC00007350199E06065826561656204F12800EB
:109ED00001F0EBFD214B224AC4E92735234604F566
:109EE000A07743F8A42F2946C4F8AC301022C4F858
:109EF0003851A4F83E51384662F056FA02A801F0F3
:109F000004FE88222946A4F83C5104F1B00062F016
:109F10004BFA2378264643F0010306F82C3B3046E3
:109F200001F0C6FE0F480AF0D1FF21892046FFF755
:109F30008FFF02A9304601F099FE618E304601F094
:109F40008FFE384608492A4601F014FE204605B027
:109F5000F0BD00BFFFFF0B0B08370020D1AD0000A4
:109F6000C5AD0000E08A0020EF5D070038B503783A
:109F7000590758BFC3F3C004C3F38002437858BFE6
:109F800084F00104054654BFE4B200249BB932B109
:109F90004388DB0503D5C169A430FEF711FF05F145
:109FA0002C001CB1BDE8384001F0F6BFE97ABDE8ED
:109FB000384001F0A7BE38BD1F2908B50CD8C268CB
:109FC000CA40D20708D50278C17242F0200202705E
:109FD000FFF7CCFF002008BD0720FCE702789106C0
:109FE00006D56FF345120270827AC272FFF7BEBFC8
:109FF000704710B50378C3F380028A4204462CD020
:10A0000061F38203037059B92178C1F3C00104F1EF
:10A010002C0001F03FFE2046BDE81040FFF7A6BF30
:10A0200043885A0606D5A430FEF790FE638823F0D5
:10A03000400363806378062B09D104F1A400FEF786
:10A0400085FE0023637004F19C00FEF715FE237863
:10A05000C3F380015B07D7D5D9E710BD1F2938B5F9
:10A0600004461FD8C368CB40DA071BD5837A8B42DE
:10A0700006D10D484FF48041FEF7F3FB002038BDB8
:10A08000817209484FF48041FEF7E2FB23780020FB
:10A090009B06A4F83C01F2D4A37AE3722046FFF7B2
:10A0A00065FFEBE70720EAE73037002043788B4273
:10A0B0001DBF438823FA01F101F001000120704720
:10A0C00029B1012303FA01F1438819434180437800
:10A0D00013B99C30FEF7D0BD70474382FF23037451
:10A0E000C368002A08BF1A4610B41A405DF8044B32
:10A0F0004261FFF7E5BFF8B51F460378DB07054669
:10A100000E4619D50121FFF7D1FFB8B90221284623
:10A11000FFF7CCFF044688B9069B6B62002A18BF84
:10A12000134628462F6208BF4FF49673324601212A
:10A13000FFF7D3FF2046F8BD0D20FCE70520FAE726
:10A14000F8B51F460378DB0705460E4614D50121F6
:10A15000FFF7ACFF90B902212846FFF7A7FF04469E
:10A1600060B9069B6B62284613462F623246022175
:10A17000FFF7B3FF2046F8BD0D20FCE70520FAE706
:10A1800008B50378DB07024609D50421FFF78EFFE7
:10A1900028B9BDE8084004211046FFF791BF08BD6B
:10A1A00008B50378DB07024609D50721FFF77EFFD4
:10A1B00028B9BDE8084007211046FFF781BF08BD58
:10A1C00038B50378DB0704460D4609D5FBF7F1FCEB
:10A1D0002844E06108212046BDE83840FFF770BF01
:10A1E00038BD38B50578EB07024611D50521FFF7D4
:10A1F0005DFF58B95388C3F3001383F0010363F381
:10A200004105157005211046FFF75AFF002000E0B8
:10A210000D2038BD70B58CB0D0F8985005AE002434
:10A220004FF6FF7101233046ADF826108DF82E3021
:10A230008DF824400594ADF8184001F089FC07AB77
:10A2400022462846CDE901440096032101F0C0F8DA
:10A250000721284601F0D9FA28460CB070BD70B528
:10A260000146D0F89850034651F8340F8CB0496835
:10A2700005AE07AA002403C219898DF82E400222D8
:10A2800030468DF824200594ADF8184001F05CFCB0
:10A2900007AB224621462846CDE9014400968DF8B9
:10A2A0002E4001F095F8284601F0C2FA4FF0FF3336
:10A2B00003700F2343708470C47028460CB070BDC7
:10A2C000F7B50B681B781A0705460C4620D50DF12B
:10A2D0000301204601F07CF99DF80330082B17D0CC
:10A2E000102B17D073BB184BA360E37EDB0705F17F
:10A2F000340509D4154F45F250462046B95901F0AE
:10A3000087F9BB590133BB512946204601F001FBB7
:10A3100003B0F0BDD5F838114FF0FF330131019390
:10A3200005F5A073A3602046C5F8381101F070F957
:10A3300001A9204601F085F9FF21204601F0AEF980
:10A34000034DE1E7FEE700BF488B002008370020FF
:10A35000E75D070021B9D0F8E8300133C0F8E830F4
:10A36000837A93420DD1B0F83E31B3F5007F3CBF04
:10A370000133A0F83E31B0F83E2100F59E700AF09E
:10A38000DBBE70472DE9FF410B689DF828801F78E0
:10A390008B8800260446154608468DF80C60E3B10C
:10A3A00001A900F02CFF2B48012201A907F020078A
:10A3B00014F05AFE40B13FB195B10E2D05D1314692
:10A3C000802226300AF0B8FE65B1B8F1000F09D03E
:10A3D000D4F8DC300133C4F8DC3004B0BDE8F081DF
:10A3E0000121EDE7D4F8B0300B2D03F10103C4F8DF
:10A3F000B0301AD1D4F8EC300133C4F8EC30E7B106
:10A40000D4F8BC300133C4F8BC3025B9D4F8C0301E
:10A410000133C4F8C03001A8FFF798FC98B1D4F814
:10A42000B8300133C4F8B830D7E70F2D02BFD4F8E5
:10A43000F0300133C4F8F030E1E7D4F8C430013330
:10A44000C4F8C430E7E7D4F8B4300133C4F8B4300A
:10A45000C3E700BF1C8E00202DE9F74398460B6828
:10A460001B781B0705460E46174604D400252846D0
:10A4700003B0BDE8F0830DF10101304601F098F81A
:10A480009DF80130052B01D00825F0E701A93046E1
:10A4900001F0AEF80DF10201304601F099F89DF897
:10A4A0000240082C3AD0102C00F08380002CEBD115
:10A4B000434839460246304601F08DFA05460028E9
:10A4C000E2D19DF80230082BD0D198F81E3003F06D
:10A4D0000F03072BCAD1D8F818309C4208D0C8F80F
:10A4E00010000146C8F8184008F10C0001F03CFBD0
:10A4F000019BD8F814200133934288BFC8F8143068
:10A50000C8F80C302F4A45F2E833D3589C42ADD9F5
:10A510002D48002221460AF01BFDA8E7B8F1000FE4
:10A52000B2D00DF10301304601F0A2F89DF80330DE
:10A530002449013BDBB245F2E8328DF803308C58F8
:10A5400004F07F02934219D1314605F1280001F051
:10A55000B9FA98F81E3003F00F03072B0CD1D8F886
:10A5600018309C4290D307D1019AD8F80C30511C76
:10A57000994223D09A4287D339469BE704F1FF39A9
:10A5800009F07F02934207D14A46314605F128007F
:10A5900001F09CFA4C46DCE7013404F07F02934260
:10A5A0007FF472AF2246314605F1280001F08EFAA1
:10A5B000CFE7064905F5A07000247BE71D2556E787
:10A5C000488B002008370020E08A0020E75D070064
:10A5D00070B588B000238DF810308DF81C301368EA
:10A5E0001B781B0706460C46154602D4002008B00F
:10A5F00070BD104600F08AFD00F44050B0F5005FD9
:10A6000001D00820F3E7284601F0C1F80028F8D16E
:10A610006946284600F0CCFF9DF80030052BF0D1AC
:10A620000DF10301284600F0D3FF9DF80330082BFD
:10A63000E7D10DF10101204601F01AF80DF10201F8
:10A64000284601F015F89DF801209DF802309A4245
:10A65000D7D101A9284600F0CBFF02A9284600F077
:10A660005DFE9DF81030002B3AD0012202A92C4843
:10A6700014F0FAFC04469DF81030022B4CD0002C4C
:10A68000BFD02068616802AB03C302238DF810308D
:10A690009DF802302349013BDBB245F2E8328DF8E8
:10A6A00002308A5802F07F018B4224D106F1640205
:10A6B000A37F03F00F03072B03D16369019999422C
:10A6C0009FD302A9284601F086F900288FD1A37FE5
:10A6D00003F00F03072B89D1019B0133636186E7E8
:10A6E000204605A900F08BFD9DF81C40002CC2D02F
:10A6F000012205A9BBE7511E01F07F018B4202D167
:10A7000006F15402D4E7013202F07F0293427FF453
:10A7100078AF06F17402CBE7002CB9D171E700BF26
:10A720001C8E00200837002038B50C4691F82450C4
:10A7300092F9151004F122000AF0A1FD0A4845F231
:10A74000A963C35C022B0ED1084B9C420BD145F28E
:10A750000473C35CAB4206D0BDE838404FF0004103
:10A760002830FEF775B838BD08370020E88D002086
:10A7700037B50D4604460DF10701284601F01AF8D9
:10A780009DF80730042B15D0072B1ED1D4F80C31BF
:10A790000133C4F80C31237813F0010013D0C3F354
:10A7A0000015DB0604D520460321FFF789FC284667
:10A7B00003B030BDD4F8043107480133C4F8043184
:10A7C00029461BF0D3FF0120F2E7D4F81031013302
:10A7D000C4F810310020EBE7788D002010B5037825
:10A7E000044661F3C30303700948FBF74DFC23786B
:10A7F0005A0704F12C00C3F3800158BFC3F3C00112
:10A8000001F048FA2046BDE81040FFF7AFBB00BF9B
:10A810000837002070B50546C6680A48FBF78AFF6E
:10A82000044650B9074807F061F8B042E8604FF4B9
:10A830008001054803D1FEF714F8204670BDFEF7ED
:10A8400007F8FAE708370020303700200148FBF707
:10A8500065BF00BF0837002007B52C30019101F01B
:10A86000C7FA019903B05DF804EB0AF0C4BC00001C
:10A8700070B508460D46144600F048FC00F4405000
:10A88000B0F5005F2BD12B681B781B0727D51A2149
:10A89000284601F01CF8064608B321461048052258
:10A8A00008F06AFC0446D0B1B3889AB2092A16D9D6
:10A8B000A0F848307388A0F84A3090F8403043F050
:10A8C000800380F84030FBF774F9D5E90223E06497
:10A8D000C4E914230348BDE8704008F063BE70BDAE
:10A8E000D08F0020808D00202DE9F0431D460B689D
:10A8F00093F800808B8885B004460E46174608F012
:10A900002008002B38D04FF0000901A930468DF8FF
:10A910000C9000F074FC01A8FFF718FA68B1A37955
:10A920000133DBB2A37133B904F12C0001F0C5FB94
:10A93000002838D0FEE784F80690B8F1000F1BD04D
:10A94000D7B14D48012201A914F08EFB81469DB973
:10A950003A4631462046FFF73BFE0546B0B9B9F10D
:10A96000000F09D03A4649462046FFF7DDFE01AA0E
:10A9700039462046FFF77CFF6378013B072B07D859
:10A98000DFE803F0070614411F06675A0E25F3E7B8
:10A99000FEE7D4F8D430618A0133C4F8D43004F12E
:10A9A000A400FEF71DFA05B0BDE8F083D4F8D0305E
:10A9B0000133C4F8D03000236370204600F00AF958
:10A9C000F1E7B38813B1B8F1000F0DD06DB1D4F831
:10A9D000CC302A480133C4F8CC30002363702A46B7
:10A9E0003146FFF7E5F8E8E7FEE7002FEFD02378E0
:10A9F000DA07ECD53B681B78DB06E8D50621204654
:10AA0000FFF75EFBE3E7D4F8C8300133C4F8C83081
:10AA100025B1D4F8E0300133C4F8E030002363708E
:10AA20002A46314616480BF06DFF14482B463A462D
:10AA30003146FFF745F8C0E7D4F8C8301148013374
:10AA4000C4F8C830002363702A46314608F082FEFD
:10AA5000B3E7D4F8C8300133C4F8C83025B1D4F80E
:10AA6000E4300133C4F8E4300023074863702A4619
:10AA700031461BF09BFFA0E71C8E0020908D00202C
:10AA8000B88C0020808D0020788D0020D0F8983080
:10AA900010B5DA7E0021C3E9041122F0170242F05A
:10AAA00004029980DA760278D10704467FD542788D
:10AAB000013A00F19801072A05D8DFE802F0050401
:10AAC0002A4D38045C6FFEE704F12C004FF6FF714D
:10AAD00001F0C0F82046FFF79DFB002867D0237CDB
:10AAE00083718376036800229A7004230376237EA1
:10AAF0004376C37EDB0603D401462046FFF7E0FB26
:10AB00000023A37104F12C0001F0D7FA002858D0DB
:10AB1000FEE72046FFF7A3FB002848D0E37A8371C5
:10AB2000837623795A1C227102689370DDE7E27AFA
:10AB30009A719A76D4F89830224804221A76D4F87A
:10AB40009830227E5A76FFF7BBF880B363795A1C9F
:10AB5000627102689370CCE7E27A9A719A76D4F8BF
:10AB60009830194804221A76D4F89830227E5A7602
:10AB70000CF0CAFCE9E7E27A9A719A76D4F8983038
:10AB8000124804221A76D4F89830627E5A761BF066
:10AB900037FE60B1C37E9A07ABD4D7E700221A769E
:10ABA000D4F898300A485A7608F010FDF1E7D4F846
:10ABB0009810002220468A80BDE810400B23FFF742
:10ABC00093BE10BD908D0020B88C0020788D0020A1
:10ABD000808D002038B543780446002B79D1037866
:10ABE00013F0010305D14380BDE83840A430FEF7DF
:10ABF000ADB843885A061AD5062363706278002AD6
:10AC000048D0012303FA02F2638804F1A40523EA81
:10AC1000020363802846FEF799F86378082B58D81A
:10AC2000DFE803F0383D424747474C474700DD0522
:10AC300007D5FAF7BEFFE369C01A002801DB082335
:10AC4000DBE76388980701D50123D6E7590701D5CB
:10AC50000223D2E71A0701D50323CEE71D0601D54B
:10AC60000723CAE79806C3F34011C3F300120CD5BB
:10AC700072B123789B070BD4042363700029BDD0E5
:10AC8000237843F002032370B8E7002AB6D0F3E735
:10AC90000523B2E72046BDE83840FFF767B92046F4
:10ACA000BDE8384000F016B82046BDE8384000F056
:10ACB0002AB82046BDE83840FFF7E8BEE17A04F143
:10ACC0002C0001F01FF828466421BDE83840FEF74B
:10ACD00087B838BD10B50446FFF78AF820B920467A
:10ACE000BDE81040FFF7D2BE218904F12C0000F02E
:10ACF000B1FF002120466170FFF784F82046BDE8CF
:10AD00001040FFF767BF38B50446FFF771F840B150
:10AD1000236A0020607043BB2046BDE83840FFF73F
:10AD200059BF638A04F12C0583B9217C284600F0C1
:10AD3000E9FF284601F056F801462046FFF778F86B
:10AD40002046FFF755F80028EFD0E1E723785B07AE
:10AD500003D4217C284600F0D5FF628A217C284656
:10AD600001F098F80028D3D138BD616A9847D3E73D
:10AD700010B50446FFF75CF82046BDE81040FFF729
:10AD8000C2BF00004378012B10B5044603D0062B48
:10AD900005D073B1FEE7BDE81040FFF79BBF00236D
:10ADA00043700748FEF76AFE2046BDE81040FFF7F3
:10ADB00011BF03785A0702D54388DB05F5D410BDCF
:10ADC000908D00200148FFF7DDBF00BF688B002099
:10ADD0000148FFF7FFBE00BF688B0020F0B589B0C7
:10ADE00000238DF810308DF81C30D0F8F43001338A
:10ADF00004460E46C0F8F4301746002A40F0AE80F4
:10AE0000002900F059810378DD0740F16D81084683
:10AE100000F0BDFC0746002840F0A08002A93046A3
:10AE200000F07CFA05A9304600F0E9F99DF81050D1
:10AE30002DB1B248012202A914F016F905469DF879
:10AE40001C30012B00F09C80022B00F0BE800DF125
:10AE50000601304600F0B9F948B9BDF806304FF6A2
:10AE6000FF72934203D022899A4240F0B7809DF846
:10AE70001030012B00F0B880022B00F0BE8005A836
:10AE8000FEF764FF002800F0C880D4F8FC300133DE
:10AE9000C4F8FC302B4602AA31462046FFF7DCFA04
:10AEA000074628B11D2859D16378062B40F016813A
:10AEB0003146204602AAFFF7DBFC91483146FEF7F7
:10AEC000F1FD95B3294632462046FFF72DFC336845
:10AED0001B78190729D50DF10501304600F078FBE4
:10AEE0009DF80530082B20D1AB7F03F00F03062B14
:10AEF00004D0072B08D0012B40F0E480304600F04E
:10AF00006DFC002800F0F08033681B7803F0070325
:10AF1000012B0AD1AB7FDA0907D11A0705D02B8C98
:10AF2000022B02D9FAF745FEA8606378022B7AD08B
:10AF3000062B00F08280012B40F08D8033681B7857
:10AF40005B0770D1D4F808310133C4F808313146B9
:10AF50002046FEF757FF002F00F09A80A7F1080067
:10AF6000152800F2C180DFE800F09BBFBFBFBFBF64
:10AF7000BFBFBFA1A7AD52B339BFBFBFBFBFBFB92E
:10AF80002378580705D505A8FEF7E0FE002840F015
:10AF9000B180628EBDF814309A421FD1002D7FF42B
:10AFA00056AF05A8FEF7D2FE00283FF450AF554A31
:10AFB00045F2AA63D55C15F002053FF448AF4F484F
:10AFC00002A914F0B7F8054641E7082204F134015C
:10AFD00005A863F05DF800283FF439AFD4F81831C4
:10AFE0000133C4F8183153E0002D6BD0286869682C
:10AFF00002AB03C302238DF81030082204F13401A0
:10B000000DEB020063F044F800287FF438AFD4F869
:10B0100028310133C4F828313AE0D4F8F83001334C
:10B02000C4F8F83036E7227CA37A9A4213D0D4F8D9
:10B0300010310133C4F810318DE79DF81C3043B155
:10B0400004F1A400FDF782FE002363702046FFF7A1
:10B05000C1FD002F82D133681B7803F00703012B59
:10B0600018D0032B0ED0002BE1D1D4F808310133D6
:10B07000C4F80831244831460CF002F82046FEF7A7
:10B0800075FF68E731462046FFF772FB0028F1D0D4
:10B0900009B0F0BDD4F800310133C4F80031E9E75C
:10B0A000D4F82C310133C4F82C31F1E7D4F8303125
:10B0B0000133C4F83031EBE7D4F820310133C4F860
:10B0C0002031E5E7D4F824310133C4F82431DFE737
:10B0D000D4F814310133C4F81431D9E7D4F81C3151
:10B0E0000133C4F81C31D3E7D4F834310133C4F848
:10B0F0003431CDE7002D7FF4AAAE58E71C8E002036
:10B10000908D002008370020B88C00200368587804
:10B110001B7843EA0020704708B5FFF7F7FF00F4FB
:10B120004050A0F500535842584108BD02681378BA
:10B1300019B143F020031370704723F02003FAE79E
:10B140000268137819B143F010031370704723F0AD
:10B150001003FAE700F44053B3F5005F1ED120F46A
:10B160004E5323F03F0348F2400293421CD00CD8C8
:10B17000B3F5446F18D005D8B3B1B3F5046018BF68
:10B1800001207047B3F50040F9E74CF64042934286
:10B190000AD000F44C40B0F54040F0E710F4406FA6
:10B1A00014BF0120002070470020704708B5FFF74A
:10B1B000ADFFBDE80840FFF7CDBF08B5FFF7F6FFCC
:10B1C000002814BF0320FF2008BD38B50C460546F3
:10B1D000FFF7F3FFFF281BBF2A68131806205978D2
:10B1E0001FBF135C43EA01232380002038BD08B54C
:10B1F000FFF7DCFF002814BF0520032008BD38B589
:10B200000C460546FFF7F3FFFF28014620D02846ED
:10B21000FFF77CFF00F44060B0F5006F05D0B0F59B
:10B22000406F0DD00020207209E02A68531858782A
:10B23000535C43EA0023238001232372002038BD9E
:10B240002B6801221944204600F06BFC0223F4E72E
:10B250000620F4E7034610F4404018BF83F0400096
:10B2600003F4405218BFC0F38010B2F5005F05D15F
:10B2700003F44C43B3F54C4F08BF0020704708B5AA
:10B28000FFF744FF0146FFF7E5FFA0B10846FFF7CF
:10B2900061FF002801F440610CBF03200520B1F5D7
:10B2A000006F03D0B1F5406F03D008BD0230C0B2CB
:10B2B000FBE70830FBE7FF20F7E738B50C4605460B
:10B2C000FFF7DDFFFF281BBF2A68131806205978F7
:10B2D0001FBF135C43EA01232380002038BD10B553
:10B2E000FFF714FF0446FFF735FF04F4406300281E
:10B2F0000CBF03210521B3F5006F0AD0B3F5406FF1
:10B300000AD02046FFF7A6FF08B10231C9B20846AD
:10B3100010BD0231C9B2F4E70831FBE738B5054684
:10B320000C46FFF7DCFF01462846FFF7EFFEFF293A
:10B3300008D000F44040B0F5004F05D0B0F5404FC4
:10B340000DD0A0B1062009E02A6853185878535C44
:10B3500043EA0023238001232372002038BD2B6899
:10B3600001221944204600F0DCFB0223F4E720729E
:10B37000F4E7102804D0182814BF002008207047D4
:10B380000420704700F00700013806280BD8DFE8DA
:10B3900000F00406080A040608000420704708208C
:10B3A000704710207047002070470000430708D006
:10B3B00000F01803083BDBB2102B04D8034AD05C22
:10B3C0007047FF2070470520704700BFFF5D0700F2
:10B3D0002DE9F7431F461B7ADDF828909DF82C6075
:10B3E000012B0546884641EA020424D0022B25D0D1
:10B3F000B97C012925D002292ED0B8F1020F04BF53
:10B4000024F02004A4B2002E14BF0820002004431E
:10B41000B2F5805FA4B203D0B2F5005F20D03ABB92
:10B4200033B329B3B9F80020B9F802309A421FD1DA
:10B4300044F040041CE044F40044D9E744F44044A0
:10B44000D6E778894FF6FF7C604514BF20200020A6
:10B45000044344F40064D0E744F44264A4B2CCE76B
:10B46000002956D199F80520002B4BD1002ADFD1B5
:10B470007F22296868461AF0FAF9214668461AF0D0
:10B4800025FA002168461AF00AFA2046FFF762FE04
:10B4900020B1B9F8021068461AF018FA07F10A014B
:10B4A00068461AF01EFA2046FFF7D4FE20B1B9F81C
:10B4B000001068461AF00AFA394668461AF011FA7E
:10B4C000BDF80430AB808EB19DF830100E4331468C
:10B4D00068461AF0E4F93046FFF768FF0246304646
:10B4E000FFF750FF1044AA881044A880B8F1030F5A
:10B4F00002BFAB880133AB80AB880233AB8003B0B3
:10B50000BDE8F083002AB3D199F80430002BAFD105
:10B510008EE713B999F80530F8E7022B82D102299A
:10B5200080D1F7E710B50446FFF714FE04F440633A
:10B5300000280CBF03210521B3F5006F06D0B3F539
:10B54000406F17D023B1FF21084610BD0231C9B2A8
:10B550002046FFF77FFE08B10231C9B204F440442F
:10B56000B4F5004F08D0B4F5404F08D0002C18BFF8
:10B57000FF21E9E70831EAE70231C9B2E4E708311F
:10B58000FBE708B58388042B05D9FFF7BFFDBDE8AD
:10B590000840FFF7C7BFFF2008BD8288022A05D9EF
:10B5A00003681B781B0701D5FFF7EBBFFF2070472F
:10B5B00038B505460C46FFF7F0FFFF281FBF2B6884
:10B5C0001B5C03F00703237014BF0020062038BD66
:10B5D00038B505460C46FFF7E0FFFF281FBF2B6874
:10B5E0001B5C03F01803237014BF0020062038BD35
:10B5F00038B505460C46FFF7D0FFFF281FBF431C98
:10B600002A68DBB200201ABFD3582360062038BD59
:10B6100038B505460C46FFF7C0FFFF2800D1FEE70E
:10B620002A68431CD9B252FA83F35454220A5A703E
:10B63000220C240E9A70DC70EB7E43F00103EB7653
:10B6400038BD38B505460C46FFF7A7FFFF2803466F
:10B6500000D1FEE72D68285C00F01800FFF789FE96
:10B66000053302462146E818BDE8384061F080BA4B
:10B6700038B505460C46FFF790FFFF2802460BD071
:10B680002B68185C00F01800FFF773FE13440344A6
:10B6900000205B79237038BD0620FCE738B50546ED
:10B6A0000C46FFF77AFFFF28024600D1FEE72B6821
:10B6B000185C00F01800FFF75CFE134403445C7153
:10B6C00038BD10B50446FFF768FFFF2806D0236891
:10B6D000185CFFF757FE0230C0B210BD0220FCE735
:10B6E00010B50446FFF74DFFFF28014610D0236830
:10B6F0001A7812070CD5A488A0420BDA185CFFF761
:10B7000055FEFF2808D00844C1B28C42B8BFFF21C3
:10B71000084610BDFF21FBE70146F9E7F8B50546ED
:10B72000FFF7DEFF84B2FF2C2DD02846FFF7EEFC9A
:10B73000830506461DD52846FFF7C3FF2F68A98855
:10B74000A21C93B210FA82F28A4207EB040C1CDCB2
:10B750003A5D02F07F0213449CB210FA83F39942DF
:10B7600013DBBCF80020C2F3C7127F2A01D0994234
:10B77000E6D12846FFF7D0FC28B906F00706032ECD
:10B7800001D10134A4B2E0B2F8BDFF24FBE738B523
:10B790000546FFF7C3FFFF28044609D02846FFF7F8
:10B7A00090FF0444A8888442CCBF0620002038BD06
:10B7B0000620FCE7F8B505460E46FFF7AFFFFF2869
:10B7C000044609D028462F68FFF7A6FC00B9013CC3
:10B7D0003B5D33700020F8BD0620FCE707B5036829
:10B7E0001B7803F00703032B03D0002003B05DF8A0
:10B7F00004FB0DF10701FFF7DDFF0028F5D19DF8EF
:10B800000700031F58425841F0E7F8B505460E46B9
:10B81000FFF784FFFF28044608D028462F68FFF76B
:10B820007BFC00B9013C3E550020F8BD0620FCE73A
:10B8300010B50446FFF772FFFF2816BF23680020EB
:10B84000C01810BD10B50446FFF7F2FF2368C01AF8
:10B85000C0B210BD38B50546FFF7F4FF04462846D0
:10B86000FFF72FFF2044C0F17F0080B238BD38B50C
:10B870000546FFF7E7FF04462846FFF722FF04448A
:10B88000A888001B80B238BD70B506460C46FFF78D
:10B89000D9FF05463046FFF714FF05442C44B48019
:10B8A00070BD10B50446FFF70CFFA388181A236873
:10B8B000184410BD08B50246FFF728FC830504D5DF
:10B8C000BDE808401046FFF70BBFFF2008BD70B56C
:10B8D00006460D46FFF7EEFF04463046FFF71EFF13
:10B8E000FF2C024613D0FF2811D0ADB294420ED8DF
:10B8F0003368195BC1F3C7118D4203EB040007D015
:10B900001B5D03F07F0302331C44E4B2EEE700202A
:10B9100070BDF0B50446E5B000230AA805930D46B6
:10B920001AF046FE23681B781B074FD50DF1130153
:10B930002046FFF73DFE002848D105A92046FFF725
:10B9400057FE0646002841D106AF9DF81320059901
:10B950003B4628461AF01EFEA1680AA81AF058FCB9
:10B960002046FFF7AEFE05462046FFF76BFF03902B
:10B970002046FFF77CFF023D0D2302460399CDE9E7
:10B9800000730AA8EBB21AF04FFC2046FFF75AFFEB
:10B99000216802460AA81AF0EBFC2046FFF748FF90
:10B9A00003902046FFF763FF039A00960346114673
:10B9B0000AA81AF021FD2046FFF773FF01460AA8E6
:10B9C0001AF0CBFDE37E43F01003E3760AA81AF0E9
:10B9D00009FE65B0F0BDF0B50446E9B000230EA83D
:10B9E00005930E4615461AF0E3FD23681B781B07E6
:10B9F00006D400240EA81AF0F5FD204669B0F0BD6B
:10BA00000DF113012046FFF7D3FD00284BD105A906
:10BA10002046FFF7EDFD002845D106AF9DF8132025
:10BA200005993B4630461AF0B5FD29460EA81AF096
:10BA3000EFFB2046FFF745FE0238C5B22046FFF770
:10BA400001FF03902046FFF712FF0D2302460399E2
:10BA5000CDE900730EA82B461AF0E6FB2046FFF74F
:10BA6000F1FE216802460EA81AF082FC2046FFF77C
:10BA7000DFFE03902046FFF7FAFE039A01210346FA
:10BA800000910EA811461AF0B7FC0AA90EA81AF0E8
:10BA900064FD2046FFF705FF2A4601460AA862F02A
:10BAA000F7FA0028A5D00824A4E738B504460430E6
:10BAB0000D4600F09BF845F2A4432046EB5823675F
:10BAC00038BD000000487047CC8B0020074945F284
:10BAD000E833CB58591E914203D00133934202D030
:10BAE000FEE7034870470348704700BF083700204F
:10BAF000BC8B0020DC8B002010B54FF6FF74FCF7E8
:10BB000051FF80B2A042FAD010BD10B50446082102
:10BB1000FDF750FB237823F0010343F00203237069
:10BB200010BD12B1012A05D070470B6803604B6845
:10BB30004360704701F10803013813F8012D00F844
:10BB4000012F8B42F9D170470123018003717047A7
:10BB5000012341804371704740F20113018041800D
:10BB60008380704700687047016070471022002191
:10BB700060F01ABC30B50B46024601F1100518689A
:10BB80005968144603C40833AB422246F7D130BD8E
:10BB9000102308608B80704738B54FF6FE73C38062
:10BBA000038A03F0FE0343F4FE43002543F0010340
:10BBB00004460382458005718560C560456180F853
:10BBC0005D502830FFF7D2FF04F13800FFF7CEFFB9
:10BBD00004F14800FFF7CAFFA56584F85C5004F142
:10BBE0006000BDE83840FDF75BB9000037B5174D80
:10BBF000019104462846FAF743FA20802846FAF7CE
:10BC00002BFA0199A06104F11C0000F079FB0021DE
:10BC1000C4E90811102204F1280060F0C5FB1022CD
:10BC2000002104F1380060F0BFFB0021102204F174
:10BC3000480060F0B9FB2346054A43F8602F2046D0
:10BC4000A366FFF7A9FF204603B030BD08370020E8
:10BC500085C200000148FAF7F9B800BF0837002094
:10BC6000C180014805F010BE1A37002013B500F15D
:10BC700008030C4608684968012203C32146684648
:10BC8000FFF74FFF0248694605F0F8FD02B010BD0E
:10BC90001A370020037C61F3000303740388DB057B
:10BCA00002D5024805F032BE704700BF08370020B9
:10BCB000837810B5044663B90748FAF747F950B9D5
:10BCC0000548FAF763F930B9A378012B01D00123B5
:10BCD000A370002010BDFEE70837002010B5044611
:10BCE0006030FDF7DDF80648FAF750F930B904483E
:10BCF000FAF736F910B9A37803B1A07010BD00BFF0
:10BD00000837002010B504460448FAF7DBFC20B9D8
:10BD1000A378022B1CBF0223A37010BD083700209C
:10BD200038B50123044603FA01F10020FCF766FE52
:10BD30004FF4A07303FB00F5237CDB070BD5A3694D
:10BD400007489979FAF7BEFC294604F16000BDE87E
:10BD50003840FDF797B80248FAF718F9F4E700BF42
:10BD600008370020837803F0FB03032B10B504464B
:10BD700025D10388DB0606D4836911489979FAF73F
:10BD8000A1FC00B1FEE7A378042B1CBF0423A37021
:10BD9000236A1BB1626AA06901219847A169094819
:10BDA00005F078FD0D2808D1A1694B6933B1002356
:10BDB000C1E90433034805F06DFD00B1FEE710BD95
:10BDC000083700201A3700200378DA0708D40B68F8
:10BDD0001B789B0604D54FF47A516030FDF752B8BA
:10BDE000704700000148FAF73BB900BF0837002050
:10BDF0000148FAF7DBBB00BF083700208378022B2D
:10BE00001CBF022383701C3000F096BA03889B0786
:10BE100010B5044600D5FEE71048FAF721F97F284F
:10BE200006D094F911307F2B01D0834200DA607480
:10BE3000F9F7BFFE6369C01A002808DA616E04F1E1
:10BE400060004FF4FA32BDE81040FDF715B894F9E0
:10BE500011102046BDE81040FFF7D0BF0837002082
:10BE6000008880F02000C0F340107047008800F088
:10BE70000C00B0FA80F040097047008880F00400A0
:10BE8000C0F380007047008880F00200C0F34000DB
:10BE900070470000837870B50446164653B3033BE1
:10BEA000042B27D903889B0709D51448FAF728F9EA
:10BEB000A378052B01D00523A370002518E0FFF718
:10BEC000E2FFC8B10D48FAF7FDFB054600B1FEE7F9
:10BED000A378052B1CBF0523A3707F236374F9F798
:10BEE00068FE30446061002104F16000FCF7CAFF85
:10BEF000284670BD0D25FBE70C25F9E70837002023
:10BF0000008880F04000C0F3801070478269837819
:10BF1000526910B50446F2B1072B1CBF072383708A
:10BF2000FFF7EEFF90B11548FAF764FBA369D3E978
:10BF300004128B18C3F5A473C34207D504F1600043
:10BF4000A1F5A471BDE81040FCF796BF2046BDE8FE
:10BF50001040FFF707BF032B1CBF03238370C1787A
:10BF6000FFF784FF0028F1D00331C9B2052920462C
:10BF700028BF0521BDE81040FFF7D2BE08370020DA
:10BF8000037C024613F0010002BF108880F4807029
:10BF9000C0F300207047000010B50446FFF7F0FF23
:10BFA00020B9A378012B07D1002004E00448F9F759
:10BFB000EDFF0028F5D010BD0123A370F4E700BF0A
:10BFC000083700202DE9FF470829DDE90C890546DF
:10BFD0000F4692461C4603D011F0EF0F13D0FEE738
:10BFE00080F85C2000F128060FCB86E80F0098E867
:10BFF0000F0005F1380686E80F0099E80F0005F1FB
:10C00000480686E80F002846FFF72AFF48B9CDE921
:10C010000190CDF800800448234652463946FAF78D
:10C02000EBFA04B0BDE8F0870837002038B590F887
:10C030005C30934204460D4607D11C3000F082F973
:10C04000A36D9D4224BF0135A56538BD1FB50446CB
:10C05000806903681B781B072DD5C37ED9062AD4B7
:10C060000DF10F01FFF7B4FA28BBA069C37EDA0710
:10C0700003D494F85C10FFF711FB2046FFF7F0FEA5
:10C08000C8B19DF80F30082B15D1A06904F1380311
:10C090008360C37EDB0709D4A16D0191FFF7B8FA75
:10C0A00094F85C2001992046FFF7C0FFA06904F1D5
:10C0B0000801FFF72EFC04B010BD38B58378052BBE
:10C0C00005460BD00024FFF7C1FF2846EC702C7109
:10C0D00085F85D40FFF71AFF204638BD0D20FCE7CC
:10C0E00037B505460C46FFF7BBFE20BB0B681B7837
:10C0F0001A0720D5CB7EDB071DD50DF102012046A6
:10C10000FFF766FA00B1FEE79DF80230082B12D166
:10C1100001A92046FFF76CFA00B1FEE70DF103011B
:10C120002046FFF7A5FA00B1FEE79DF8032001992C
:10C130002846FFF77BFF03B030BD2DE9FF411E46C7
:10C14000044660300D469046FCF7AAFE0E2E25D020
:10C1500003D81EB30B2E23D0FEE70F2EFCD10027F1
:10C16000EB7E5B0705D5AA79394604F11C0000F087
:10C17000CFF829462046FFF7B3FF9FB92046FFF7C7
:10C1800075FE78B1E3782A7E9A420BD90133E370C9
:10C19000204604B0BDE8F041FFF7B8BE0127DFE755
:10C1A0000127E6E70023E3702379002E32D02046F2
:10C1B000FFF763FE074620B16F7E9F4294BF0027C2
:10C1C000012704F11C00009732462946039000F035
:10C1D000A5F8039807B3237901332371EB7E0E2E64
:10C1E00043F00203EB76D3D1A37894F85D10062BCD
:10C1F0001CBF0623A3702046FFF792FD94F85D3024
:10C200000133DBB2052B28BF052384F85D3004B071
:10C21000BDE8F0813746D4E7A378022B1CBF022388
:10C22000A37042463346294604B0BDE8F04100F011
:10C230007DB800008378033B10B50446042B1DD85D
:10C24000DFE803F0030718140300BDE81040FFF710
:10C2500089BD83690A489979FAF734FAA1692046B9
:10C260000E23BDE810400022FFF767BFBDE8104075
:10C27000FFF74CBEBDE81040FFF7C8BD10BD00BFC2
:10C28000083700200148FFF7D5BF00BF948B00207E
:10C29000036A70B505460C4616462BB121B11AB992
:10C2A000426A3146204698472846FFF7D9FD40B9F3
:10C2B0003CB1E37D9B0704D5227D21692846FFF729
:10C2C000B5FE3246214605F11C00BDE8704000F085
:10C2D00019B8000008B512B1836D8B4200D2816598
:10C2E000FFF7BEFD48B905481AB1BDE80840FAF7A6
:10C2F000B7B9BDE80840FAF7A5B908BD083700206E
:10C30000704700000148FEF769BD00BF688B002040
:10C310000148FEF71FB800BF688B00209DF80000A1
:10C3200000900148FEF72EB8688B00200148FEF708
:10C33000DBBA00BF688B00200148FEF719BD00BFC3
:10C34000688B0020014808F06BBD00BFE08A002028
:10C3500030B545F26C43044685B02E48CD5805F003
:10C36000C9FA284018BF03904FF000014FF078023F
:10C3700004F1080008BF039560F016F801220023BD
:10C38000C4E9002300232381A37203A81AF07FF9D4
:10C390002567A4F85A00FFF7AFFBA4F8580004F192
:10C3A0006C0008F0DEFB102104F12000FCF702FF16
:10C3B000054658BB102104F15C00FCF7FBFE054666
:10C3C00020BB082104F14100FCF7F4FE0546E8B962
:10C3D00004F1490002F0D1FE0546B8B9B4F858306E
:10C3E0000D4A009311210D4B04F1300060F05AFD0D
:10C3F000012340F2011284F8743084F87B304FF04E
:10C400000133A4F87620A4F87820E367284605B025
:10C4100030BD00BF083700201B5E0700105E07001C
:10C4200010B500210446C0F80011A0F80411FE2246
:10C430005FF0BAFF204610BD38B5B0F8045104468D
:10C440000544AC4217D26378FF2B01D1002038BDE0
:10C45000A31C9D42FAD3204619F034FC20448542A7
:10C46000F4D3204601F030FE0028EFD0204619F02A
:10C4700029FC0444E5E70120E9E70A46B0F8041185
:10C4800019F0E0BD2DE9F3410C460746802200215A
:10C4900020465FF089FF3D46012604F11008B7F8F9
:10C4A00004313B449D4280F095802B780E2B0BD8B5
:10C4B0000E2B0FD8DFE803F01A66345A764A0E3F87
:10C4C0000E0E0E0E860E1300342B22D0352B15D0F7
:10C4D000332B60D0284619F0F5FB0544DFE72146F1
:10C4E000A81C01F0FBFE84F87460F3E7B5F8033094
:10C4F00084F87C605BBAA4F85A30EBE769462846BA
:10C5000001F0C8FD0028E5D1009B236784F87F6017
:10C51000E0E7D5F8023084F87A601BBA6365D9E7A2
:10C520002A4652F8023FC4F841305368C4F84530F7
:10C5300084F87860CEE72A4652F8023FC4F84930C2
:10C540005368C4F84D3084F87960C3E7AB1C04F13C
:10C55000200C05F1120E18685968624603C20833B0
:10C5600073459446F7D184F87660B3E72946684668
:10C5700001F0EDFC694604F1300001F02CFE84F876
:10C580007760A7E7AA78EB7884F87B6043EA022318
:10C59000A4F858309EE74146A81C01F09FFE84F89D
:10C5A000756097E7AB1C04F15C0C05F1120E18687E
:10C5B0005968624603C2083373459446F7D184F83C
:10C5C0007D6087E7284601F0F3FC84F87E600090E8
:10C5D000E0667FE702B0BDE8F0810B46B0F80421C9
:10C5E00010B501460446184660F0C2FAB4F80421BA
:10C5F00080F8FE2010BD91F8FE20A0F8042160F024
:10C60000B7BA38B515460C4661B90E21FFF735FFAC
:10C6100010B91724204638BD50F8023F2B604368FC
:10C620006B60F7E73321FFF728FF0028F1D050F8BF
:10C63000023F2B6043686B600024EBE7FE2B70B574
:10C6400004461E460846114602D90625284670BDF6
:10C650002246FBF73EFD05460028F6D1A4F804610A
:10C660002046FFF7E9FE0028EFD0F9F7A2FAC4F858
:10C670000001EBE7B0F80431F7B505460F46164662
:10C68000002B3DD000290CBF182219228DF8042060
:10C690000A3B022201A930468DF80530FBF76BFDFD
:10C6A00038BB2C46B5F804312B449C4228D2237861
:10C6B00037B90E2B08D1204619F004FB0444F1E7EA
:10C6C000012F01D1332BF5E7342B14D1F9F771FA8F
:10C6D000D5F80031D4F80220C11A12BA91423ABFFB
:10C6E0009B181A1A00223421304619F09CFC0028AD
:10C6F000E1D003B0F0BD3146204619F0F6FAF6E776
:10C700000020F6E738B50446084679B14D78B4F80C
:10C71000042102350B1B55FA83F3D21A29445FF02A
:10C7200029FEB4F804315D1BA4F8045138BD2DE98D
:10C73000F843B0F804518846044617461E46FFF7F2
:10C740009CFEC5F1FE05ADB2014618B14378023337
:10C750001D44ADB206F10209A94518D82046FFF7DD
:10C76000D1FFB4F80431E0189944A4F8049104F816
:10C770000380467019F0B0FA3246394660F0F8F995
:10C78000F9F717FAC4F800010020BDE8F883032088
:10C79000FBE737B50C46054609780191204619F0AC
:10C7A000A2FA637801990246284603B0BDE83040FA
:10C7B000FFF7BDBF91F8743037B505460C4643B15D
:10C7C000684601F09BFD08236A460E212846FFF7C4
:10C7D000AEFF94F8753053B104F11001684601F0D2
:10C7E0008DFD08236A4633212846FFF7A0FF94F801
:10C7F0007A3043B1636D1BBA00936A460423342137
:10C800002846FFF794FF94F87C3053B1B4F85A10DF
:10C81000684611F0ECFE03236A4600212846FFF724
:10C8200086FF94F87F3053B1216F684601F08CFC8D
:10C830009DF806306A4635212846FFF778FF94F8C0
:10C84000783033B1082304F1410202212846FFF772
:10C850006EFF94F8793033B1082304F149020721BF
:10C860002846FFF764FF94F8763033B1102304F1C3
:10C87000200205212846FFF75AFF94F877305BB174
:10C8800004F13001684601F09BFC9DF80430009AE9
:10C8900003212846FFF74BFF94F87B3053B1B4F8DF
:10C8A00058305BBAADF800306A46022301212846B1
:10C8B000FFF73DFF94F87D3033B1102304F15C02A3
:10C8C00004212846FFF733FF94F87E3063B140F22D
:10C8D0000C4304F16C016846ADF8003001F085FBB3
:10C8E00069462846FFF755FFF9F763F9C5F80001D7
:10C8F000002003B030BD082311B90E21FFF717BF88
:10C900003321FBE710B50446FFF7B7FD014620468B
:10C91000BDE81040FFF7F6BE2DE9F04F01F5A8493C
:10C9200085B001F5A74680460D46174609F1600916
:10C930005836FFF781FD002868D00FB100233B7007
:10C9400005F5AD4A44460AF1280AB8F804314344D3
:10C950009C425DD223780C2B1AD8DFE803F0071233
:10C960001E2544301949191919194E00B4F803103D
:10C9700049BAC9B24846FDF771FB48B105B0BDE8F8
:10C98000F08FA178E378484643EA0121FDF760FA89
:10C99000204619F097F90444D7E705F5A740A11CF4
:10C9A000283000F0AFFDF3E72146684601F0CFFAEA
:10C9B00005F5A7406946303001F05EFCE8E76946BE
:10C9C000304608F060FA04F1020B3FB110226946CC
:10C9D000584661F05DFB08B101233B705946304673
:10C9E00008F040FBD4E7A11C304608F067F9CFE718
:10C9F000A11C50460DF01AFDCAE7204601F0D8FAF6
:10CA000069460090304608F0F9FAC1E70620B5E71C
:10CA10000020B3E710B533210446FFF773FF20462B
:10CA20003421BDE81040FFF76DBF0273427B002147
:10CA300022F0030281604273016041607047000090
:10CA400010B5017B0446054819F02EF80023236039
:10CA50006360637B23F00303637310BD68370020BA
:10CA6000F8B50A4607460C46017B1A4818F0FEFF47
:10CA7000064620B10023A4F804313046F8BD3B7BC4
:10CA800063B933212046FFF73DFF34212046FFF7ED
:10CA900039FFF9F78EF8C4F80001EEE7342120469B
:10CAA000FFF7EBFC05460028E7D0F9F782F8BA68F3
:10CAB000D5F80230811A1BBA99423ABFD218131A1C
:10CAC00033461A0EAA701A0CEA701A0A2A716B7190
:10CAD000DFE700BF68370020437B6FF3000370B5CA
:10CAE000437304460E46FFF7BBFF054678B9637BE8
:10CAF000217B43F00203637322463046FFF781FD3A
:10CB0000627BB0FA80F35B0963F30002627328462C
:10CB100070BD30B5C3B004460D466846FFF780FCD3
:10CB2000FF22002128465FF03FFC20466946FFF7C0
:10CB300097FF044618B929466846FFF74EFD204680
:10CB400043B030BD70B50D460446B5F80461017BB5
:10CB5000BEB9114818F0A8FF637B66F34103217B3F
:10CB6000637322462846FFF74CFD637BB0FA80F0E2
:10CB7000400960F300036373F9F71BF8A06000201D
:10CB800070BD05482A4618F065FF0028F8D1637B80
:10CB900043F00203E3E700BF6837002010B5C4B0DC
:10CBA000044602A80191FFF73BFC019902A8FFF798
:10CBB00022FD02A92046FFF7C5FF44B010BD38B5DD
:10CBC000044604301D46FFF730FF237F224623F042
:10CBD0000303237742F8205F0023C4E90B33A262EA
:10CBE0006361A361204638BD037F13F0010314BFC6
:10CBF000143018467047000010B5C2B004466846AD
:10CC0000FFF70EFC6946201DFFF72AFF20B90246F8
:10CC100002496846FFF780FE42B010BD0837002089
:10CC2000037C0448002B0CBF4FF080514FF00051A3
:10CC3000FBF70EBE3037002030B5C3B0044668465F
:10CC4000FFF7EEFB04F12000FCF780F8237F6FF381
:10CC5000000323776946201DFFF73EFF0546B0B964
:10CC6000217C04F114026846FFF7CBFC237FB0FA65
:10CC700080F0400960F300032377237C23B9054942
:10CC80002A466846FFF748FE2046FFF7C9FF2846B8
:10CC900043B030BD08370020FFF7CEBF73B50D4657
:10CCA00000F11406017C04460023324628468DF824
:10CCB0000730FFF7A6FCF8B1237F13F0010F08BF80
:10CCC0000026637C13F001030CBF1946211D30467A
:10CCD00001F05CFB9DF807300BB900281DDD2946EB
:10CCE000201DFFF72FFFB0B9104813F033FA20468C
:10CCF000FFF796FF00200EE0237F43F00103237728
:10CD0000237C002BDDD10A490DF107022846FFF7ED
:10CD100003FE0028D0D002B070BDE8D041F28831C7
:10CD200004F12000FCF75CF8E1E700BF8CB40020C0
:10CD30000837002010B5027F002363F30002044689
:10CD40004361836102770430FFF77AFE04F120002B
:10CD5000FBF7FCFF2046BDE81040FFF761BF000075
:10CD600030B5C5B0044602A80D46FFF759FB201D9B
:10CD700002A9FFF775FE044688B9352102A8FFF71E
:10CD80007CFB58B101A901F085F940B90549019B27
:10CD900045F26C428A5813402B6003B91724204691
:10CDA00045B030BD0837002030B5ADF5137D0446E1
:10CDB0002622002104A85FF0F7FA4FF2BF030EA865
:10CDC000ADF83230FFF72CFB207F830750D4324A76
:10CDD00045F2A963D35C023B012B49D8617C10F07A
:10CDE000010018BF04F1140011F0010118BF211D4A
:10CDF00001F0CCFA00283BDA257C75B950A8FFF782
:10CE00000FFB50A92548FFF72BFE02AA294650A880
:10CE1000FFF7F7FB10B3237C6BB31B21204817F0FF
:10CE20005DFC054658B30EA9201DFFF719FEBDF89D
:10CE30003C210EA92846FBF79EF9F0B904A816F08C
:10CE400087FB184B1648009404AA294618F0BCF832
:10CE500098B9237F43F00203237709E0617C11F046
:10CE6000010118BF211D02A801F090FA0028D2D1BB
:10CE70000DF5137D30BD0C21D0E7032807D141F219
:10CE8000883104F12000FBF7ABFF002DF0D02846DD
:10CE9000FBF761F8ECE700BF08370020748A002038
:10CEA0002C8900206FCF00000E4A45F2A96310B50F
:10CEB000D35C032B044607D8012B10D863B120465E
:10CEC000BDE81040FFF7ACBE042BF8D1FFF7B4FE6D
:10CED000054813F03FF9F2E7FFF7AEFEEFE7FFF783
:10CEE00063FFECE7083700208CB4002038B5054616
:10CEF0000430FFF753FE044610B92846FFF7D4FF6D
:10CF0000204638BD0148FFF74FBF00BF3C8A0020D4
:10CF10000148FFF749BF00BF708A002013B5002207
:10CF200004468DF80720084663B90DF10702102169
:10CF300018F0E8FF0346C0B99DF80720AAB1FF2A00
:10CF400008BF2523227F6FF341022277E26A22B1D4
:10CF50000021E1621846216B904741F2883104F1CB
:10CF60002000FBF73DFF02B010BD0623EAE7FFF704
:10CF7000D5BF00002DE9F041C2B0074668460D4616
:10CF800016461C469DF82081FFF74AFA6946381D6F
:10CF9000FFF766FD2946224817F0DDFB054600280D
:10CFA0003BD0B8F1000F15D01E4FA04444452DD002
:10CFB00014F8011B052902D13B78DB07F6D568463A
:10CFC000FFF75BFA0028F1D0294618F08EFE002802
:10CFD000ECD017E0134F6C46BDF804316B449C4213
:10CFE00014D22378052B07D13B78DA0704D42046E6
:10CFF00018F068FE0444EFE72946204618F075FE55
:10D000000028F4D02846FAF7A6FF06E00448324686
:10D01000294617F0E5FF0028F4D142B0BDE8F081C1
:10D020002C8900205E8B00202DE9F0470F8C94B0F6
:10D0300080460E469146F38BBB420AD800240094EA
:10D0400004AB4A4631464046FFF794FF14B0BDE8B2
:10D05000F087022303AA39463046FBF73AF8054623
:10D060000028EBD19DF80C309DF80DA00D2B22D19E
:10D0700054463F2C28BF3F24B91C234604AA89B23A
:10D080003046FBF706F8BAF1000FD7D098F8103009
:10D09000012BD4D104AB13F8012B342ACFD00135A6
:10D0A000EDB2AC42F7D814AB621C1C44342304F834
:10D0B000403CD4B2C3E70AF102010F44BFB2BAE761
:10D0C00010B5C4B002A801911446FFF7A9F901995F
:10D0D00002A8FFF76FFB28B9BDF80C2102A9204672
:10D0E000FBF749F844B010BD2DE9F0418CB005467E
:10D0F0000C4690460021262202A81F465FF054F9F4
:10D100004FF2BF03ADF82A302B7F9B0736D42B7C20
:10D110001C48002B0CBF0C211B2117F0DFFA064620
:10D1200070B3024621462846FFF7CAFF044660B99D
:10D130007FB902A816F00CFA134B1248009502AA08
:10D14000314617F041FF044660B13046FAF703FF5D
:10D1500010E03A4641463046FBF70DF804460028F9
:10D16000E7D0F2E7129BEB62139B2B632B7F43F01C
:10D1700002032B7720460CB0BDE8F0810524F9E7C7
:10D180000324F7E72C8900206FCF00002DE9F0433E
:10D190000D4691B0074691460021262206A89846E2
:10D1A000189E5FF001F92C784FF2BF03ADF83A30CA
:10D1B0001CB10E238DF8083001246B7833B110AA0E
:10D1C000631C1444332204F8382CDCB2AB7833B13E
:10D1D00010AA631C1444052204F8382CDCB2EB7846
:10D1E00033B110AA631C1444032204F8382CDCB2B7
:10D1F0002B7933B110AA631C1444022204F8382C92
:10D20000DCB26B7933B110AA631C1444072204F812
:10D21000382CDCB2AB7933B110AA631C144434222D
:10D2200004F8382CDCB2EB7933B110AA631C144437
:10D23000012204F8382CDCB22B7A33B110AA631C1B
:10D240001444002204F8382CDCB26B7A33B110AAF3
:10D25000631C1444042204F8382CDCB2AB7A33B1DA
:10D2600010AA631C14440C2204F8382CDCB2EB7AAC
:10D2700033B110AA631C1444352204F8382CDCB2F4
:10D280003B7C2748002B0CBF0B21192117F026FAF5
:10D290000746002841D018EB04030ED106A816F06B
:10D2A00057F976BB1E4806AA394617F099FE05467F
:10D2B00018BB284611B0BDE8F0830D228DF804207C
:10D2C00001A902228DF80530FAF755FF0546A0B9ED
:10D2D0005CB9B8F1000FE1D0424649463846FAF74A
:10D2E0004AFF05460028D9D007E0224602A9384661
:10D2F000FAF741FF05460028EBD03846FAF72BFE37
:10D30000D7E70AAA06F1100430687168134603C310
:10D310000836A6421A46F7D1C4E70325C9E700BF7D
:10D320002C89002010B5034B04460022FFF747FC70
:10D33000204610BD05CF0000427C0346C2F34000EA
:10D34000920742BF187FC04300F001007047427C43
:10D350000346C2F34000920744BF187F00F001006B
:10D36000704730B5C5B0044602A80D46019200933F
:10D37000FFF756F8DDE90021BDF8203102A8FFF7DC
:10D380005DF940B901462A4602A8FFF7B4FA02A99E
:10D390002046FFF783FC45B030BDFFF745BE0000D7
:10D3A00010B5064B04460122FFF709FC2346044A48
:10D3B00043F8342F2046E36310BD00BF11CF0000B7
:10D3C000F5D4000010B50446FFF7B4FC04F13400B6
:10D3D000BDE81040FBF7BABC10B50446C2B06846C1
:10D3E000FFF71EF8227F002363F300026361A3614D
:10D3F000227769462046FFF751FC42B010BD10B5B8
:10D40000C2B004466846FFF70BF86946201D343465
:10D41000FFF726FB2046FBF799FC34216846FFF70F
:10D420002CF858B1D0F8023040991BBA6FF0004286
:10D430009A4228BF1A462046FBF7CCFC42B010BDEA
:10D4400070B5C4B0054602A80E4601920093FEF7DF
:10D45000E7FFDDE90021BDF8203102A8FFF7EEF873
:10D46000044668B93246012102A8FFF744FA02A92E
:10D470002846FFF713FC044610B92846FFF7BFFF04
:10D48000204644B070BD38B50546FFF72FFD044671
:10D4900010B92846FFF7B3FF204638BD10B5C2B01B
:10D4A00004466846FEF7BCFF6946201DFFF7D8FA20
:10D4B00034216846FEF7E1FF78B1D0F80230A16B65
:10D4C000409A1BBA881A984207D2521A1A4404F199
:10D4D0003400FBF77FFC42B010BD6846FFF79AFAB4
:10D4E00069460348FFF7DAFB2046FFF76BFFF2E7D8
:10D4F0003C8A00200148FFF7D1BF00BF708A00209E
:10D50000FFF792BD38B5082204460D4660F0C0FD15
:10D5100030B9BDE8384008484FF40031FBF7A1B9F5
:10D520002B6823606B6863600348BDE838404FF4A4
:10D530000031FBF78DB900BF3037002010B5002354
:10D540000446036043600249FFF7DCFF204610BD3C
:10D55000235E070010B50446043003F082FF234623
:10D56000074A43F8382F94F84A202364002363F3D2
:10D5700000026364A4F8483084F84A20204610BDB5
:10D5800035D8000007B590F84A30DB0704D5B0F86D
:10D59000480003B05DF804FB06480DF1060112F0E7
:10D5A0006FFC18B14FF47A73ADF80630BDF8060081
:10D5B000EFE700BF8CB40020F8B5174A45F2AA6324
:10D5C0000446D35C9B0726D5144812F0C2FCB8B1C0
:10D5D0002046FFF7D7FFA68A0546E6B9271D224653
:10D5E0000F49384604F028F929460122384603F04D
:10D5F000B3FF2A4631460B48BDE8F84002F07EB939
:10D60000A28A42B10748012102F078F9201DBDE845
:10D61000F84004F02DB9F8BD083700208CB4002084
:10D62000B5D90000DA8A00208B0501D5FFF7C4BF09
:10D63000704790F84A20A0F8481042F0010280F8A4
:10D640004A20FFF7B9BF000070B5C2B06846FEF7C8
:10D65000E7FE1848142117F041F8044630B390F85B
:10D660003030042262F3C60380F830306946124835
:10D67000FFF7F6F9B0B9114E082516F8011B6846F8
:10D68000FEF7FBFE70B1214618F02FFB50B9013DAB
:10D69000F3D10B4A45F2E8330621D258204618F060
:10D6A000C2FC18B12046FAF756FC0024204642B0CE
:10D6B00070BD00BF2C890020408A00202B5E07002F
:10D6C0000837002073B504460E46FFF7BDFF054638
:10D6D00080B122460A490B4817F02CF90094084BF8
:10D6E00008483246294617F06FFC044620B9204608
:10D6F00002B070BD0324FAE72846FAF72CFCF6E7DF
:10D7000031D800002C89002002460846C98B3B29ED
:10D7100000D8FEE73C393C2389B2FAF7DABC26226E
:10D7200000215EF041BE0000F0B5074691B02448EC
:10D730000C4606211546FAF7D1FF064601A8FFF769
:10D74000EEFFB6B3234601AA04F1200C186859680D
:10D75000144603C4083363452246F7D11868206095
:10D760009B88A3804FF2BF03ADF82630F8F721FA6B
:10D7700032302A460B900CAC1035106851682346A5
:10D7800003C30832AA421C46F7D13C2201A9304605
:10D79000FAF7F1FC78B907F1440001223146FAF7B3
:10D7A00028FE3B6C07F13800984202D10B99FBF739
:10D7B00007FB11B0F0BD3046FAF7CDFBF9E700BF2B
:10D7C0007C37002030B5044693B003A8FFF7A7FFCD
:10D7D000636CABB1596899B1236C04F138059D4273
:10D7E0000ED103A80191FFF78FFFF8F7E2F90D9B27
:10D7F0000199C01A002805DA19462846FBF7E0FA15
:10D8000013B030BD04F14400FAF738FE07480EA902
:10D8100007F020FB03A92046FFF754FF0028EFD0B4
:10D8200000212846FBF7DCFAEAE700BFE08A002087
:10D83000FFF7C8BF0148FFF7C5BF00BF08B600200B
:10D84000F0B593B00C460322002106466846FAF76D
:10D8500058FB08A8FFF763FF204617F03FFD00289C
:10D8600042D00DF102021221204618F05DFB002883
:10D870003AD108230DEB03021321204618F078FB60
:10D8800090BB11210DF1060301AA204618F0AEFA53
:10D89000014648BB371D6A46384603F08FFE0546F1
:10D8A00010B3BDF80630BDF804202146FAF77AFC23
:10D8B000E0B902A90CA801F09AFDBDF80230ADF85C
:10D8C000423008AA2946384603F00CFF70B91023ED
:10D8D0000DEB03021521204618F04AFB20B904AADB
:10D8E00008A93046FFF720FF13B0F0BD2846FAF72D
:10D8F00032FBF9E770B58CB002A80D461646FFF76B
:10D900000EFF4FF2BF032848ADF82A300DF1020197
:10D9100012F0AEFA002845D124481C2116F0ECFE86
:10D92000044600283ED0728C122118F070FBB0BB68
:10D93000082306F118021321204618F034FB70BBAF
:10D940001B4A45F2B8631421D25A204618F05FFBF7
:10D9500028BB2A8CEB8B9B1A4FF61172ADF8042072
:10D9600004225BBA0DEB02012046ADF80630FAF74F
:10D9700002FCA0B9BDF806302A8C5BBA9BB22946DE
:10D980002046FAF70FFC50B9BDF8021002A815F0B6
:10D9900007FE064802AA214617F022FB10B12046D6
:10D9A000FAF7D9FA0CB070BD8CB400202C89002095
:10D9B00008370020FFF79EBF70B5027A531E3F2B39
:10D9C0000FD80731D0E900450E461046072809D97F
:10D9D000230A083806F80149C0B243EA05642D0A53
:10D9E000F4E7FEE7D308C3EB4313A1EBD20102EB4C
:10D9F000C30212F0FF0209D001239340DBB20A7880
:10DA00005842013B0240234013430B7070BD102964
:10DA100000D9FEE700F8011B102200215EF0C4BC13
:10DA200070B503784BB30C88DA00D5B2013BB4FB78
:10DA3000F5F205FB1242DCB2C2F3C403E31A50FA5A
:10DA400083F302F007025B78012606FA02F2134024
:10DA500013D04A88B2FBF5F105FB1122C2F3C403CF
:10DA6000E41A50FA84F302F007025B7806FA02F235
:10DA7000134214BF3046002070BD1846FCE77FB546
:10DA800004460D4602A841F2210117F0BFFE48F2FC
:10DA9000050103A817F0BAFE04F10806B4420AD043
:10DAA00014F8011B019102A817F0B4FE019903A814
:10DAB00017F0B0FEF2E7BDF80A302B80BDF80E304B
:10DAC0006B8004B070BD13B500230C466946CDE9E8
:10DAD0000033FFF771FF21466846FFF7D0FF02B021
:10DAE00010BD10B510F8014B0023DAB2944207D9EB
:10DAF00010F8012B8A4203F10103F6D0002010BD7B
:10DB00000120FCE730B5C7B0054608A80C4618F060
:10DB100071FD08A818F083FD0822294608A818F00E
:10DB200084FD694608A818F086FD6B4603CB20608B
:10DB30002378616043F00203237008A818F067FDA2
:10DB400047B030BD2DE9F0479946274B8EB00446CB
:10DB50000DF1100A18680490904620469A889B7927
:10DB6000ADF814200F468AF80630FBF74CF818B9C8
:10DB700007200EB0BDE8F0874FF480712046FAF719
:10DB800059FF112106463846FAF754FFB31F9BB2DE
:10DB9000F92BC5B2ECD8102DEAD81222002109A821
:10DBA0005EF002FC9AE80300D8F800300690ADF869
:10DBB0001C10CDF81E302A46D8F80430CDF822309B
:10DBC00039460DF126005EF0D3FF4FF4804310225A
:10DBD000CDE90032CDF8089005F10E0306AA3146D2
:10DBE0002046FBF7F3FAC4E7145E07004278102AD8
:10DBF00028BF1022002102305EF0D6BB0346074A40
:10DC000010B543F8042FC36047F230530361044654
:10DC1000FAF7C8FEA4F85600204610BD7DDD0000CE
:10DC2000F8B50546164817461E4616F094FD0446FC
:10DC3000B8B13246102118F0DFF9E0B9EA682B1DBF
:10DC40009A420FD1012E06D1B5F856200B2120465D
:10DC500018F0DDF978B90A483A46214617F0C0F9BC
:10DC600048B9F8BD05F1140340220A21204618F0F6
:10DC7000B2F90028E6D02046BDE8F840FAF76BB9C3
:10DC80002C89002037B50D480193154616F063FD29
:10DC9000044680B1019A102118F0AEF928B907485E
:10DCA0002A46214617F09CF928B1204603B0BDE86A
:10DCB0003040FAF750B903B030BD00BF2C890020C6
:10DCC00030B58BB026220D46684600215EF06CFB15
:10DCD0004FF2BF030B48ADF82230112116F0FEFCC5
:10DCE000044660B12946684615F072FC05486A464C
:10DCF000214617F075F910B12046FAF72CF90BB050
:10DD000030BD00BF2C8900204A1E47F22E539A4294
:10DD10009ABF0161002007207047000007B540F25C
:10DD20000B23ADF80430B0F85630013304229BB217
:10DD3000A0F856300DEB02015BBA0448ADF806308E
:10DD400012F055FE03B05DF804FB00BF8CB4002058
:10DD500010B504460430FAF7F9FF2046BDE810403C
:10DD6000FFF7DCBF044A45F2A963D35C042B01D161
:10DD7000FFF7EEBF704700BF083700200148FFF7EC
:10DD8000F1BF00BF54B60020F7B545F2A9631746AE
:10DD9000204AD35C042B04460D4638D10DF1050210
:10DDA0001021284618F0AEF888BB0DF106020B21B1
:10DDB000284618F0B9F850BB1748092112F033F87B
:10DDC00060B1B4F85620BDF806309A4206D19DF8ED
:10DDD0000560012E04D02046FFF7BAFFFF2610E0B1
:10DDE000F98B43884ABA5BBA92B29BB29A4203D08B
:10DDF0004180094812F0A2F94CF25031201DFAF787
:10DE0000EFFF33463A4629462046FFF73BFF03B073
:10DE1000F0BD00BF083700208CB4002013B50923E3
:10DE200003700446022349BA4370418043710B21B9
:10DE300052BA08230171C280237210230830637222
:10DE40000190FFF7D3FE012301986372FFF7CEFE26
:10DE500002B010BD08B5083017F034FF0830C0B26A
:10DE600008BD0000F0B545F2A9631546284AD35C09
:10DE7000042B99B004460E4607D0FF232A463146AC
:10DE80002046FFF7CDFE19B0F0BD224805F1100184
:10DE90000CF0BEFB0028F0D0402207AB0A21304630
:10DEA00018F01CF802460028E7D1E368271D9F42BE
:10DEB00009D007A904F11400FAF720FE0028DCD0ED
:10DEC0002046FFF745FFB4F85630E98B01339AB28C
:10DED00049BAA4F8562089B26846FFF79FFF684602
:10DEE000FFF7B8FF694602460B4812F080FD034673
:10DEF0000028C2D107AA412104F11400FAF78DFECF
:10DF00004CF250313846FAF76BFF0123B6E700BFF9
:10DF100008370020B08D00208CB4002000BA704774
:10DF20004200400800F0553002F0AA32024393004C
:10DF3000920802F0333203F0CC33134318011B096B
:10DF400003F00F3300F0F030184300BA70474A78FE
:10DF5000102A28BF1022023101600271704710B5EB
:10DF6000044610220846A11C00F018F9607010BD8C
:10DF700041780230FAF718BE38B50D4641780446AC
:10DF8000102928BF10212846FFF741FD6278102A8A
:10DF900004F1020105F1010028BF1022BDE838405C
:10DFA0005EF0E6BD4078022894BF00200120704753
:10DFB00013B50446684606F0D4FD62786388023AD9
:10DFC000D2B2022A5BBA28BF02226846211DADF8F0
:10DFD000003006F0CBFD009B00209AB262F30F00E8
:10DFE0001B0C63F31F4002B010BD0A88034652BAEF
:10DFF00008465A80191D022206F007BE00232DE9AB
:10E00000F3410B60438904460D462BB1DFF8808055
:10E01000608910B1022803D8062002B0BDE8F08163
:10E02000606870B3218902236A46FAF732F86E46B7
:10E03000737862899F1CBA42EED33278C2B9042B3E
:10E04000EAD1606820B1218906236A46FAF741F8CF
:10E05000D6F80200FFF762FFFFF762FF3378002B6C
:10E0600018BF00222B6808BF4246104003432B60B4
:10E070006389DB1B638163682BB123891F4427817C
:10E08000C6E72668D4E723681F442760C0E700BFBF
:10E0900000F8FF071FB500230293ADF80C30831C76
:10E0A00001934378ADF80E3001A8FFF7A7FF05B044
:10E0B0005DF804FB07B501A9FFF7ECFFB0FA80F0AB
:10E0C000400903B05DF804FB02780C2A034611D81E
:10E0D0000C2A11D8DFE802F0120720181E1E1020AB
:10E0E000101010101A0002225878904234BF0020FD
:10E0F00001207047352A0BD0012070474278022A50
:10E100000CD9023010F079BAFFF732BFFFF74ABFDF
:10E11000FFF7D0BF1022E7E70822E5E700207047AD
:10E120001FB50023CDE902030C46019303AA0DF1AC
:10E130000E03352117F05AFE18B9214601A8FFF742
:10E140005DFF04B010BD0000002310B583710A4BC1
:10E150001B780446002B094818BF002008400AD04D
:10E16000237004236370FFF7DBFEFFF7D7FE06235F
:10E17000C4F80200A37110BD075F070000F8FF0795
:10E1800013B504466846FFF7DFFF9DF806306A4680
:10E190003521204617F007FF02B010BD70B50B46C1
:10E1A00005460021184616465EF0FEF82C792968CF
:10E1B000B44228BF344622465EF0DAFC204670BDE9
:10E1C00038B50D46044611212846FAF733FC256080
:10E1D0002071204638BD70B50E6809790546304675
:10E1E000FAF728FCC4B2102C10D822462946304633
:10E1F0005FF04EFF08B92B5D53B1224631462846E9
:10E200005EF0B6FC00232B55184670BD0720FCE7D6
:10E210001820FAE713B511230446084600918DF83B
:10E220000430FAF7F0FC28B169462046FFF7D3FF27
:10E2300002B010BD0720FBE710B50C4619B1182934
:10E2400007D0204610BD06484FF48031FAF700FB96
:10E25000F7E703484FF48031FAF703FB0024F0E7B7
:10E260003037002010B50446FFF7D4FF01462046A2
:10E27000BDE81040FFF7E0BF10B50446FFF7ABFF65
:10E2800001462046BDE81040FFF7D6BF08B5113063
:10E29000FFF7C0FF182808BF002008BD10B50023F5
:10E2A0000446037043740449FFF7DCFF034920462A
:10E2B000FFF7ECFF204610BD105E0700335E07003D
:10E2C00010B50446D0F80200FFF728FE218800228E
:10E2D00049BA8BB2101843F1000110BD38B50C4695
:10E2E0000546FFF7EDFFC4E90001EB885BBAC3F315
:10E2F0004E0203F001032281A37238BD38B50546F2
:10E30000D1E900030C465BBA2B80FFF707FE228998
:10E31000A37AC5F8020043EA42035BBAEB8038BD3A
:10E32000F8B50E460746FFF7CBFF044630460D46CC
:10E33000FFF7C6FF8D4208BF84421AD1FB885BBA43
:10E34000C3F34E0299B2F3885BBA98B2C3F34E039B
:10E350009A4202D015D90120F8BD01F0010300F066
:10E360000102934210D0002B0CBF4FF0FF30012070
:10E37000F2E7A94208BFA0422CBF4FF0FF300120B6
:10E38000EAE74FF0FF30E7E70020E5E720B9081E95
:10E3900018BF01204042704709B1FFF7C1BF0120FB
:10E3A000704773B50646154601910024311901A83E
:10E3B000FAF770FB78B9019B032C1A7806D02E2A45
:10E3C00004F1010407D101330193EFE7954218BF2F
:10E3D000062002B070BD0620FBE7837C5A0702D5F9
:10E3E000C3F3C300704701F0B6B8000070B5002653
:10E3F00004460D461022C0E90166067031460C3015
:10E400005DF0D2FF0C4B2946C4E9073604F1240025
:10E4100018F0BDFD294604F12C0003F02AF8294626
:10E4200004F1380001F00CFB294604F1D80002F099
:10E43000D7F8204670BD00BF41F1000030311346CF
:10E4400002488AB20021FAF70AB900BF7C370020DF
:10E45000014AFFF7F3BF00BFB05D0700024B00F0B9
:10E460003800185C704700BF415E070020B10228E9
:10E4700014BF0020202070470820704730B587B0B7
:10E4800093798DF80430383000230D46144602A9E4
:10E4900008328DF8053001F0E7FA02A801F089FA98
:10E4A000023081B204A801F0BDFAA8B102A801F0BF
:10E4B00080FA02A902462846F9F7A8FEB0B902225E
:10E4C00001A92846F9F7A2FE80B9A388A0715BBA1A
:10E4D00008335BBAA38009E004A801F06AFA04A932
:10E4E00002462846F9F792FE0028DFD007B030BD7B
:10E4F0002DE9F04F0C468FB0282304AA00212046B6
:10E50000F9F7E7FD9DF8166026B1002630460FB0FA
:10E51000BDE8F08F02236A4628212046F9F7D9FD8D
:10E520009DF80180E38B08F101084FEAC80808F163
:10E53000280B5B4501D20626E8E7B246B1463746CE
:10E540002A255B462A46214601A801F039FA9DF8A2
:10E550000430012B11D96D2B3CD1002FEBD19DF84C
:10E5600005A0BAF1040FE6D82A2D2BD19DF8013071
:10E57000002B2F4608BF4FF0010901A801F019FA3E
:10E580000544ADB2AB45DCD8D5D1B9F1000F30D0E0
:10E59000082208F120012046F9F7B8FE2A2F1CD1E5
:10E5A0009DF800308DF81630BDF814305BBA083B8A
:10E5B0005BBAADF8143004AA282300212046F9F7ED
:10E5C000B7FDA3E705F108032F465B4508BF4FF0F1
:10E5D0000109D2E74FF00009CFE79DF80130013B78
:10E5E0008DF801306A46022328212046F9F7A0FD64
:10E5F000DAE7002F89D00AF10201C9B202A801F0BE
:10E6000004FA02A801F0D5F902AA03463946D5E773
:10E6100010B504460C30F9F7B1FF04F11C00BDE859
:10E620001040FAF729BB2DE9FF470C8C0F468146B5
:10E6300090469A4602AA022321463846F9F749FD38
:10E640000646002838D19DF80950FB8B013504EBB4
:10E65000C505ADB2AB4233D30234A4B208F1080809
:10E6600009F13809AC4223D22B462246394603A889
:10E6700001F0A6F9A8B99DF80C30012B05D803A824
:10E6800001F097F90444A4B2ECE76D2B0BD1CDF85F
:10E6900000A0434622463946484601F04EFB00287A
:10E6A000EDD0064608E013F0C00FE8D0022603E0E4
:10E6B00021463846F9F77AFC304604B0BDE8F087C9
:10E6C0000626F9E737B50D460823098C6A46284621
:10E6D000F9F7FFFC044660B9BDF802305BBA9AB2A4
:10E6E000C3F3CC0343B9D30706D408212846F9F76E
:10E6F00051FC204603B030BD0224FAE738B5044689
:10E700003AB1012A0FD02368002B0CBF0320002050
:10E7100038BD0D680A6000688542F4D008B1F9F789
:10E720001AFC2560EFE70868C18BF9F7E3FF05469F
:10E730002068A842F1E700002DE9F74F0846884617
:10E7400000F009FF414682463B48DFF8ECB00BF091
:10E750005FFF3A4A009045F27C134FF00009D7580A
:10E760004D46002F63D0394658460BF060FF002815
:10E7700055D13946404600F02BFF3A7C824206468E
:10E7800014D838460192FFF728FE019A044616462F
:10E790001022414638465FF07BFC002846D03DB948
:10E7A0003A7CB2423DD9B1463D4638E05446EFE7A7
:10E7B0003846FFF712FE01902846FFF70EFE019A39
:10E7C0008242384608D2FFF708FEA04234BF00203C
:10E7D00001200028E4D122E0FFF7FFFD0190284648
:10E7E000FFF7FBFD019A824207D92846FFF7F5FDA6
:10E7F000A0422CBF00200120EBE7B87CAA7C42405D
:10E80000D30702D500F00100E3E7B145C8D306D134
:10E81000394658460BF0FCFE009B9842C0D07F69F9
:10E820009FE73846FFF7D9FD8246BCE73D462846BC
:10E8300003B0BDE8F08F00BFB08D00200837002086
:10E84000F0B50C468DB002F118010546084601915D
:10E85000164600F0B0FE019960B11F4804F0D2FDE9
:10E8600040B1E18B2046F9F745FF014610B128463B
:10E87000FFF7CEFE6023029340238DF80F30B3885C
:10E880005BBA28335BBA08A8ADF80C3000F0F8FD8D
:10E89000292308A928468DF80E30FFF74DFF0346BF
:10E8A000B8B104AE00F1100718685968324603C2C7
:10E8B0000833BB421646F7D102AA21462846FFF785
:10E8C000DDFD20B9282202A92046F9F79FFC0DB0F2
:10E8D000F0BD1420FBE700BFD08F00202DE9F047EA
:10E8E000112BB1F81EA08AB080460D4616469946F7
:10E8F00002F1100775D1538C52483A46314614F054
:10E9000025FF00286DD095F83100C0F3410014F0C8
:10E910005DFF840104F47C6444F4C044602364BA61
:10E9200096F825200093ADF80040C4F3072402F0C8
:10E93000030324F0300444EA031496F824308DF8DD
:10E9400001409AFA9AFAADF804A08DF806901BB926
:10E9500012F0080F08BF402330468DF8073000F052
:10E9600012FD002844D13378FF2B41D0334602AC4E
:10E9700018685968224603C20833BB421446F7D1CF
:10E9800006AA3B4607F1100C9246186859681446CF
:10E9900003C4083363452246F7D1384600F0FFFD33
:10E9A000C0BB282269462846F9F730FC0446C8BB9C
:10E9B00028464B46524602A918F0B5FA384600F0F0
:10E9C000FAFD98BB96F8253095F83120C3F3001373
:10E9D00063F3861285F8312029464046FFF718FE7A
:10E9E00020E095F83100C0F34100FFF73FFD90E7CC
:10E9F00039464046FFF7A0FE08B3034602AC00F1DB
:10EA0000100C18685968224603C20833634514463F
:10EA1000F7D1B5E76A4629464046FFF72FFD044681
:10EA20000028BED020460AB0BDE8F0876A462946D5
:10EA30004046FFF705FF0028C4D00446F2E714243F
:10EA4000F0E700BF2C89002070B50B480E4611F08E
:10EA5000A7F8044668B9094A45F27C13D5584DB168
:10EA60003146284600F0B4FD2B7C834201D96D6904
:10EA7000F5E70124204670BD8CB400200837002043
:10EA800007B509480DF1060311F08CF940B90749A3
:10EA9000BDF8062045F2B863CB5A9A4208BF04205D
:10EAA00003B05DF804FB00BF8CB4002008370020E1
:10EAB00070B53C2204460E4600215DF075FC3146DF
:10EAC000204600F05BFF054680B9A379112B05D0E5
:10EAD0003A2B03D0062B0AD1142300E0082304F1BB
:10EAE000280228213046F9F7F4FA00B10625284615
:10EAF00070BDF0B5044603C989B006AD85E80300D2
:10EB0000294604A817461E4607F0F8FB10B9BDF8C1
:10EB100014308BBBBDF81C3073B3069B1B7803F01D
:10EB2000E003602B28D106F5A8465C3600953B46ED
:10EB30000DF10F022146304606F0A0FF98B9A379E7
:10EB4000112B07D03A2B15D0062B0CD1142204F12F
:10EB500028010BE09DF80F3004F128012BB12A4663
:10EB6000304607F0A2F909B0F0BD0822284616F099
:10EB70001EFFF8E70822EAE71720F4E78379062B5F
:10EB800001D0112B03D1408D40BA80B270470020D4
:10EB9000704710B50446006808B1F9F7DCF9204663
:10EBA00010BDF0B585B00F469DF828501146112DC7
:10EBB0004FF00002064603920AD03A2D08D0062DE7
:10EBC00006D0002403A8FFF7E4FF204605B0F0BDFF
:10EBD0009DF82C20019303A8FFF790FD0446002820
:10EBE000F0D1112D019B0BD03A2D10D0062DE8D17C
:10EBF000039A394606F1D80002F00AFA0446E1E722
:10EC000003991A4606F12C0002F090FDF6E70399ED
:10EC10001A4606F1240018F0EBFAEFE72DE9F0436D
:10EC200085B01F46002301930B689DF830809DF846
:10EC30003490164693F83220D20705460C4601D48C
:10EC4000042407E04268002AFAD0DB8BB3F5A06FFA
:10EC500007D9022401A8FFF79CFF204605B0BDE8B4
:10EC6000F083334806F110010BF0CAFC10B1B9F182
:10EC7000000FEED02B786BB1B8F1000F0AD02C4802
:10EC800031460BF0BDFCC0B9112F36D03A2F21D040
:10EC9000062FD5D021469DF8382001A8FFF72EFD7C
:10ECA00004460028D6D101992846FFF721FC019897
:10ECB0000194D5E901319847CCE706F108084046B0
:10ECC00000F01FFB0028DFD0404600F04EFB00287C
:10ECD000DAD1B5E7314605F1240018F009FA002829
:10ECE000D8D0206808230DEB0302018CF9F7F1F965
:10ECF0009DF80830802BCDD1ABE720680823018C2C
:10ED00000DEB0302F9F7E5F9BDF80A10094849BA15
:10ED100089B202F049FD002892D0BDF80A100548DA
:10ED200049BA89B202F036FD0028B3D088E700BFA7
:10ED3000B08D0020B48700202DE9F04786B0DDE9D2
:10ED40000E8705460C4691461E464FF0010A38785C
:10ED500010B998F800307BB920680223018C05AA0D
:10ED6000F9F7B7F940B998F800302C2B12D006D833
:10ED70004BB12B2B08BF022006B0BDE8F0873B2B20
:10ED80001DD03C2BF8D121683B4632462846FFF780
:10ED90004AFC0DE0CDF808A03A782146CDE9000202
:10EDA0004A462846FFF73AFF21682846FFF78AFCC3
:10EDB0000028E1D19DF8143088F80030C7E7022020
:10EDC000DAE700002DE9F04F9DB00F460DF1200964
:10EDD000002180469246484626225DF0E5FA00234F
:10EDE00039688DF8163012A800F0C8FD06460446B2
:10EDF000002871D10DF1500B10909BE80F000CAC66
:10EE000084E80F0018AC94E80F0089E80F009DF823
:10EE10004F308DF844309DF84930C6F307221B115E
:10EE200063F301029DF860308DF84520FF2B59D126
:10EE30003B6893F8323013F00C0F51D1204600F0AC
:10EE4000BAFB064620B1AB48214604F0DBFA064681
:10EE50003B6893F8322012F00C0F03D093F8313056
:10EE60005A066ED5A448214601F081F801230546D3
:10EE7000002866D08DF8163038682821F9F796F802
:10EE80009DF84E308DF817300DF1160301930DF1FA
:10EE9000170300934A4612AB39464046FFF74CFF32
:10EEA0000446C8B99DF81630002B70D09DF8173075
:10EEB000292B6CD13B6806903246394606A893F858
:10EEC00031B0FFF71BFCCBF3801B054600283AD07E
:10EED00006A8FFF75EFE2C4620461DB0BDE8F08F69
:10EEE0000126B5E78448214601F00DFA054628B110
:10EEF00001238DF8163035462E46BDE73B6893F862
:10EF0000323013F00C0F11D0204600F057FA98B9A8
:10EF100021464046FFF798FD70B9224659464046C3
:10EF2000FFF7AEFDB0FA80F6760906E0204600F065
:10EF300045FA0028E0D1E7E7012686F00105EDB2A9
:10EF40009AE7012598E7069890F83130018C6BF329
:10EF5000861380F83130F9F741F8069A6748214660
:10EF600008F031FB069B524607A94046CDE906430F
:10EF7000FFF728FF07A8FFF70CFE06A88DF816403C
:10EF8000FFF707FE9DF8163043B3002501E0002D82
:10EF9000F8D0BAF1000F13D19DF8163085F00105B5
:10EFA000002B14BF1A463246EDB2CDE9013200956E
:10EFB0009DF817304A4639464046FFF72FFE044673
:10EFC0009DF8163053B19DF81730009301964B46CB
:10EFD0003A4612A94046FFF7E4FD0446002E3FF4EE
:10EFE0007BAF3B6893F8323013F00C0F0AD14448E2
:10EFF00009F079F900283FF46FAF9DF84F30013BDD
:10F000008DF84F309DF84F30FBB18DF81C303868CB
:10F01000012307AA0721F9F78BF89DF817303A2B3F
:10F0200015D138680123018C07AAF9F752F8044674
:10F0300000287FF451AF9DF81C10324A062312F8C5
:10F04000010B814203D0013BF9D1022444E7386827
:10F0500090F83250C5F38105022D17D19DF8173075
:10F06000112B13D1018C02312B4607AA89B2F9F773
:10F0700030F8044600287FF42FAFBDF81C305BBA8F
:10F080009BB24FF2BF0293423FF425AF386890F82D
:10F090003230C3F38102012A1FD1DB071DD49DF852
:10F0A0001730112B19D1018C0231022307AA89B222
:10F0B000F9F70FF8044600287FF40EAFBDF81C30B6
:10F0C0005BBA99B2ADF81C309DF81730112B04D102
:10F0D0000D4802F069FB0028B7D03B680793002376
:10F0E00006483B6007A908F071FA07A8FFF751FD31
:10F0F000F2E600BFD08F002084880020B88C00206A
:10F10000B08D00207A5E0700B487002073B50546F5
:10F1100000F10C063046F9F7D5F9044668B101460E
:10F120003046F9F748FA002201A928460194FFF772
:10F1300049FE01A8FFF72DFDECE702B070BD00000D
:10F140000148FFF7E3BF00BF8887002070B5013991
:10F1500005460024E6B2F300B242D8B20CD92B5DCA
:10F1600001340E5DB342F5D073401A0604D4013069
:10F170005B00C0B2DBB2F8E770BDFD2300F8013BD5
:10F180000721FAF717B838B5054614460732D208F2
:10F190005DF0EEFC2C7438BD027CD31DDB1010B585
:10F1A00008D0591EC2EBC3044FF0FF32A240445CAA
:10F1B00022404254002299B20F2902D8C25401338E
:10F1C000F9E710BD102A00D9FEE7FFF7BFBF10B561
:10F1D000037C0C7C9C4208D1E21DD208FFF7F2FFB1
:10F1E00084428CBF0020012010BD0020FCE72DE9E7
:10F1F000F0410F7C047CBC42A04628BFB84608F111
:10F200000702D20806460D46FFF7DCFF804505D809
:10F21000BC422CBF00200120BDE8F081C0F3C70331
:10F22000F45CE85C8442F4E700F0E703202B06D0AE
:10F2300000F0DF00A0F14003584258417047012020
:10F240007047036823B94068B0FA80F040097047FE
:10F2500000207047036803330AD182884FF6FF739A
:10F260009A4205D18379FF2B02D1C079C00970473A
:10F270000020704708B50821F9F79CFF00B1FEE7B0
:10F2800008BD0B6803604B684360704713B50446C4
:10F29000086849686B4603C39DF80030002283F07C
:10F2A0000203694620468DF80030FCF73AFC02B0B4
:10F2B00010BD10B50C46002201462046FCF731FC7B
:10F2C000237883F00203237010BD10B50C46002292
:10F2D00001462046FCF725FC02232372237883F0A5
:10F2E0000203237010BD4FF0FF320023C27049BAF1
:10F2F0006FF0010203704370837002714371C1802B
:10F3000070470368B3F17F4F05D18088A0F1FE03F9
:10F310005842584170470020704708B50246FFF731
:10F32000F0FF38B19079FB289ABF80F00200C0F35B
:10F330004000002008BD08B50246FFF7E2FF20B1FB
:10F340009079A0F1FC035842584108BD08B5014628
:10F35000FFF777FF40B90846FFF77CFF20B9BDE80B
:10F3600008400846FFF7E7BF08BD08B5C288FFF7A9
:10F37000C8FF38B150BA00F57C7080B21F288CBF2E
:10F380000020012008BD026842B9436833B9826891
:10F3900022B9C068B0FA80F0400970470020704779
:10F3A00002684AB943683BB982682AB9C06800F16B
:10F3B0007F4358425841704700207047038848F205
:10F3C000FE0023F47C531B1A5842584170476FF0DB
:10F3D0000102002302706FF07F0242708370C370DD
:10F3E000037143718371C3710830FFF74FBF6FF032
:10F3F0000102002302706FF07F0242708370C370BD
:10F40000037143718371C3710B6883604B68C36080
:10F410007047000030B5074C034604F11005224642
:10F4200003CAAA4218605960144603F10803F6D1D2
:10F4300030BD00BF885E070030B5074C034604F1BD
:10F440001005224603CAAA4218605960144603F107
:10F450000803F6D130BD00BFB05E070030B5074CE1
:10F46000034604F11005224603CAAA4218605960F7
:10F47000144603F10803F6D130BD00BFC45E070097
:10F4800030B5074C034604F11005224603CAAA42D0
:10F4900018605960144603F10803F6D130BD00BF6F
:10F4A000D85E070010B50C7CE21DD208FFF78AFE7B
:10F4B000A04234BF0020012010BD10B51446073211
:10F4C000D208FFF77FFEA04234BF0020012010BD0C
:10F4D0000B6803604B6843607047F8B5D40802F0CE
:10F4E0000707224605460E465DF042FB67B1013F25
:10F4F00080233B412A5DDBB2591E0A402A55315D0B
:10F500005B420B401A432A55F8BD0A7C402A04D9B5
:10F51000403AD2B20831FFF7E0BF70470A7CFFF7EC
:10F52000DCBF38B5044615460430FFF7D6FFE5705A
:10F5300038BD0B6803604B6843604FF0FF31002318
:10F54000C17252BA6FF00101037243728372017388
:10F550004373C281704708B50278FF2A03D140780F
:10F5600000F00F0008BD038848F2FE0223F47C532C
:10F57000934206D0FFF714FF002814BF00200E208E
:10F58000F0E70220EEE708B50378FF2B05D1FFF77F
:10F59000E2FF831E5842584108BD0020FCE708B531
:10F5A0000378FF2B05D1FFF7D6FFC31E5842584101
:10F5B00008BD0020FCE708B50378FF2B06D1FFF754
:10F5C000CAFF032894BF0020012008BD0020FCE7EB
:10F5D0001022FFF7BBBD022910B504460BD003294A
:10F5E0000FD0012911D1FFF7CEFE80B92078FF3866
:10F5F00018BF012010BD0078A0F1FF035842584108
:10F60000F8E7BDE81040FFF7D6BF0120F2E7002081
:10F61000F0E770B50546087C0E461446FFF704FE79
:10F6200000B9FEE71022002128465CF0BDFE3146FD
:10F630002846FFF773FF337C621EDB080334082B78
:10F6400012F8010F14BF194609214B1C944268544B
:10F65000DBB2F4D170BD2DE9F3470B783A2B0746A6
:10F660000D4690461FD14B783A2B03D0062002B0AE
:10F67000BDE8F0870235002100262A784245F3B222
:10F6800066D0AE464FF0000C70461EF8014BA4F158
:10F690004102052A09D8373CE2B202EB0C1CBCF54A
:10F6A000803FF1D3E2E7FF21E6E7A4F16102052AFA
:10F6B00001D8573CF0E7A4F13002D2B2092AECD9C4
:10F6C0008542D3D02E2C1ED1062BCFD836D04FF06A
:10F6D00001090624FF29C9D05B1AD8B2034607EBFB
:10F6E000410A201A5A00514607EB40005CF042FEE6
:10F6F000A21B5200002150465CF056FEB9F1000FEB
:10F700001CD10020B3E73A2C01D0A045AED1082E81
:10F71000ACD09CFA9CFC27F816C0027801333A2A38
:10F72000DBB203D142783A2A03D0013001360546D4
:10F73000A3E7FF299AD102301946F7E74246294646
:10F7400001A8FEF72EFE002891D1019BFB608EE7F9
:10F75000082BD6D04FF000090824BBE70022FFF7A2
:10F760007ABF00002DE9F843DFF83890DFF83880E1
:10F7700006460D4617460024A74210D014F0FF0F8E
:10F7800003D049462846F9F7E8F936F814305BBA51
:10F790009AB241462846F9F7E0F90134ECE7BDE8B2
:10F7A000F88300BF8C700700423407002DE9F04158
:10F7B000027C073288B0D210013203AE04460D46F7
:10F7C0005208034600F1100CB046186859683746D5
:10F7D00003C7083363453E46F7D101921B783B705F
:10F7E0004046FFF7D9FC019A2946FFF7BBFF237C6F
:10F7F0000733772B03D806492846F9F7AEF9227C60
:10F8000004492846F9F7A9F908B0BDE8F08100BF1E
:10F81000805E0700835E070013B504466846F9F76B
:10F8200074F969462046FFF7C1FF02B010BD0822F7
:10F83000FFF798BF38B5282204460D4600F10801AD
:10F84000F9F763F928462146FFF7F1FF204638BD56
:10F8500013B504466846F9F758F969462046FFF79C
:10F86000E6FF02B010BD08B510225EF011FCB0FA40
:10F8700080F0400908BD000030B591F8314014F027
:10F88000010491B0054603D00124204611B030BDDB
:10F8900001A8FFF70DF90028F7D107A8FFF78EFDA3
:10F8A00010B3154A45F2A963D35C002BECD001A834
:10F8B000FFF764F99DF80A20062A05D0112AE4D141
:10F8C00044F64C539842DFD02A792B4605EB42028E
:10F8D0009A421C460ED02188814203F10203F7D1DF
:10F8E000003C18BF0124D0E707A8FFF74CFE002812
:10F8F000D7D1CAE70024F3E708370020F0B5044663
:10F900000AB3037900EB4306864205461FD02F88D1
:10F91000974200F10200F7D159B1E3B1013BDBB2EC
:10F9200023711AB204EB43039D421CBF34F812301A
:10F930002B80002105E0022B07D0581C207124F8F1
:10F9400013200846F0BD0721FBE70321F9E7002952
:10F95000F1D01721F5E71B88FFDE037803F0F003F1
:10F96000602B09D1808840BA80B22830B0F5A06FF2
:10F970008CBF0020012070470020704770B50E46F4
:10F9800002460546282300213046F8F7A2FB04462C
:10F9900068B92846FFF7E1FF48B1AB88F28B5BBA44
:10F9A0009BB22833934218BF0624204670BD06241C
:10F9B000FBE7037813B140780230704701207047AD
:10F9C0002DE9F0410F46154606460246984629465F
:10F9D00001233846F8F77DFB044610B934781CB98A
:10F9E00074702046BDE8F08102233246294638462D
:10F9F000F8F76FFB04460028F3D13046FFF7D9FF34
:10FA000028444045C8BF0624EBE7002301290360D2
:10FA100018BF0239C0F8033017BF01230370037009
:10FA20004170704711F0070108B506D0C1F1080117
:10FA3000C9B2FFF7EAFF002008BD1820FCE700006C
:10FA400010B503460021074A80F88C10C0F89010CA
:10FA500043F8942F0446C0F89C308C225CF0A4FC40
:10FA6000204610BDE1FE000038B50C4605460E49A3
:10FA7000104610225EF00CFB6D23237048B9022360
:10FA80006370A07095F88C305A1C85F88C20E37058
:10FA900038BD042363704023A370044A45F2B86361
:10FAA000D35A5BBAA380EDE7688F002008370020A7
:10FAB0002DE9F84300250F46904606460446844645
:10FAC0002A462B46294696F803E0BEF1000F09D1DD
:10FAD00000EB8504002908BF2146E578002D46D0BB
:10FAE0007BBBFEE7B6F800E0BCF80090CE450BD03B
:10FAF000B94503D111B90133DBB23146934284BF1A
:10FB00001A4664460023B446BE4512D196F802E078
:10FB1000C64505D100EB85000523C37002203BE0FC
:10FB200039B9A8EB0E0E1EF0800F1EBF0133DBB2F9
:10FB3000314601350133232DDBB206F10406C2D173
:10FB4000CBE7BCF80050BD4204D119B9013300F134
:10FB50008C01DBB29A423CBF1A466446012ADDD9C9
:10FB600081B18142DAD931F8043CBB42D6D1234677
:10FB700099420C4612D2814200D2FEE75A1A081D61
:10FB80005CF0F8FB05230A48278084F80280E370C4
:10FB9000082116F025F80020BDE8F883F2D9834249
:10FBA00000D2FEE70C1FE21A191D1846E8E700BF55
:10FBB00058370020002330B4014600F18C051C4664
:10FBC000CA785AB900EB83000022222B13DCC178DB
:10FBD000043081B100F8012C0133F6E7013AD2B2CA
:10FBE000CA7022B10A6840F823200124013304318D
:10FBF000A942E5D1E6E724B930BC0348082116F054
:10FC000007B830BC704700BF58370020044A45F29F
:10FC1000A963D35C033B012B94BF022000207047F3
:10FC20000837002002460846C98B0B2900D8FEE79A
:10FC30000C390C2389B2F8F74CBA0846C98B0C3939
:10FC400008B589B2F8F78BF900B1FEE708BD0246A6
:10FC50000846C98B0C390C2389B2F8F769BA70B51C
:10FC600005460E46144652B111460020F8F7A6FE8E
:10FC70002B7A03443344241A2B602C7270BD104637
:10FC8000F6E72DE9FF411F46002306460D46904644
:10FC90008DF80330FFF7BAFF002847D0C98B2846FC
:10FCA000F8F728FD0446002840D095F8323013F0CC
:10FCB0000C0F14D101230DF1030207212846F8F798
:10FCC00008FA9DF803305A1E012B8DF8032030D915
:10FCD00001230DF1030207212046F8F729FA95F8D0
:10FCE0003230ADF8088013F00C0318BF01238DF8F3
:10FCF0000B3000238DF80C308DF80A70F5F759FFA2
:10FD00004022014601A8FFF7AAFF0C2201A92046C4
:10FD1000F8F731FA68B9214606F190000122F8F7A8
:10FD200068FB019906F19400F9F767F804B0BDE8A3
:10FD3000F0812046F8F70FF9F8E7F0B50D4685B0E9
:10FD4000114607461E4602AA042328460191F8F7E9
:10FD5000C0F90446B0BB9DF80A30019903F0C00217
:10FD6000402A27D016D8CAB1BDF80C109DF80B2038
:10FD700049BA89B23846FFF79BFE044628BBBDF856
:10FD80000C209DF80B3052BA92B229463846FFF744
:10FD900078FF17E01B06E7D5062413E006F10800FC
:10FDA000FFF7AFFAD0B1B37BF27B43EA0223ADF8A1
:10FDB0000C30D9E7062302AA2846F8F78AF9044648
:10FDC0000028D1D0204605B0F0BD95F8323013F0B0
:10FDD0000C0FF7D00A9B00241C70F3E70224F1E714
:10FDE0002DE9F04F87B00746F5F7E3FE07F19009DC
:10FDF00000F100468046494601A8F8F7A7FB013EFE
:10FE0000DFF8D8A03546019C002C5CD0214603A821
:10FE1000FFF708FF039BA8EB0302002A08DAEA1A9F
:10FE200015EA220538BF1D4601A8F8F79EFBEAE750
:10FE30009DF813100131C9B238468DF81310FFF741
:10FE4000E5FE814204D921464846F8F717FBEBE767
:10FE500033D24022414603A8FFF701FF214603A801
:10FE6000FFF7F5FEDDF80CB0E18BA5EB0B022046A9
:10FE70003BEA220B28BFAB46F8F73CFC0446D0B166
:10FE80009DF81320012A81BF94F83020052363F3E5
:10FE9000C60284F83020214603A8FFF7CEFE94F86E
:10FEA000322022F00D0242F0050284F83220214671
:10FEB0005046FEF7ADFB5D46B6E721464846F8F7EB
:10FEC000B8FAAB46DCE7AE1B002E04DA294607F190
:10FED0009400F8F775FF07B0BDE8F08F8887002021
:10FEE0000148FFF77DBF00BFC0870020002370B529
:10FEF0000E4615461360044644B110223146204692
:10FF00005EF0C6F810B12C602469F5E7204670BD9C
:10FF1000002370B50E4615461360044644B1102206
:10FF2000314620465EF0B4F810B12C606469F5E704
:10FF3000204670BD0023C0E90033C0E903330372DB
:10FF4000436100F1780100F11803994204D042693D
:10FF50005A6143611833F8E70023C0F88C3000F190
:10FF60007C03C0F8A03000F190038367704707B5A9
:10FF7000406801AAFFF7BAFF003818BF012003B09C
:10FF80005DF804FB0129F7B50D4604461F460CBF7A
:10FF90004FF480514FF400510E481646F8F758FCC4
:10FFA000B7B9E368A3B1802330468DF804300096DA
:10FFB000FFF7D1FA9DF8053000F00F0023F03F0362
:10FFC00003438DF805302946D4E903326846984743
:10FFD00003B0F0BD30370020F8B506460F46144692
:10FFE0001D46AC4207D02246002339463046FFF773
:10FFF000C9FF2469F5E7F8BD42680B49002392B1B7
:020000021000EC
:100000008A420CD013461269F9E72BB943600023EA
:10001000054A1946FFF7E0BF00221A61F7E7034AD5
:100020009342F2D1FEE77047885E0700C45E070086
:1000300043680B49002223B18B4203D01A461B6947
:10004000F9E7FEE7074B9A4209D0074B2AB943600C
:10005000034B054A0121FFF7BFBF1361F8E7704763
:10006000885E0700C45E0700B05E070043680A4967
:1000700000227BB18B4204D01A461B69F9E7136159
:1000800003E0064B002AFAD14360044B024A0021E8
:10009000FFF7A2BF704700BFB05E0700885E070091
:1000A00043680C491A4652B18A4211D01269FAE7E4
:1000B0001A461B69002BFBD1064B136103E0002B92
:1000C000F6D1044B4360034A00230121FFF784BFAC
:1000D000704700BF885E0700426813461BB1994213
:1000E00007D01B69FAE70A6141600A460121FFF760
:1000F00049BF7047F7B50B78FF2B05460C4629D151
:10010000406801AAFFF7F2FE30BB164E10222146CE
:1001100030465DF0BDFF08B33669002EF6D1AA6FF8
:10012000F2B11369AB671646234604F1100718684D
:100130005968344603C40833BB422646F7D16B687E
:10014000094813614FF480516A60F8F781FB002081
:1001500003B0F0BD0720FBE71820F9E72520F7E7FB
:100160000320F5E7B05E07003037002073B5937CBD
:10017000DB0904460D46164633D001290CBF202169
:1001800040211C48F8F764FB04F118039E4203D396
:1001900004F178039E4222D3E36803B3337C8DF8E5
:1001A0000430B37C00965A0720D5C3F3C300B37C58
:1001B000C3F3000200F00F03F07C43EA0213C0F324
:1001C000000043EA40139DF8050020F03F00034380
:1001D0008DF805302946D4E903326846984702B0C5
:1001E00070BD01290CBF01210221CAE73046FFF78B
:1001F000B2F9DCE73037002038B5CB7CDB070546A9
:100200000C4603D50A492046FFF762F92A681346CF
:100210001BB19C420AD05B69FAE7626128462C60F8
:1002200022460121BDE83840FFF7A0BF38BD00BF1E
:10023000308F0020036837B50C461546CBB19C4281
:1002400012D05B69FAE7224600210190FFF78EFF8A
:10025000A37C019865F3000322460121A37403B037
:10026000BDE83040FFF782BFA37C03F00103AB423F
:10027000E9D103B030BD2DE9F3410B78FF2B0546E2
:100280000C4603D1072002B0BDE8F081006801AA46
:10029000FFF73EFEC0B105F118039842F2D378355E
:1002A000A842EFD2237C0374637C4374A27C837CDA
:1002B00062F300038374A37C827CC3F3400363F383
:1002C000410282740020DEE72046FFF777F800281D
:1002D000D8D16E69AEB173696B610FCC37460FC769
:1002E00094E8030087E80300738A23F46073738241
:1002F0002B68736132462E6001212846FFF736FFD6
:10030000E0E70320BFE707B5006801AAFFF700FE9A
:10031000003818BF012003B05DF804FB2DE9F0415F
:1003200004681D4E0546B4B1E37CDB0711D52246B7
:1003300000212846FFF71AFFE37C6FF341033146A3
:100340002046E374FFF7C4F8224601212846FFF750
:100350000DFF6469E7E7114E6C68A6F1500706F1DE
:100360001408B4B1B44201D0444510D10023194659
:1003700022462846FFF706FE402239462046FFF770
:10038000D0F80023224601212846FFF7FBFD24690F
:10039000E7E7BDE8F08100BF308F0020808F0020AC
:1003A00010B51822044600215BF0FEFF014B2361CB
:1003B00010BD00BF4000030010B50446FFF7F0FF7A
:1003C000638A23F4BE7343F48E73638210BD70B5E9
:1003D000144605460E461822002144F002045BF044
:1003E000E3FF04F0030401232E746B74AC7470BD3E
:1003F00038B505460C467CB16B6803F17C0294422B
:1004000001D22469F7E7A4339C42FAD2297A204624
:10041000FFF7E1F80028F4D02C6038BD10B50023B8
:10042000C0E90031044602724968FFF7E1FF204647
:1004300010BD034621B9006830B102691A607047E7
:10044000086908B103690B617047436870B50D46D0
:10045000044600217BB19D4202D019461B69F9E791
:10046000201DFFF7E6FF00232A4620461946BDE877
:100470007040FFF787BD70BD37B5044601AA4068DC
:10048000FFF734FD0546B0B104F17C03984214D364
:1004900004F1A403984210D20199201DFFF7C9FF6F
:1004A00007484FF40051F8F7D3F9A36F2B610020F0
:1004B000A56703B030BD1720FBE72520F9E700BF93
:1004C000303700204168F8B5044600F17C0600F1A1
:1004D000A40749B1B1420D6904D3B94202D2204602
:1004E000FFF7CAFF2946F4E7F8BD034621B90068C3
:1004F00030B142691A607047486908B143694B617D
:10050000704738B503680C460546002193B19C42FC
:1005100002D019465B69F9E72846FFF7E6FFE37C5E
:100520006FF34103E374224628460021BDE83840BA
:10053000FFF71CBE38BD37B5044601AA0068FFF7B7
:10054000E7FC0546B0B104F11803984214D304F156
:100550007803984210D201992046FFF7C6FF204643
:100560002A460021FFF702FE63696B610020656186
:1005700003B030BD1720FBE72520F9E7F8B50546A5
:10058000044655F8181B00F1780749B1A9424E6995
:1005900004D3B94202D22046FFF7CDFF3146F4E73B
:1005A000F8BD000030B504468DB00D4601466846E2
:1005B000FFF740F9238A034902AA2846F8F7CDFA43
:1005C0000DB030BDEC5E070013B504466846F8F781
:1005D0009CFA69462046FFF7E5FF02B010BD000017
:1005E0000246074942F8041FC260064A026100221F
:1005F000C0E90522C2614FF440420284704700BF47
:10060000990C0100C90C0100F0B5034690F85500A3
:100610008BB00C4698BB12F0010FD3F8C81004F150
:1006200010071AD021F00041C3F8C810224605AEC9
:1006300010685168354603C50832BA422E46F7D1D4
:10064000228A01A952BA1846ADF80C201AF09CFD76
:10065000003818BF01200BB0F0BD41F00041C3F8D5
:10066000C810224603F1400152F8045B41F8045BD4
:10067000BA42F9D1228A52BAA3F85220EBE70D20F0
:10068000E9E738B500F511750C4600F514722946F6
:1006900018301AF070FF2560002038BD70B500F1E9
:1006A0001806054630460C461AF018FFA0420BD338
:1006B00064B1214630461AF04CFF28461AF0EBFD93
:1006C000003818BF012070BD0120FCE72046FAE782
:1006D00008B51AF0F3FD003818BF012008BD08B5B1
:1006E0001AF038FE002008BD45F2701310B50468FA
:1006F000E15800220B466BB198420DD01A46D3F850
:100700001832F8E7D2F8183273B1D3F81832C2F8B9
:10071000183209E0172010BD002AF3D121B145F2AB
:100720007013D1F81822E2500024C0F818421AF0D1
:1007300011FE2046EFE700000238C0B20E289ABF33
:10074000014B185C00207047F45E0700032938B5A0
:1007500005460C4600D9FEE7022911D0032911D025
:10076000012906D001211AF019FB003818BF012019
:1007700038BD02211AF012FB30B904212846F2E7F5
:100780000821F0E71021EEE72046F1E770B50546B5
:100790000E461446F5F70DFA21183046FFF7CCFF48
:1007A00005EB8000C0F83412286800F5A240BDE8CF
:1007B00070405C30F8F721BB2DE9F74F04468846BE
:1007C00091461F46002500F50D7A4FF0010BE9B266
:1007D00020460191FFF7BAFF064690B35AF825303C
:1007E000A8EB0302002A23DB022D19D0019903296B
:1007F0001AD0012907D020461AF018F908B330465C
:1008000003B0BDE8F08F022120461AF0C7FA18B1F4
:1008100020461AF00FFAF1E720461AF077F9EDE7D3
:1008200020461AF01FF9E9E720461AF0CDF9E5E76E
:100830003A6889F800B0D11A33EA210328BF134679
:100840003B600135042DC2D10026D8E710B504461F
:1008500008301AF0E1FFD4E933329B1A184410BD76
:1008600037B590F86E4214F0040405460ED0D0F867
:1008700028425CB108301AF0CFFF01902846FFF7FC
:10088000E5FF019902462846A0470124002320469F
:1008900085F86E3203B030BD70B50E46154604467D
:1008A000FFF7D4FFA919814210D9D4F828326BB1CF
:1008B00094F86E32206843F0040300F5A24084F8F7
:1008C0006E326830BDE87040F8F7D6B970BD2DE9DA
:1008D000F04304468DB00D469146FFF7B7FFD4F8BC
:1008E000C830D5F80880002B074624DA04F140030D
:1008F00007AA04F1500C18685968164603C6083355
:1009000063453246F7D1B4F85230ADF8143003AB3A
:1009100000932A46002309F0010120461AF066FCE4
:10092000054650B920463A464146FFF7B5FF2846EE
:100930000DB0BDE8F0830023EAE70120F8E72DE9D8
:10094000F04104468CB00E4602F00108FFF77EFF2E
:10095000A36807464BB3D4F8C830002B23DA04F160
:10096000400507AA04F1500C28686968134603C3C0
:10097000083565451A46F7D1B4F85230ADF8143051
:1009800003AB009300223346414620461AF02EFC6A
:10099000054660B920463A463146FFF77DFF2846B6
:1009A0000CB0BDE8F0810023EBE70D20F8E7012053
:1009B000F6E770B590F8553004460D460BB90020A7
:1009C00070BD0B8CB0F850205BBA9BB29A42F6D146
:1009D0004B8CB0F852205BBA9BB29A42EFD100F137
:1009E00030063046FEF7CFFC30B91022294630469B
:1009F0005DF04EFB0028E2D11022A91804F140005E
:100A00005DF046FBB0FA80F04009D9E738B50D46F5
:100A100045F27411034669580C462CB1A34201D02B
:100A2000E469FAE7182038BDD96145F27411184617
:100A30006B50116819625168926859629A62214636
:100A40001C225BF0B1FC45602046ECE710B510229B
:100A50000446002108305BF0A7FC002020832060C2
:100A600010BD45F2741310B54468E15800220B46DE
:100A70004BB1984209D01A46DB69F9E7D3695BB1FB
:100A8000DB69D36108E0172010BD002AF6D119B147
:100A900045F27413CA69E2500023C3611846F3E7B4
:100AA00038B50368012B0D4614D10B8C028B5BBA51
:100AB0009BB29A420ED100F108042046FEF763FC77
:100AC00038B91022294620465DF0E2FAB0FA80F0EB
:100AD000400938BD0020FCE72DE9F0410D8A866908
:100AE0006DBA07460C46ADB2D6B1B6F85030AB423F
:100AF00002D0D6F81862F7E72046FEF744FC60B94A
:100B000006F130084046FEF73EFC30B9102221467F
:100B100040465DF0BDFA0028EBD10020BDE8F08131
:100B2000FE69C6B1338BAB4201D0F669F9E72046C6
:100B3000FEF729FC0028F0D106F108073846FEF739
:100B400022FC0028E9D11022214638465DF0A0FAA7
:100B50000028EAD1E1E70120E0E738B5054608467C
:100B60000C46FEF710FCC0B9286800F5A2402146EB
:100B70005830FFF7B1FF90B1234605F1300204F180
:100B8000100153F8040B42F8040B8B42F9D1238A6D
:100B90005BBAA5F85030002038BD0720FCE70D20D7
:100BA000FAE770B5054640680E8A00F5A240583055
:100BB0000C46FFF791FF80B1214605F1080304F1CF
:100BC000100251F8040B43F8040B9142F9D176BAA4
:100BD00001232E832B60002070BD0D20FCE7000058
:100BE000F8B504469DF8186015467BB11748FDF727
:100BF000A3FD034608B90020F8BD2A4600F1100104
:100C000053F8040B42F8040B8B42F9D1BEB14FF4F8
:100C100080464FF6FF77238C2B82BB421ABF0133ED
:100C20009BB24FF44043238429462046FFF754FFEC
:100C30000028E1D1013EB6B2002EECD1DBE7294617
:100C40002046BDE8F840FFF747BF00BF8887002077
:100C5000F7B50446F4F7ADFF00F100470646013F43
:100C60000023A5698DF8033001975DB101AB0DF14B
:100C7000030231462846FFF79FFD0028F0D1D5F842
:100C80001852F2E79DF803301BB10199201DF8F7C7
:100C9000B4F803B0F0BD00000148FFF7D9BF00BFB2
:100CA0006088002038B58469054664B12046FFF7A6
:100CB000D7FD28B105F11000BDE83840F7F7DCBFDB
:100CC000D4F81842F1E738BD0148FFF7EBBF00BF89
:100CD0006088002008B5002100F5A140FDF7B8FBB1
:100CE00028B190F8313043F0010380F8313008BD6D
:100CF0000846F7F730B9062300F5A140FDF7EEBD31
:100D0000F4F757BFFFF7FCBFFFF740BD7047D0F8BF
:100D100030325BB16F2905D0742905D0002918BF86
:100D2000022118470121FCE70421FAE7704770B55A
:100D300004460D4671B900F1180630461AF0CEFB94
:100D4000014630461AF005FC65602046BDE870405B
:100D500019F036BD70BD0FB400B5A3B024AB80212F
:100D600053F8042B019302A85DF084F923B05DF8D9
:100D700004EB04B0704700000FB400B5A3B024AB7F
:100D8000802153F8042B019302A85DF073F9034905
:100D9000034802AAF6F792FFFEE700BF1B350700E3
:100DA000035F070010B400F5A2409DF804400194D1
:100DB00058305DF8044BFFF713BF07B504210DEB66
:100DC0000100F8F7F7F9019803B05DF804FB40BAA9
:100DD00080B2704708B5FDF7A1F808BD036823B1DC
:100DE000994207D0D3F81832F9E71720B0FA80F00B
:100DF000400970470020F9E72DE9F8430F461646F1
:100E000000214FF4067204465BF0CEFA07F5A240CB
:100E100021467030FFF7E2FF054600284CD145F22D
:100E200070130146FA58C4F81822FC503368C4F80D
:100E30001C327368C4F82032B368C4F82432F368F3
:100E4000C4F828323369C4F82C327369C4F83032DC
:100E5000102204F50D705BF0A7FA2946122204F562
:100E600017705BF0A1FA84F86E52D6E90696092352
:100E700006F1080204F10800B2FBF3F2B61A1AF008
:100E800063FC3246494604F118001AF021FB16F0C3
:100E9000070118BF012109EB060801EBD601404606
:100EA000C4F828801AF069FA2046656019F088FCB9
:100EB00027602846BDE8F8831820FBE72DE9F74FA7
:100EC00000F1180528460C9F0C4616469946FFF778
:100ED00085FF002800F0998094F85530002B00F031
:100EE00094803B7B23B1D4F820320BB12046984745
:100EF00021462846FFF772FF002800F0868094F80C
:100F00005530002B00F08180D4F8243223B37B6865
:100F1000FEB14FF00008C3467B6843451CD0D6F8AD
:100F200000A0B8F1000F09D021462846FFF756FF70
:100F300000286AD094F85530002B66D0C6F800B06F
:100F40003146D4F824322046984708F10108564625
:100F5000E2E7002BDDD0FEE721462846FFF73EFF03
:100F6000002852D094F85530002B4ED0D4F82832B7
:100F7000BBB12046FFF76AFCBB6806460BB9484583
:100F80000FD204F10800D4F828821AF045FC32464A
:100F900001462046C04794F86E3223F0040384F8DB
:100FA0006E3221462846FFF719FF70B394F855308A
:100FB0005BB37B7B0BB9BB7BABB1D4F82C6296B136
:100FC00004F1180738461AF089FAE26A01900132F2
:100FD00018BF0122384600921AF082FADDE900219A
:100FE00003462046B04721462846FFF7F7FE60B18A
:100FF00094F855300A2B08D1D4F830322BB10321A4
:10100000204603B0BDE8F04F184703B0BDE8F08FAD
:101010002DE9F04F2DED028B98468B885BBA1FFAB5
:1010200083FB8946D38B118C5B1A9B459BB0824610
:10103000154606D0062420461BB0BDEC028BBDE849
:10104000F08FBBF1130FF5D90C3101230DF11B0209
:1010500089B22846F7F73DF804460028EBD19DF801
:101060001B301B119B00A3F11402D2B2282A8DF869
:101070001B30DFD89B45DDDB06224146284615F0B4
:101080003BFF04460028D6D19DF81B30298C0BAAC3
:101090002846F7F71EF804460028CCD10C98FCF738
:1010A0003DFF0C900D98FCF739FFBDF83A30DAF8A7
:1010B00018600D905BBAADF83A30BDF83E305BBABF
:1010C000ADF83E30BDF82C305BBAA8F82230BDF840
:1010D0002E305BBAA8F820303EB141463046FFF7CB
:1010E00068FC90BBD6F81862F6E7DAF81C70F7B126
:1010F00041463846FFF7D4FC40B9FF69F7E7079946
:10110000002998D0002300961A4646E007AE102228
:10111000002130465BF048F9CDE9007600232A46ED
:101120000BA9484617F070FF0130E8D1FEE76F23A6
:1011300001939DF81B30ABEB030300933A46194B28
:101140000BA9484616F066FD75E7304607AF50F824
:10115000083F08EE103A1AF05FFBD6F8D030039043
:1011600005931022D6F8CC300493002138465BF06A
:101170001BF900230093019733462A460BA94846E2
:1011800017F042FF0130B0D0DDE903321344059A75
:1011900000979B1A18EE102A31465046FFF78EFE34
:1011A00049E700BF083700202DE9F043D0F8288038
:1011B00087B006460D46B8F1000F24D001AFD1F834
:1011C0000090144602F1100E3A4620686168BC4651
:1011D000ACE80300083474456746F6D15BBA29468B
:1011E0003046ADF81430C04709F5A24029467030AA
:1011F000FFF7F4FD20B195F85500003818BF012025
:1012000007B0BDE8F0830120FAE72DE9F041D0F8FE
:10121000248086B00446B8F1000F04D14FF0FF30AF
:1012200006B0BDE8F08101AE45680B4601F1100E35
:10123000B44618685968374603C7083373453E46B5
:10124000F7D152BAADF8142061466A462046C0472D
:1012500045F27413EB58002BE0D09C4210D0DB69B0
:10126000F9E7009C05F5A24021467030FFF7B6FD76
:101270000028D3D094F85530002BCFD12046CFE7AB
:101280002368002BCAD00028EBD0012814BF4FF0F0
:10129000FF300020C4E70023C0E90012C0E9023398
:1012A00080F828307047C3688B4230B500D2FEE723
:1012B000D0E901425B1AA51AAB4221BF1B1B9B1848
:1012C000836090F82830C16035BF9B18C3F10103DB
:1012D000836080F8283030BD4268C068101A7047BB
:1012E0000023C0E9023380F828307047C368002B20
:1012F00014BF05200020704743688B4200D8FEE7EA
:101300008818591A914298BFC01A70472DE9F84FB2
:10131000D0F804B09246C268ABEB02094B4528BF37
:101320004B4604460F461D46002B68D002B982602A
:10133000A1682046FFF7E0FF0B9B13F0010806466B
:1013400005D04D452CBF4FF000084FF00108206834
:10135000ABEB06094D45304429D82A4651465BF08F
:1013600007FCF6B9E26894F8283012B1C3F1010322
:10137000DBB20C2101FB0342002010612068114602
:10138000C2E90505103142463846FFF7A0FA0028A9
:1013900018BF0025E3682B44E3600A9B1D60BDE88D
:1013A000F88F424629463846FFF7C9FAEFE7A5EB22
:1013B0000B0B4A4651465E445BF0DAFB32460AEBC1
:1013C000090120685BF0D4FB012249463846FFF74B
:1013D000B6FAB0B994F82810C1F101030C215943B1
:1013E00063181031186122682144C3E90526384684
:1013F0004246FFF76CFA002818BF4D46CAE7184668
:10140000C8E70025C6E738B5028A0B8C9A42044625
:101410000D4601D0002038BD0B78FF2B03D1638C23
:101420006BB90120F7E7FDF7AEFF0028F7D11022D6
:10143000294620465CF02CFE0028F0D0EAE76A8CB2
:101440009A42E7D112342046FDF79DFF0028E8D1EB
:101450001022A91820465CF01BFEB0FA80F040096B
:10146000D9E710B53422044600215AF09DFF2046EA
:1014700010BD4FF4404202800022C0E901227047B3
:101480004FF2BF03984208D000F53B50213080B2A4
:1014900013288CBF0020012070470120704710B531
:1014A00084680022234683B1994207D01A461B6BF9
:1014B000F9E7136B3BB11B6B136304E0002AF8D10F
:1014C0000CB1236B836000230B6310BD028810B541
:1014D00001464FF6FF74A2421ABF013292B24FF496
:1014E00040421046FFF7CCFF0028F4D10A80104696
:1014F00010BD0000F8B5064610460D461446FDF72F
:1015000042FF88B122462B4604F11007106851684B
:101510001C4603C40832BA422346F7D112882280FF
:101520002C8A4CB10020F8BD06482146FEF7EBFEA0
:101530000028E7D10720F6E73046FFF7C7FF2882EB
:101540002046F0E78488002013460A4601460148F9
:10155000FFF7D0BFB487002030B587B004461546EA
:10156000ADF814101022002101A85AF01DFF2A46E0
:1015700001A92046FFF7E8FF07B030BD30B401F104
:10158000120302F1100452F8045B43F8045BA24218
:10159000F9D112881A800B8A23B930BC01230A467C
:1015A000FFF7A8BF002030BC704700000831024898
:1015B00089B2FCF743BF00BF888700200148FFF7CE
:1015C000F5BF00BFB487002037B5138C5BBAADF808
:1015D0000030538C5BBAADF80230CB8B08330C462D
:1015E0005BBA1546ADF80430082200236946204650
:1015F000ADF80630F6F70AFE48B901462046F6F780
:10160000D5FC044811232A462146FDF767F903B0AB
:1016100030BD00BF888700202DE9F04116461A8CA6
:101620008AB005460C4632B1098A914203D00720A0
:101630000AB0BDE8F0816A4603F1200E174618682B
:1016400059689446ACE80300083373456246F6D106
:101650001868CCF800009B88ACF8043004A8FDF7AB
:1016600092FE98B104F112084046FDF78CFE002866
:10167000DDD1434604AA04F1220E18685968944645
:10168000ACE80300083373456246F6D1BDF822305A
:1016900023B9638C002BCAD0ADF822303846FDF751
:1016A00072FE58B12346BC4604F1100E1868596802
:1016B000624603C2083373459446F7D1238A43B187
:1016C000238AADF820303A4631462846FFF77CFFA2
:1016D000AEE70123224621462846FFF70BFF0028EC
:1016E000EED0A5E713460A4601460148FFF794BF2E
:1016F000B487002070B585680C461646ADB13146FA
:101700002846FFF780FE40B92D6BF7E76B6AA86AA1
:1017100032462146BDE870401847218C2046F6F736
:101720005DFC238C002BF1D0FEE770BD2DE9F34169
:101730000D468046098C164608236A462846F6F769
:10174000C8FC044610BB11223146284615F0D4FBD4
:101750000446D8B908212846F6F71CFCBDF800302D
:10176000D8F804705BBA7384BDF802305BBA338476
:101770003FB17B68B86832462946984730B93F6820
:10178000F6E7324629464046FFF7B4FF204602B04E
:10179000BDE8F081806828B1038A8B4201D0006BDC
:1017A000F9E701207047000044F64C53994210B508
:1017B0000C460AD04FF2BF03994206D00448FBF70B
:1017C000E1FE001B18BF012010BD0020FCE700BF98
:1017D00008B6002003681BB1994206D01B6BFAE7DC
:1017E0001720B0FA80F0400970470020F9E7122274
:1017F00000215AF0D9BD2DE9F04100F10808054655
:1018000040460C4617461E46FFF7E4FF00B1FEE7D0
:101810002046FFF7ECFF04F11200FFF7E8FFC4E9F0
:10182000097621464046FFF7D5FF10B9AB68236320
:10183000AC600020BDE8F08113460A46014601482D
:10184000FFF7D9BFB487002038B5054608300C46ED
:10185000FFF7C0FF50B121462846FFF720FE204683
:10186000FFF7C5FF04F11200FFF7C1FF002038BDEC
:1018700001460148FFF7E8BFB48700200148F4F7AC
:10188000EFBA00BF083700200148F4F7F7BA00BFED
:10189000083700200148F4F789BB00BF0837002053
:1018A00048F23013C35C13B1133015F0D3BC70474A
:1018B00048F23013C35C13B1133015F0D1BC70473C
:1018C00010B448F23014045D24B15DF8044B1330B9
:1018D00015F0CCBC5DF8044B704748F23013C35C84
:1018E00013B1133015F0C8BC7047000000487047B2
:1018F00000F8FF0708B5FFF7F9FF08BDF5F7C2BB11
:1019000000207047FF207047FF207047704700009D
:1019100003685A8A4FF6FF739A421DBF47F6681351
:1019200003EB4213024A002318BF9B180360704761
:10193000083700202DE9F041D2E9007506460C4633
:1019400000F5816800F20C4106F2144C00F582604B
:101950004346B5B91FB9D6F808541F46F8E74745BE
:1019600003D1D6F80C540B46F7E78F42034602D159
:10197000D6F81054F1E7874265D1D6F8145463467F
:10198000EBE7698A4FF6FF7399421DBF47F668136C
:1019900003EB41132D49002318BF5B18C2E9007304
:1019A00000212C2220465AF0FFFC2B46A44605F1CC
:1019B000100E18685968624603C20833734594468E
:1019C000F7D12B8A238247451FD1638A23F4FF7303
:1019D00023F0010343F4807363826B69E27C01337B
:1019E00018BF012363F38202E2746B695A1C0AD0A8
:1019F0006361174904F11800FDF76AFD55F8183FB7
:101A000023626B68636200201EE006F20C439F4273
:101A10000BD10123A3742A7EE37C62F30003E374F9
:101A2000AB8A2385EB8A6385EDE706F58266B742CC
:101A300001D10223EEE70323A3746A7EE37C62F301
:101A40004103E374E7E71720BDE8F0810837002081
:101A5000308F002008B908687047438A4FF6FF723C
:101A600093421FBF47F6681000EB4310024BC018AB
:101A700008BF0020704700BF083700202DE9F04F55
:101A800087B01E4600F58163029300F20C43039376
:101A9000002500F58263DFF854B0049300F214408F
:101AA00017460590A8464FF6FF7947F6681A02AB2D
:101AB00053F825303B601C68C6F8008074B11022D2
:101AC000204601915CF0E4FA60B13460648A0199C7
:101AD0004C4503D00AEB44145C44EFE70135042D78
:101AE000E5D10024204607B0BDE8F08F083700207C
:101AF0007FB500F5816300F20C4014460293039019
:101B000002AE022556F8043B1B680193019B4BB1C2
:101B10001A8A8A4208BF1C8201A8FFF7F9FEF5E77E
:101B20000125EFE7012DFBD104B070BDF0B589B000
:101B30000E4615460021122202A8CDE900115AF0E6
:101B400033FC104A45F2AA63D35CDB0716D50E4F6F
:101B500002AA694638460FF0A5FC044670B99DF804
:101B60001A30012BF4D1102202A930465CF090FA11
:101B70000028EDD1BDF81C302B8000E01724204652
:101B800009B0F0BD0837002000B6002030B58BB09A
:101B900026220C46684600215AF006FC4FF2BF038D
:101BA0001248ADF82230022112F0A6FD0546D8B148
:101BB00022461023002114F0F6F9044640B9684685
:101BC00011F0E4FC09486A46294613F009FA044674
:101BD0000748022114F004F81CB115B12846F6F7A5
:101BE000BAF920460BB030BD0324F1E72C89002060
:101BF00058370020F0B58BB00F461646002126223C
:101C000068461D465AF0D0FB4FF2BF031D48ADF8A1
